:1000000001000000000000A0000200000AB6BD1BB5
:100010001CF09FE51CF09FE51CF09FE51CF09FE5A0
:100020001CF09FE51CF09FE51CF09FE51CF09FE590
:100030000F1D0F1284120200CC110200DC1102000D
:100040003412020044120200541202006412020030
:1000500070120200000000EA528300EA28008FE2DA
:10006000000C90E800A08AE000B08BE001704AE24A
:100070000B005AE14B83000A0F00BAE814E04FE28C
:10008000010013E303F0471013FF2FE144160200B1
:10009000841602000030A0E30040A0E30050A0E37B
:1000A0000060A0E3102052E27800A128FCFFFF8A44
:1000B000822EB0E13000A128003081451EFF2FE1E3
:1000C00004309FE503308FE013FF2FE19D0F020006
:1000D0001D48802110B549F3DAEB1C48582149F33B
:1000E000D6EB1B4800210A0006C0202117485830D3
:1000F00049F3CCEB002010BDF0B50024144F0837B5
:10010000012609E0C519686801F052FC69683000F1
:10011000884010498860641CE00039580029F1D1FA
:100120000B4F0024283709E0C519686801F040FC2E
:1001300069683000884008498860641CE0003958CC
:100140000029F1D10020F0BD00170200F00F0004DB
:10015000400E0004009000A8009100A85E48042210
:100160000621027041700271417102724172704742
:10017000F8B505F002FB002803D002F005FD0028C9
:1001800079D1554800241838046000F02CFB05F0A4
:10019000C1FA52490D5C01F0B7FD290049F3BEECEC
:1001A0004F4E2300320049F338E9401C61410504F9
:1001B0002D0C05F0AFFA4B4940000F5A05F083FBB8
:1001C000390049F3ACEC2300320049F326E9401C26
:1001D00061410004000C290000F014FB05F09AFABC
:1001E00041490D5C01F090FD290049F398EC230092
:1001F000320049F312E9401C614105042D0C05F061
:1002000089FA3A490F5C01F07FFD39001FF66F2E25
:1002100001000000FC0100A000020000CE6362307B
:1002200049F386EC2300320049F300E9401C6141A8
:100230000004000C290000F006FB082000F0F2FA90
:1002400001F06CFD310049F38EEC401C0004000C01
:1002500000F0F1FA01F062FD052149F36AEC294A48
:10026000230049F3E4E81922801861410006000EDA
:1002700000F0EFFA601E04F0DDF8FF24641C20009B
:1002800004F0D2F8200004F0DBF804F0EBF804F0FE
:10029000FDF8402002F020FC00F0ECFA00F0E1FA5A
:1002A00019490120086004F01DF904F035F904F043
:1002B0003CF904F06FF90C2001F025FDC02001F09D
:1002C00022FD04F07FF904F08FF904F096F904F0B0
:1002D000A6F9302001F017FD0320000201F013FD04
:1002E000FFF746FF00F090F9F8BD0000B05900B0EC
:1002F0002C00000440420F001600000442000004DD
:1003000037000004C0C62D00E85900B010402DE9A8
:10031000648400EB78409FE5000094E5000050E322
:100320000300000A6A0100FA000094E5000050E3AF
:100330005E84001B080200FA0000A0E3E71500FB42
:10034000950100FA0000A0E35B0100FB5B0100FAED
:10035000000094E5000050E34C01001BAF0100FBDE
:10036000DF0100FB000094E5000050E30100000AFB
:10037000AB0100FB461600FAA90100FA00000FE1EC
:10038000BF0000E200F021E13F1500FA0000A0E309
:100390001080BDE8506600B010B500F0A3FC05F376
:1003A0009FF905F081FB00F077FC002801D00120C7
:1003B00010BD05F079FF002010BD10B5FFF7E2FE7B
:1003C00020F07EFE0400012003F0C2FF200020F098
:1003D0007BFE05F0DCF9002805D002F0DFFB0028E9
:1003E00001D002F0C6FB002010BD10B502F04AFD9E
:1003F00010BD9308002210B502E09400521C015178
:100400009A42FAD310BD064A0648002110B5FFF7FC
:10041000F0FF00F015FB00F09BF90020DCFD98C90F
:1004200001000000F80300A0000200003A8BDC8D00
:1004300010BD000060530000B0910004F8B505F055
:100440008DF90500874801680222114301600168A7
:1004500008231943016083494031CB681343CB60C3
:10046000436813434360CA6840263243CA60CB687E
:1004700080221343CB60016831430160016811435E
:100480000160416831434160416811434160764CED
:1004900020681E2188432060744FF96A2020814320
:1004A000F96204F0A6FF022005F0F5F8000604D575
:1004B0004021272005F02CF903E00321092005F055
:1004C00032F9A80703D4B86801210843B860684826
:1004D000C16B0122D2059143C163C16B0322D204D7
:1004E0001143C1630721082005F01DF903210720EE
:1004F00005F019F904F0ACFF2068E0218843206082
:1005000060691521884360616069B043606160691A
:1005100001218906884360616069052109078843D4
:100520006061E06953490840E061E06940084000CB
:10053000E061E0691027B843E06104F045F84E4AF5
:1005400010682021084310604C4A10680421884339
:1005500010604B480D21006889014018016852065F
:1005600011430160A069B043A0616068454908403B
:1005700060606168444801406160A168434A11407D
:10058000A160A1680140A160E168414A1140E160B9
:10059000E1687A039143E160E1680140E160374A34
:1005A0001820C043C03A1168014039431160394AEC
:1005B000A906116803D501400820014301E001406C
:1005C00039431160344801690904090C016141692A
:1005D0000904090C416181690904090C8161E06920
:1005E000012189038843E061E06989008843E06173
:1005F000E06909118843E061E069052109060843C3
:10060000E06104F057F8F8BD10B500F008F8234891
:100610000068002801D0FFF711FF10BD7047124895
:10062000016803221202914301604169291E42F2CE
:1006300001000000F40500A000020000237302FD89
:1006400042019143416141694200914341618169A5
:10065000C200914381610F480068016F012211437C
:100660000167016F022291430167C0300168D20621
:1006700011430160704700000023008000280080C3
:100680000029008000910090FBFBFFFF0027008005
:10069000403D0080045A00B0DFFFD5FD7FFF7FFFA3
:1006A000D5FDD5FDD5FDD7FDC03C008000220080E2
:1006B000506600B0084810B50168084B0A001031B8
:1006C00008001960111D5960242149F3FEE804490E
:1006D000022002F053FC10BD34C800B0F85900B03D
:1006E000C5380000F8B5002425001C48A7001426D2
:1006F0006643C5511A481421301849F3E6E81848F2
:1007000014211430301849F3E0E81548142128303A
:10071000301849F3DAE8114830222838C159104816
:1007200062433C301018C4608160456185610D49A9
:10073000C56101610C4901620C498562416206F3A1
:10074000EBF8641C012CD0DB0949082001F04EF9BC
:100750000849FF20401C8860F8BD0000C86600B052
:1007600064FF00B0313B00004D3D0000773F0000CA
:100770005B410000009000A80F490E4810B50860CA
:100780000F490E48086010490E48086010490F488C
:10079000086011490F4808601048802149F394E827
:1007A0000E488021803049F390E80D48802149F3BC
:1007B0008CE810BD451602003CE50004E94200004B
:1007C00040E500042D43000044E500044054890046
:1007D00034E50004A086010038E50004DCCE00B05A
:1007E000DCCF00B010B5084C00206062DF200002B2
:1007F000E0620648A06201210548490249F364E825
:1008000001206062002010BDC09B00A800ADDEEF9B
:100810005CD000B026484068C168264A1143C160D8
:10082000704700B5FFF7F6FF214840684168012294
:100830005202114341604168D20011435A6AB02B01
:1008400001000000F00700A000020000D79BBC40A0
:10085000416000BD090401431A4840688161704746
:1008600018494968CA681204120C00040243CA609D
:100870007047144949684A69120C120402434A61DC
:100880007047090401430F484068C16370470D4930
:1008900049684A68120A120202434A6070470948CE
:1008A0004068FF30413041681D22914341607047EC
:1008B00004484068FF304130416802229143416062
:1008C00070470000005A00B08F0300008FC08FE215
:1008D0001CFF2FE101210920000701600021416078
:1008E00070476848012101600021416070476648F7
:1008F000016B80221143016370477047634800B564
:100900000068002801D0FFF7F2FFFFF7EAFF00BD03
:1009100010B55F4C20F0EEEDA04221D05D490840BB
:10092000040004F07AFD262004F0C9FE0109200726
:100930000901000F08430106090E262004F0B1FE4C
:1009400004F09AFD200A4107534A490F0429117007
:1009500001DD04211170000702D5107840421070AB
:1009600010BDFF20C130202100B504F05AFF00BDAA
:1009700010B54A4C207900280BD10120207104F0D9
:1009800066FF062004F09BFEC006C00F607104F0F5
:1009900050FF607910BD70B50600FFF7E9FF404DCC
:1009A0002C0D002811D004F052FF8021262004F0E5
:1009B000C3FE04F03EFFA8682043A8603948816860
:1009C000220211438160002003E0A868A043A860D0
:1009D000300005F095F870BD10B507F07DFA04F011
:1009E000F2FC02F0C9FE7D24E4010021200004F0A5
:1009F000F2FC0021200004F0F1FC0021200004F0B2
:100A0000F0FC0021200004F0EFFC274C0221200024
:100A100004F0E4FC0221200004F0E6FC234C6068B2
:100A2000234908406060E068172149020843E060FC
:100A300004F0A8FE2168C2061E4801D5014300E06B
:100A40008143626862602160216801432DB467A51B
:100A500001000000EC0900A0000200001082BE1D91
:100A600021600F480068002802D0B520FFF79DFFE5
:100A700010BD7047704710B504F04FFF0C4C0028B4
:100A800002D005F09AF801E005F0A6F8E06010BD8C
:100A90000F490E4808607047003000A8400C0090D5
:100AA000506600B0FFFF00003F0F0000005A00B08A
:100AB000C85A00B08028008040230080409C00007D
:100AC00000210080FF7FFF7F000000208B58000086
:100AD0004C5C00B0F8B5324800680002000F0828EE
:100AE00028D1304C6069E5042843606160694000AA
:100AF0004008606120680826304320602068EF12BB
:100B0000B84320604821452004F0D5FD0421482049
:100B100004F0D1FD20683043206020683843206015
:100B2000322004F0ECFE60692843606160692105B1
:100B300008436061F8BD1C4810B5006800282DD03E
:100B400004F08FFEFFF7C6FF2021192004F0FEFD00
:100B50000221162004F0FAFD2F21332004F0ABFD12
:100B60000321572004F0A7FD9221242004F0A3FDC7
:100B70006221252004F09FFD262004F0AAFD8008B4
:100B80008000022108430106090E262004F093FD8F
:100B90006621412004F08FFD04F055FE10BD0000D9
:100BA0000020008000280080506600B070B5444CE2
:100BB000444D2068444E002808D0E817306070602B
:100BC00004F0D4FF286A4000400828623D48C0383D
:100BD000816A090C09048162816A8B2292001143A7
:100BE00081623A4900208860900639490122120446
:100BF000036880188842FBD3002001688018904267
:100C0000FBD30120800600682068002855D004F03E
:100C100028FE0F21622004F04EFD1021332004F045
:100C2000A0FD04F010FE706B0121C902084370633F
:100C30003068632188433060F06826490840F060DE
:100C400004F0F5FB07210D2004F08BFD07211B208C
:100C500004F087FD04211B2004F078FD97097F41F3
:100C600001000000E80B00A000020000E46A00A000
:100C70004021252004F074FD4021172004F070FD70
:100C8000022004F030FD400603D540210B2004F083
:100C900067FD04F005FC04F089FD800604D4F068CB
:100CA000012189038843F0601048C168104A11404F
:100CB000C160C1680F4A1143C1602068002806D096
:100CC000012040046862801CA8620B48E862002092
:100CD00070BD0000506600B0C09000900021008000
:100CE00000230080000001B0C0FFFF7F802800804B
:100CF000F0F0FFFF0A0A00000202020000B50D49F1
:100D0000002087B00860020001001E2003AB07C36B
:100D100002000948FF21491C6B4607C3A838074A4F
:100D2000002307A103F3EEFB0006000E00D0012014
:100D300007B000BD9C0E0004EC1600044F620000DA
:100D400049646C650000000010B5FFF7E9FC06F08F
:100D5000ACFD07F035FA07F069FA10BD11483C21E7
:100D600010B548F3D0ED0F4800210160416081606B
:100D70008161016201630C4A4163C2620B4C816371
:100D80000B48EE22210048F31AED0948094B0422D2
:100D900021003EF3FEF810BD10B500F00DFB002061
:100DA00010BD00005CD6000483880000DC05000054
:100DB00068100004E3EE3300F8B5C54C20680C253C
:100DC000A8432060C348C168820C1143C160C16858
:100DD000072252021143C160C16801221206114369
:100DE000C160C16889098901C160C168C20D9143B0
:100DF000C160C168C20C9143C160C1685603B14370
:100E0000C160C1680722D2069143C160C168F21077
:100E10001143C1600168B04A114301607D20002187
:100E2000400204F0ECFA7D27FF010021380004F0B5
:100E3000ECFA0021380004F0E5FA0021380004F053
:100E4000E7FAA649086A1022104308622068A843FE
:100E50002060606851068843606004F015FFA06858
:100E6000B1000843A0602069A90588438E386C92C0
:100E700001000000E40D00A000020000FD92DED0A1
:100E800020612069304320619A4D686800206860C5
:100E9000686819210906084368609648803001682F
:100EA0004026B143016001680F22120291430160A4
:100EB0000168032252021143016001680F221203EC
:100EC00091430160016803225203114301600168EC
:100ED000090909010160016806273943016020689A
:100EE00030432060206830218843206004F058FCA3
:100EF0000528206802D910210843FFE720602868F0
:100F00000121084328602868B84328607648C168F2
:100F1000020D1143C160816A31438162012004F0F6
:100F20004EFF012005F0A0FAF8BD10B505F0E0FA7B
:100F30007149088071487249000C000408607249C8
:100F400070480860724971480860734971480860C8
:100F5000734972480860744972480860744973485C
:100F60000860754973480860754974480860764997
:100F70007448086076497548086077497548086084
:100F80007749764808607849764808607849774814
:100F900008607949774808607949784808607A4953
:100FA000784808607A49794808607B497948086040
:100FB0007B497A4808607C497A4808607C497B48CC
:100FC00008607C487C4908607D497C4808607E490F
:100FD0007C4808607E497D4808607F497D480860FC
:100FE0007F497E48086080497E48086080497F4884
:100FF000086081497F48086010BD0121080010B5D4
:1010000002F07EFD04F0CCFB7C494000085A7C498C
:10101000086000F0FBF90221012002F071FDFFF7EA
:10102000D5FE0321012002F06BFD20F086EA0421A9
:10103000012002F065FDFF22724919321C2005F3E0
:1010400089FD0521012002F05BFD0621012002F04F
:1010500057FDFFF76AFF0721012002F051FD6A49A1
:10106000E1204002086020F06CEA0821012002F033
:1010700047FD65490422072020F066EAD3FC6BD2C5
:1010800001000000E00F00A000020000097A606D7E
:101090000921012002F03EFD614800210A0006C03E
:1010A0005F4A60496048614B05F3CDFE0A2101208B
:1010B00002F030FD00F0C2F90B21012002F02AFD00
:1010C00000F072F90C21012002F024FD00F0B0F8CC
:1010D0000D21012002F01EFD0E21012002F01AFD5B
:1010E000002010BD10B500F0B9F900F0F3F900F0E0
:1010F0005FF9002010BD0000002F0080002100805B
:1011000000081C200028008080260080C8E8000419
:101110003C7000B0BCEA0004056300006CE500040C
:10112000518F00005CE50004878F000060E500043B
:10113000A18F000068E50004998F000064E50004B9
:10114000C11200B098E600040D0F00B09CE6000448
:10115000651100B0A0E60004AB1100B0A4E60004E5
:10116000C71100B0A8E6000485E3000080EC00048D
:1011700097E3000084EC0004A9E3000088EC00047D
:10118000BF1200B0ACE60004AF1A00B0B0E6000435
:10119000591B00B0BCE600048F1B00B0C0E6000481
:1011A000931B00B0C4E60004BFDE00008CE6000420
:1011B0008FDF000090E60004BF630000F4F6000437
:1011C00021740000BCE50004A3580000B4E600044C
:1011D000A5580000B8E60004AB740000B4E50004B4
:1011E00065740000B8E500049B6E0000B0E50004E3
:1011F000516E0000ACE50004A363000084E6000427
:10120000B163000088E60004F363000094E6000484
:10121000000000047CE50004A833000494E5000409
:101220004C5B00B0B81B0000F0170004345900B04C
:101230000449034810B54860080005F094F810BD53
:1012400097650000705B00B01149104808601249B2
:101250001048086012491148086013491148086095
:101260001349124808601449124808601449134889
:101270000860154913480860154914480860164964
:101280001448086016491548086070477C76D99E56
:1012900001000000DC1100A0000200007761C7DD42
:1012A000F36A0000A0F50004F56A000090F5000460
:1012B0002B6B000094F50004316B000098F50004DE
:1012C000596B00009CF50004636B0000B0F500044E
:1012D0007B6B0000B4F50004A96B0000A4F50004CA
:1012E000C16B0000A8F500048D6B0000B8F5000488
:1012F0009B6B0000ACF5000410B50124A40220484B
:10130000EE22210086B048F378EA11F00BFF0DF0D1
:10131000F1F9012200210C2003AB07C30200184899
:1013200002920090174A0019002317A1019403F3B9
:1013300007F900281DD1194815A101F393FE18489B
:101340001A4A4168174881601749016100214161CB
:101350008261174AC161026241621649816205F3E6
:1013600017FB002805D11449112000F07BFB002851
:1013700002D0012006B010BD00F0D4FA0020F9E739
:10138000683C0004BD7A00004E66635461736B00D4
:101390004E6663466C6167730000000010410004F4
:1013A000F45B00B010EB00B0B97A0000B57A000031
:1013B000A17A0000977A00007D7A0000064900209B
:1013C00008807047064905480860074905480860D5
:1013D0000749064808607047C0ED00B02180000052
:1013E00004FD0004F77F000000FD0004F57F00000D
:1013F000FCFC0004084804A1016008A141600C49FC
:101400000A480860704700006D6465765F61697521
:101410007265636F7264000018ED00046D64657698
:101420005F616975706C617900000000E9890000F6
:101430009CF8000470B500240B4D04E0401940688E
:1014400000F010FB641CE00029580029F6D170BDA3
:1014500006488168FF22521C114381608168102276
:1014600011438160704700007C5C00B0009000A8D0
:1014700010490F4810B5086010490F48086011491D
:101480000F480860114910480860FFF7E7FE20F098
:1014900074E800F059FA0F490D480860831B5F108B
:1014A00001000000D81300A00002000083897960C9
:1014B0000F490E48086006F3F3FD0F490D48086018
:1014C00010BD00008964000024F60004916400004F
:1014D0001CF600049964000020F600044F2700B0B9
:1014E00024F50004671600B054F90004591A00B03E
:1014F00058F90004A9310100C0FC00047649754880
:1015000010B50860764975480860774975480860E5
:10151000774976480860784976480860784977487E
:1015200008607949774808607949784808607A49BD
:10153000784808607A49794808607B48794941626F
:101540007B4A4164794911607B4A7A4911607C4A3F
:101550007A4911607C4A7B4911607D4A7B49116060
:10156000C11D7C4AF9314A617C4A7B4911607D4941
:101570007B4A0A607C4A4A607D4A7C4911607E4A07
:101580007C4911607E4A7D4911607F4A7D49116026
:101590007E497F4A116001007E4A80310A610265FE
:1015A0007D4A4A6142657D4ACA61C265C2667C4A1B
:1015B00002677C4A0A627C4A4A627D4A7B49116022
:1015C0007D4A7C4911607E4A7C4911607E4A7D4992
:1015D00011607F4A7D4911607F4A7E491160804ACF
:1015E0007E491160804A7F491160814A7F491160BC
:1015F000804901668049824A41668049116081497B
:10160000016201648149804808608249804808601D
:10161000824981480860834981480860834982483B
:1016200008608449824808608349844802F00AFFC0
:10163000844983480860854983480860854984480F
:10164000086086498448086086498548086087495B
:101650008548086087498648086088498648086048
:1016600088498748086089498748086089498848C7
:1016700008608A49884808608A49894808608B4917
:10168000894808608B498A4808608C498A48086004
:101690008C498B4808608C49012008708C498B4824
:1016A00008608D498B4808608D498C48BB181972B9
:1016B00001000000D41500A0000200009A71A710DC
:1016C00008608E498C4808608E498D4808608F49B3
:1016D0008D4808608F498E48086090498E4888611F
:1016E00090498F48086010BD1996000034FD000431
:1016F0008790000050F4000455900000C0FB0004E7
:10170000C395000018F900041196000014F90004B4
:10171000E5A80000C8F30004C59A000040FC0004DE
:101720003DA20000BCFC000453A100003CFD0004ED
:101730001BA4000054F70004CBA4000040EB0004FD
:1017400053A6000018F600044DA70000C4FB0004D7
:10175000BFA70000E4F6000401A80000D8FC0004C4
:10176000E79B000048FC00041FA8000039A8000007
:1017700034F70004E9A90000D8E800040FAA00002B
:1017800035AA000030F500044FAA000004F8000458
:1017900085AA000058F800040BAB00002CFD0004E3
:1017A000DBAB0000DCFC00046DAC000019B30000F2
:1017B000ABAD000007C2000053C20000C5C300006B
:1017C000B1B300008CF70004C9B3000080F7000437
:1017D000FDAD00002CF7000475B300004CF80004C8
:1017E000CDC100003CF8000401B40000ECF400049A
:1017F00017B500000CF80004DDB6000040F8000446
:10180000E9B6000014F8000403B7000047B7000071
:10181000EBB9000060F80004D1B80000B1BB0000D3
:10182000A4F700048DBB000094F70004DDBB0000AA
:1018300098F7000409BC0000C0F700042DBC0000AC
:101840005CFC00042DC1000038F700040798017A01
:10185000C051320051C400002CF80004E9C400005B
:1018600098FB000443C50000C0F600046BC50000EF
:1018700030F4000491C50000B0F600045FC300001E
:1018800050F700048DC3000020F8000459C6000082
:1018900024F8000495C6000044F80004ABC600001C
:1018A000D4F90004FFC6000090F40004FBC7000058
:1018B000ACF9000419C80000A0FB0004088E1F5CEE
:1018C00001000000D01700A0000200006E9919ADC1
:1018D00009C8000058F600047DC800006CFB000435
:1018E0009FC8000048F60004EBC80000A4FC0004F8
:1018F000C5EA000429CA0000F8F70004D7CA0000AE
:1019000068FB0004FDCA000078F600040BCB000061
:1019100024E600047FCB00008CFC00048FCB000089
:1019200084FC00049FCB0000DCF60004F9CB00002F
:1019300068E900042FCC0000C4F30004054810B58A
:101940000078102804D1044904484C2207F0D0FB49
:1019500010BD0000A50E0004B20E0004E20F00044A
:101960000548064910B50078097800F029F80448C0
:101970000068804710BD0000004000AA004000AA97
:1019800074F00004074906480860084906480860E2
:10199000084907480860094907480860704700007F
:1019A0003B8F0000CCF3000401320100D4F70004A7
:1019B0000F320100D8F700041D320100D0F70004F7
:1019C000064808B502680092054A06491300080057
:1019D0000C386C3303F372FF08BD0000980E00044E
:1019E000A02101B0006600B00449054A4978127888
:1019F0000120914200D0002070470000000002A9A1
:101A0000000002A910B51FF0FCEC01F34FFD00200F
:101A100010BD10B50C0001F0DFF884490860C10763
:101A200002D02100052015E0810702D52100062003
:101A300010E0410702D5210007200BE0010702D585
:101A40002100082006E0C00602D52100092001E09F
:101A5000210000201FF04AED012010BDF1B500204B
:101A600073490E68734F340005000AE0E10706D0A1
:101A7000A9007A58002A02D00099300090476408E3
:101A80006D1C002CF2D1012803D0009900201FF01A
:101A90002EEDF8BD654910B5486001F024F910BD80
:101AA000202800D3FEE7634A80001358002B00D0A3
:101AB000FEE71150002070475F480068002800D002
:101AC0000120704702688368C1681000065141A177
:101AD00001000000CC1900A000020000A9801BF04A
:101AE000184770B55A4D6C6AE00703D0FFF2E6ED77
:101AF000A81768625748A10706D52021C160421780
:101B00006A6282680A438260610703D5A96A042277
:101B10009143A96221070AD5A96A08229143A962C3
:101B20008021C160D2436A6282680A4382600120D8
:101B300070BDF8B5484D2C6BE00702D0A81728639C
:101B40000440200606D58020C043286380208443BB
:101B500001F043F8200709D50820C0432863082076
:101B6000844301F038FE082000F0B3FC600604D581
:101B70004020C043286340208443A00606D520208F
:101B8000C04328632020844300F06CFE600707D523
:101B9000042000F057FF0420C0432863042084433E
:101BA000200407D50126F603300001F016F8F043B3
:101BB0002863B4436003400F06D0072000042100CF
:101BC0000140C943296384430B2620003605304079
:101BD000070005D0380000F09DFBF8432863B443AC
:101BE000E000400F09D00727BF0626003E40300026
:101BF00000F0F9FAF0432863BC43002C06DA012018
:101C0000C00700F01AFB154828630440144804423A
:101C100005D0200000F076F9200001F062FA0D48AE
:101C200081680122D20411438160F8BD094B012271
:101C3000D20410B5DA60FFF77CFF012010BD000070
:101C4000380E0004009100A800170200A8FD00044F
:101C5000009400A8009000A880220080FFFFFF7F72
:101C60000010000110B503F00AFE002801D0AC48B6
:101C7000807D10BDF8B50027AA4D3C00E968A86832
:101C80003E0079407840084303D004F371FF06001A
:101C90000C00FFF7E7FF04F093FA1FF08CEB04F061
:101CA00090FAE968A8687940084309D004F360FF16
:101CB000AA68801BEB68A14180185941E960A860BF
:101CC000F8BD10B502F012FC002826D002F00DFC81
:101CD00095490120C0048860001100F0D61C896875
:101CE00001000000C81B00A0000200005D68A54DB7
:101CF00075FF93480088002801D102F051FC02F0E2
:101D0000BAFC02F094FC02F05BFC01F024FEFFF749
:101D1000B3FF1FF05AEB01F029FE02F049FC02F07C
:101D2000B3FC02F08DFC02F04CFC02F0E7FB10BDAE
:101D3000FEB50024250026001FF044FA019000F0B3
:101D4000D4FE002802D1FFF79FFF44E000F091FC91
:101D500000F008FE00F0F7FE77480068810702D522
:101D6000C10700D00124010702D5410700D5012594
:101D7000810602D5C00600D5012604F097FC00902C
:101D800001F09EF9070002D1012001F0ADF9012018
:101D9000C007807804210840400702D400F04DFCC1
:101DA00005E0002CCFD0002DCDD0002ECBD0009858
:101DB0000028C8D0002FC6D0604CA568E017E060AE
:101DC00001263603300000F012FFFFF784FF3000D9
:101DD00000F004FFA56001981FF0F8F9FEBD10B5F2
:101DE00000F081FC00F00DFE00F0DEFEFFF7A0FF2A
:101DF00010BD10B51FF0E6F90400FEF77DFC01F000
:101E00002FFD20001FF0E2F910BD10B504001FF0F7
:101E1000D9F9494A1168214311601FF0D7F910BD63
:101E200010B503F003FD47494000085A464B4749A7
:101E30005843096A0B071B0F47F306EF080507060F
:101E40000609090B0B06400810BD800810BDC0082C
:101E500010BD000910BD10B504001FF0B3F9364ADB
:101E60001168A14311601FF0B1F910BD324A0100A1
:101E700012680020914300D101207047F8B52E4C24
:101E800004F380FE22696369851A99410E00E168B6
:101E90000091A0686422070047F3C8EE33002A00CF
:101EA00047F346EB0099060000253800694068407A
:101EB000084309D10120E560A06004F363FE6A1EB7
:101EC00080185141616120613000F8BD1A4800213D
:101ED0008160C16001614161704710B502F022FB71
:101EE00010BD70B5040002F01DFB041B6C3C732D8B
:101EF00001000000C41D00A00002000044907B3DD2
:101F000003F077FD050017490026200047F39CEEFB
:101F100033002A0047F316EB70BDC00005D50B480F
:101F20002C304068002800D0004770470300012093
:101F300010B5FFF7A5FF002804D0D80102D5002076
:101F400000F0DBFA10BD0000A0020080985900B03C
:101F5000009000A84A5B00B000000004A0860100C9
:101F60000028008040420F00022910B505D0032947
:101F700003D0042901D0052903D1C14BFF21491CFD
:101F80009960042A05D0052A03D0062A01D0072A21
:101F900007D1002805D100210A2208000B0004F017
:101FA000DEFB10BD7047052803D2B6498000085CEF
:101FB0007047FF20704710B50C000020FFF7F3FFBB
:101FC000A04201D100F080FA0120FFF7ECFFA0420F
:101FD00001D100F051FC0220FFF7E5FFA04201D142
:101FE00000F03AFD10BD10B50C000020FFF7DBFF3C
:101FF000A04201D100F07CFA0120FFF7D4FFA042FB
:1020000001D100F03EFC0220FFF7CDFFA04201D13C
:1020100000F027FD10BD042910B507D004DC02290B
:1020200004D0032906D101E0052903D100F01BFAF1
:10203000002800D0012010BD022910B505D00329C9
:1020400003D0042901D0052901D100F0B5F910BD54
:10205000022910B505D0032903D0042901D0052990
:1020600001D100F068F910BDFF280BD0854A00218E
:102070008B00D35C834202D10806000E7047491CD6
:102080000529F5D3FF207047FF280CD07D4A002199
:102090008B009B185B78834202D18800105C7047EC
:1020A000491C0529F4D3FF207047052804D275493F
:1020B0008000401840787047FF207047FF280CD000
:1020C000704A00218B00D35C834203D188008018C2
:1020D00040787047491C0529F4D3FF207047FF283A
:1020E0000CD0684A00218B00D35C834203D1880066
:1020F000801880787047491C0529F4D3E8F9C44555
:1021000001000000C01F00A000020000B078C580E0
:10211000FF207047F7B582B007000E000C2901D2EE
:10212000092F02D3002005B0F0BD00255A49A800B0
:102130000A5CBA421ED14418A278B2421AD02806CC
:10214000000E3900019001F016FC002812D0A67094
:10215000E07804994007400FC9000843E0700198F7
:102160003200390001F009FC002808D0E078022193
:102170000843E0706D1C052DD8D30120D3E74648F5
:10218000AA00FF2110188170E0784007400FE0702E
:10219000C8E7F0B5060008003F4F00220421930075
:1021A000FC5CB44209D1DD19EC7823000B43002814
:1021B00002D02300FB242340EB70521C052AEED3EF
:1021C000F0BD354A00218B00D35C834206D18800E4
:1021D0008018C0784007C017401C7047491C05296B
:1021E000F1D3002070470020704770B505000C0047
:1021F000100002F0B5F9200000F00DFD2800FFF7F7
:102200004DFF022805D0032803D0042801D005285B
:1022100003D1200000F09CF870BD2000FFF787FE7E
:1022200070BD10B50400C00005D5012212031104D1
:102230000C20FFF7DAFF200105D50122D20211049C
:102240000B20FFF7D2FF600105D501229202110495
:102250000A20FFF7CAFF10BD0120C00310B502F02D
:1022600079F90120C00700F0CDFC0C48016A8022FA
:102270001143016210BD0120C00310B502F070F9D6
:102280000120C00700F0C7FC0449086A802290437F
:10229000086210BD009000A8B05900B0002800806E
:1022A000F3B581B00F000198FFF7E8FE0400019834
:1022B000FFF70EFF06000198FFF71BFF0500002C3B
:1022C00003D0012C01D0022C19D1331F0126760531
:1022D00047F3CEEC040309090E15102002F040F973
:1022E0000120000509E0202002F03AF9300004E066
:1022F000802002F035F90120C00500F09AFC002F83
:102300001DD10198FFF75DFF002818D04CCEBAF818
:1023100001000000BC2100A000020000B8A7345D4D
:102320002B1F47F3B0EC06161616160A0416019872
:10233000FFF763FF01000D2009E00198FFF75DFF43
:10234000694AA1008918C978CA080100100000F084
:10235000D2FFFF2201991000FFF741FEFEBD0800E9
:102360000021A7E710B50400C00203D50121022017
:10237000FFF7A0FFA00207D501210320FFF79AFF76
:1023800001210420FFF796FF200203D5012105203B
:10239000FFF790FF01200007844205D040108442DF
:1023A00002D0401084421AD1FF208206A11808D022
:1023B000891804D0C206891804D10C2002E00B2031
:1023C00000E00A20FFF774FE022805D0032803D09E
:1023D000042801D0052802D10121FFF76BFF10BDB1
:1023E000F8B504000D0017000800FFF78CFE06008A
:1023F000002C03D0012C01D0022C22D13B1F01273D
:102400007F0547F340EC04030C0C141E102002F06F
:10241000ABF8102002F0BAF8012000050FE02020F0
:1024200002F0A2F8202002F0B1F8380007E0802086
:1024300002F09AF8802002F0A9F80120C00500F00F
:10244000EBFB331F47F31EEC061D1D1D1D0E041D67
:102450002800FFF7D2FE002801D1012100E0002171
:102460000D200CE02800FFF7C8FE002801D1012153
:1024700000E000211C4AA0008018C078C00800F0CD
:102480003AFFFF2229001000FFF7C1FDF8BD70B52B
:1024900004000020002C03D0012C01D0022C20D1FC
:1024A000124D00222868462104F359FB002817D159
:1024B00028680022082104F352FB002810D1022CC6
:1024C00006D0012C04D01FF0ACE800280AD007E0A9
:1024D00005F0DEFA002803D105F0B6FC002801D192
:1024E000002070BD012070BDB05900B0800E000406
:1024F000022010B5FFF7CDFC02F01CF8002804D034
:10250000012000F0B0F900F0C0F900210822080015
:102510000B0004F038F910BD022010B5441E59829A
:1025200001000000B82300A0000200004C4F8AE028
:10253000FFF793FC10BD70B50020FFF752FD0400BB
:102540000020FFF7D0FD05000120FFF7ACFC854916
:10255000086A10221043086283499003886002F0E1
:102560003FF8082000F06BFB2A0021000020FFF755
:1025700019FD70BD70B51EF04DFE05007B4800686A
:10258000C00710D00020FFF7D6FF7D20C00003F069
:1025900038FA002036F3F1FF040002E0002036F3A1
:1025A000ECFFA042FAD028001EF038FE70BD0020DB
:1025B00010B5FFF716FD04000020FFF794FD0200A0
:1025C00021000020FFF762FD10BD10B51EF022FEB5
:1025D000040066480068800701D5FFF7E8FF200087
:1025E0001EF01CFE10BD002010B5FFF7FAFC040021
:1025F0000020FFF778FD020021000020FFF729FDF1
:10260000002800D0012010BD38B501F09DFF002842
:1026100026D1401E00905548554C0068C00711D087
:102620006068401C18D0A068FFF783FC514947F34D
:1026300044EB00906168884201D3002000E0081A52
:10264000009009E0684603F0E4FF00280CD00098F1
:102650006060FFF76AFCA06021780098884203D38D
:10266000FFF7C1FF002801D1002038BD012038BD8F
:102670003E4810B50068C00705D0FFF7C5FF002829
:1026800001D0012010BD002010BD002010B5FFF7C3
:10269000A8FC04000020FFF726FD02002100002016
:1026A000FFF7E8FC10BD10B5FFF79DFF002804D030
:1026B000002004F016F9002801D1002010BD0120EF
:1026C00010BD2A4810B5006880070DD42A4800784C
:1026D000022809D1FFF7CCFF002805D0FFF7E3FF60
:1026E000002801D0FFF7D1FF10BD70B50020FFF723
:1026F00078FC04000020FFF7F6FC2049050009687B
:1027000017204883082000F091FA01F061FF01F0E2
:1027100053FF154901208004C8602A0021000020D1
:10272000FFF75EFC0F48016A102291433C525E8E17
:1027300001000000B42500A00002000055B754902D
:1027400001620120FFF793FB70BD0D4810B50068D2
:10275000C0070FD1FFF762FF00280BD01EF064FD09
:102760000400FFF75BFF002801D0FFF7C8FF20003F
:102770001EF05EFD10BD000000280080009000A843
:10278000985900B0DC5900B0E20400006C5B00B066
:1027900084EA0004F8B51EF047FDBE4D0700286826
:1027A00000282ED103F0E9F84021182003F05AF850
:1027B00003F0D5F8B84E30690221084340084000C4
:1027C000306101F0E1FE040001F0DEFEA042FBD02A
:1027D0003069032108433061B04A906801214906FD
:1027E00088439060AD4A803AD0688843D06003F057
:1027F000C4F80821332003F040F803F0B0F80120BA
:10280000286038001EF014FDF8BDF8B51EF00CFD70
:10281000A04D00902868012835D103F0AEF80821BA
:10282000332003F01FF803F09AF89C498039C868F8
:10283000012676063043C860984FB868B043B86048
:10284000954908690222104340084000086101F0E0
:102850009BFE040001F098FEA042FBD00A2003F08A
:10286000DAF8B8683043B8608B490869800880009E
:10287000086103F082F84021182002F0FEFF03F007
:102880006EF80020286000981EF0D2FCF8BD10B54C
:1028900004000120FFF7AFFB002C05D18049096837
:1028A000CA0705D0490603D5062801D0FFF7F2FC78
:1028B00010BD012010B5FFF79EFB062803D001F0E4
:1028C0004DFE0028FBD110BD082010B5FFF7F5FA2A
:1028D00010BD082010B5FFF7CAFA10BD38B50020AA
:1028E00000900120FFF787FB04000120FFF705FCA3
:1028F00005000420FFF7E1FAFFF787FF01F0C0FEB3
:10290000202000F0A6F901F08FFE684605F0C4F81B
:102910000121644A4906002800D0009891602A00ED
:1029200021000120FFF748FB38BD10B51EF07CFCEC
:1029300004005B480068400702D50020E64AFB1609
:1029400001000000B02700A000020000A15FEA2DF6
:10295000FFF7CEFF20001EF075FC10BD012010B562
:10296000FFF753FB04000120FFF7D1FB0200210019
:102970000120FFF782FB002800D0012010BD08B520
:10298000684605F08FF8002803D0FFF7E7FF00281E
:1029900001D1002008BD012008BD464810B50068DF
:1029A000400705D5FFF7EBFF002801D0012010BD3F
:1029B000002010BD70B50120FFF727FB04000120A7
:1029C000FFF7A5FB05000020FFF71FFBA04204D086
:1029D0002A0021000120FFF761FB70BD354810B5CA
:1029E0000068000709D4FFF7D8FF002805D0FFF7DB
:1029F000B5FF002801D0FFF7DDFF10BD10B501F0D5
:102A00001DFE03F020F810BD10B501F017FE03F015
:102A10001AF810BD38B5002000900120FFF7F5FA34
:102A200004000120FFF773FB0500202000F012F9DD
:102A300001F027FE204901204006C860684605F0E5
:102A400035F8002808D101F00BFE05F036F8002813
:102A50000AD0FFF7A9FE07E00098002802D1FFF78F
:102A6000CDFF01E0FFF7D0FF2A0021000120FFF792
:102A7000CBFA0420FFF705FA38BD0E4810B5006800
:102A800040070FD4FFF77BFF00280BD01EF0D6FBCA
:102A90000400FFF774FF002801D0FFF7BBFF200000
:102AA0001EF0D0FB10BD0000E85900B000280080E7
:102AB00080210080985900B0009000A8202010B517
:102AC000FFF705FA10BD202010B5FFF7DAF910BDA9
:102AD00070B501F059FE01F073FE0128FBD1022010
:102AE000FFF793FA04000220FFF711FB0500102006
:102AF000FFF7EDF9554901204004886001F032FEEE
:102B0000042000F0B0F801F01BFE2A002100022092
:102B1000FFF75CFA4E480068800601D401F047FEDA
:102B200070BD10B51EF08AFB040049480068C0065D
:102B300002D50020FFF7CCFF20001EF083FB10BD64
:102B4000022010B5FFF761FA04000220628EE393C1
:102B500001000000AC2900A0000200006646E870F9
:102B6000FFF7DFFA020021000220FFF790FA0028A9
:102B700000D0012010BD10B505F08EF9002803D05B
:102B8000FFF7E8FF002801D1002010BD012010BD93
:102B9000344810B50068C00605D5FFF7ECFF0028E3
:102BA00001D0012010BD002010BD70B50220FFF73C
:102BB00036FA04000220FFF7B4FA05000020FFF700
:102BC0002EFAA04204D02A0021000220FFF770FA5A
:102BD00070BD244810B50068800609D4FFF7D8FFFF
:102BE000002805D0FFF7B6FF002801D0FFF7DDFF72
:102BF00010BD70B50220FFF712FA04000220FFF7A3
:102C000090FA0500042000F02FF801F0ACFD01F06F
:102C1000A1FD134901204004C8602A0021000220C0
:102C2000FFF7FCF91020FFF736F901F0AEFD01F0D7
:102C3000BEFD70BD0B4810B50068C0060FD4FFF78D
:102C40009AFF00280BD01EF003FB0400FFF793FF50
:102C5000002801D0FFF7CDFF20001EF0FDFA10BDC7
:102C6000009000A8985900B036494A6A02434A6267
:102C7000CA6A0243CA620120704732494A6A8243E3
:102C80004A62CA6A8243CA62012070472D494031B4
:102C90000868086070472B49C043086301207047EB
:102CA000284B80339969DA6909011209090912016F
:102CB000002804D00520400701430A2003E0052036
:102CC0000007014305200243D961DA6170471E48BD
:102CD000016B022291430163016B40229143016326
:102CE000016B04229143016370471748006B810711
:102CF00001D500207047400601D502207047012011
:102D0000704710B502F00BFE002804D00F49886907
:102D1000CA0B9043886110BD10B502F000FE002878
:102D200003D00A488069C007C00F10BD10B502F07B
:102D3000F6FD002804D005488069012109040840F7
:102D400010BD00008022008000210080C02A008089
:102D500070B5002402F0E3FD002808D031EA87A214
:102D600001000000A82B00A00002000092AE56CD8A
:102D7000FFF7E6FF002803D1FFF7D8FF002800D0B7
:102D800001241EF06FFA0500002C07D102201EF06E
:102D90003DFD002802D014490120086000210120D7
:102DA00001F086FB28001EF061FA002070BDF8B526
:102DB00001200E4900F03AFF0B4E0024361D01277A
:102DC000FF0308E02104090C3943012000F02EFF25
:102DD00070598047641CA50070590028F2D103F097
:102DE00041FF04F0B6FEF8BD506600B07F8B0000D6
:102DF000FF4841680068814201D1012070470020EE
:102E00007047FB4810B541680068012292070B002B
:102E1000040093439443A34205D1114010408142E2
:102E200001D0012010BD002010BDF24900204861F2
:102E3000F14A5060EE4A1060C8607047EC48416843
:102E400001600168EB4841610021C1607047F8B53D
:102E500004000D0016001EF005FA070000210320F3
:102E600001F026FB002C0ED0002D0CD032002900E2
:102E7000200046F34CED032001F03CFB38001EF02F
:102E8000F5F90020F8BD38001EF0F0F9FEE7D9484A
:102E900010B58068342146F3D6ED10BDF8B50C00AE
:102EA0000700002600281CD0D24D2878012818D110
:102EB000012C02D11EF0D6F906000021032001F0FA
:102EC000F7FAFFF733FF00280DD0FFF7AEFF002021
:102ED0002870032001F00EFB012C02D130001EF0FF
:102EE000C5F90120F8BD1EF0BDF98446FFF789FF42
:102EF000002804D060461EF0B9F9002013E0E8680D
:102F0000401CE860BA4800680C210004000C4143F2
:102F1000BA480818002105000A000B000EC06046E0
:102F20001EF0A4F92800002800D1FEE7FA78082A4C
:102F300001D8121D00E00C22390046F3E8ECAC4841
:102F400000F045F9AE49886B0122104388630320E5
:102F500001F0D0FA012C02D130001EF087F90020D8
:102F6000F8BD1CB50024E443A6480122251100BD8C
:102F700001000000A42D00A0000200008B5688BDB7
:102F8000032101AB009400F36BF901980028F5D000
:102F90000128F3D100F062F9F0E710B51EF06CF9EA
:102FA00004000021032001F08DFA9848001D00F074
:102FB00018F99849C86BCA0D1043C863032001F083
:102FC000A3FA20001EF05CF910BD002810B508D04F
:102FD0000078012805D1FFF73BFFFFF7DEFF002057
:102FE00010BD012010BD10B50178042901D00120C9
:102FF00010BD85494A68521C4A600969002901D000
:10300000884701E0FFF7C9FF002010BD0EB504217D
:103010006B461970012159700221D970017819711C
:103020004078587178484168491C4160FFF7B5FF06
:1030300001216846FFF73CFF00200EBDF0B587B0C8
:103040001EF01AF907007548FFF722FE74490120A7
:10305000C0048860C412200001F0C2FA200001F010
:10306000CBFA6D486F49283001606F4901616F49A3
:103070004160654C0026266101220A20059202006B
:1030800003906B48012189026B46049607C3002315
:103090006148684AA83868A101F3DEFA002802D026
:1030A000012007B0F0BD5C4865A100F367F800217E
:1030B0000320267001F006FAA068644D0068A8425B
:1030C00007D1FFF73DFE00280AD0FFF743FE002896
:1030D00006D0FFF7E6FEA0680560FFF7B0FE0DE042
:1030E000FFF7B6FE4948466001206B461874DE744F
:1030F0002070002104A8FFF7DBFE2670032001F0FA
:1031000003FA38001EF0BCF80020CAE700290CD0F2
:1031100005280AD2042802D13B48016103E03E4A57
:10312000800028321150002070470120704770B590
:10313000FFF706FE344C002802D00020207014E077
:103140001EF09AF82F4D060008E0E168002910D023
:103150002D48491E1430E16000F043F86069696849
:103160008842F2D130001EF08BF83A4938480863A3
:1031700070BDFEE72348016840688142444EFB274A
:1031800001000000A02F00A0000200007FBE36005A
:1031900001D0012000E0002021494A6809688A42E4
:1031A00001D0012100E0002108430121484070477F
:1031B00001001E48002210B500F3ECF810BD70B5F8
:1031C000040016480178012901D001210170E001B5
:1031D0000CD5254925480863CD0D280001F010FACB
:1031E000280001F007FA0120FFF7E2FFE00401D513
:1031F000FFF7A7FF70BD026801231104090C9B07AC
:10320000491C1A4011430A009A43082A01D3594025
:103210001940016070470000001300C02CC800B0C6
:10322000801300C0081300C0802A0080780401B019
:1032300000100001009000A8312E00000B2E0000AD
:10324000EF2D0000D0FF00B09B2D000049636354B8
:1032500061736B0049636351466C616773000000E2
:10326000CDAB0000FFEFFFFF80220080FFFFFFFEDD
:10327000F8B51EF00BF8144C144E154D07001BE06A
:10328000FFF768FD002803D012490020087017E0FE
:1032900070680C230004000C584340190CD00178CE
:1032A000052905D28A00A258002A01D0002902D19E
:1032B0002168884700E09047706831688842DFD114
:1032C00038001DF0E7FFF8BDA00401B0801300C076
:1032D000881300C02CC800B0F8B504000D00764873
:1032E000764A0168126801209047002848D00120E2
:1032F0002700734E0100103F0200A140BA40704BFE
:103300004036002D2ED00325082C07D21E686200FF
:1033100095409040AE4306431E6009E0102C0AD24F
:103320005E68083C620095409040AE4306435E6094
:10333000986888431AE0182C07D2F36979008D4009
:103340008840AB430343F36109E0202C07D2336A82
:10335000183C61008D408840AB4303433362706A80
:10336000904307E0102C03D298680843986002E06D
:10337000706A104370625349012009688847012030
:10338000F8BD70B504004C484C4A0D001442FE28AC
:10339000010000009C3100A00002000001A591B0D6
:1033A000016812680120904700281AD00122102CD1
:1033B00008DA4849C868A2409043002D00D0104365
:1033C000C8600AE0434B4033986A103CA2409043E7
:1033D0000100002D00D0114399623F490120096886
:1033E000884770BD10B504003848394A0168126832
:1033F0000120904700281AD00122102C06D235480F
:103400008168A24011438160006907E03148403083
:10341000416A103CA24011434162C06AE0402E491B
:10342000C4070968E40F01208847200010BDFF2071
:1034300010BDF8B52548264A01681268012090475A
:10344000002840D0254801210903C1602148016AB4
:1034500020484030C06B0F043F0C0006000A0743B1
:1034600000241F4801261EE04068E2008158002920
:1034700018D010184068320082403A4212D005003D
:103480008847102D06D21349086A3200AA4090439B
:10349000086207E00F494031C86B103D3200AA4076
:1034A0009043C863641C0E4801788C42DCD30B48FF
:1034B00081680122120311438160074901200968D4
:1034C00088470020F8BD0120F8BD000038E5000461
:1034D00040E500040002009044E50004009000A8CC
:1034E000EC5900B0F8B50025FF4F387D012802D90E
:1034F0007D2000023860787DC00709D002F094FE7C
:103500003968884204D2787D4008400001257875EA
:10351000787D400731D502F0A3FE79680400FB26D0
:10352000814220D8F868A0421DD8052002F031F869
:10353000A04218D8052002F02FF8A04213D801208D
:1035400002F027F8A0420ED8012002F025F8A04290
:1035500009D8022002F01DF8A04204D8022002F08F
:103560001BF8A04201D9787D04E0787DC10701D025
:10357000810702D43040012578752800F8BD70B568
:103580001DF08EFE0500FFF7ADFF0028FBD1D64CE5
:10359000607DC00706D002F01BFE00288F09028A5A
:1035A00001000000983300A000020000F54D2F0D2F
:1035B00002D1012002F079FC607D800706D502F07F
:1035C00014FE002802D1012002F0F1FC607D4007CA
:1035D00009D502F0E8FD002802D1012002F096FD95
:1035E000607D400706D402F0DEFD002802D00020F6
:1035F00002F08CFD607D800706D402F0F6FD002805
:1036000002D0002002F0D3FC607DC00706D102F09A
:10361000E9FD002802D0002002F047FC606800218C
:1036200001F0B5FFA068002101F0B7FF607DC00781
:1036300009D120687D210902884201D1012000E0E2
:10364000002002F01BFEE068002101F0A3FF2069CA
:10365000002101F0A5FFAA490020087028001DF0F4
:103660002DFE002070BDF0B506000D0087B0A34907
:103670000027182201A846F3DCE9A04C607D000772
:1036800002D4012007B0F0BD002E02DA76007608E1
:1036900001273300042646F350EB0852051420445A
:1036A000512C385202F0CAFDA84204D2607D400875
:1036B0004000607503E0617D012001436175256074
:1036C0003DE002F0D7FDA842607D02D2FB21084018
:1036D00000E030436075656031E002F0CBFDA84248
:1036E000607D02D2FB21084000E030436075A56098
:1036F00025E002F0BFFDA842607D02D2FB21084018
:1037000000E030436075E56019E002F0B3FDA842C7
:10371000607D02D2FB21084000E0304360752561E6
:103720000DE0280002F0A2FD0028607D02D1FD21FD
:10373000084001E002210843607500E025756F49EB
:10374000182201A81DF008FC002802D06C490120B5
:103750000870002F01D0FFF71CFF002092E7FEB594
:1037600000207D24E401270001250194009011F33D
:1037700026FD8821694306000291405C02282FD172
:103780002804000C1CF383FC0099491C0906090E4F
:1037900000910279012A02D18179012904D002998C
:1037A00089194B7D092B08D102997D20F342E35AF8
:1037B00001000000943500A000020000ECB5F17D8E
:1037C0008919C9788001002910D140100EE0052A1E
:1037D00005D18079052802D17D20000201E07D20FD
:1037E000C001C978002901D17D208001844209D817
:1037F000040007E0012805D17D20C0018442F7D9EB
:103800002000F5E76D1C082DBBD30098012805D9D1
:103810007D200002844200D9200004003E48C06997
:1038200000280BD07D200002844200D92000040033
:103830007D20C001874200D93800070037488079D1
:1038400002280BD17D200002844200D92000040010
:103850007D20C001874200D938000700019901206E
:10386000FFF70BFF39000320FFF707FF21000220BD
:10387000FFF703FF0020FEBD10B5254C607D00075B
:1038800034D502F0C2FC002802D1012002F019FC5C
:1038900002F0B8FC002802D1012002F0D3FB02F0B4
:1038A000B7FC002802D1012002F08AFC1C48016804
:1038B0000420FFF7E2FEFFF75CFF7D21490160680D
:1038C0000C008A00904201D9140011000720FFF774
:1038D000D4FE21000620FFF7D0FE0E480078002815
:1038E00004D001200021C007FFF7C7FE10BD084823
:1038F00070B5407D000724D57D24E401062001F049
:103900005CFE050002F059FC002811D00AE000001E
:10391000C4CE00B0F45900B008D70004D0D10004E0
:1039200094E5000402F0B0FCA04200D320000400A3
:10393000A54206D20021200001F033FE07490120F4
:10394000087070BD06480822417D114341757047DB
:103950000348F722417D114041757047F45900B08A
:10396000C4CE00B0002010B5FEF795FB0400002087
:10397000FEF713FC020000202100030000F08CF889
:103980000120FEF788FB04000120FEF706FC020080
:1039900021000120002300F07FF80220FEF77BFBCE
:1039A00004000220FEF7F9FB0200210002200023A0
:1039B00000F072F810BDF8B501263349919697656D
:1039C00001000000903700A000020000185D4FC009
:1039D000334F082A15D0092A43D1002B41D108685A
:1039E0008C0C2043086001210D20FFF79DFC002175
:1039F0000D20FFF7EEFC7869A0437861B869A04319
:103A000022E0002B2DD1820026481418E078C0084F
:103A1000192801D3002624E00B6801252A008240E2
:103A200013430B602900FFF77FFCE0780121C008F9
:103A3000FFF7CFFCE178C808102807D279698540E4
:103A4000A9437961B869A843B8610AE014484030D5
:103A5000026B4906090F8D40AA430263416BA943DB
:103A600041633000F8BD0123AFE70023ADE70E4806
:103A700010B50068002804D000221100032002F0D5
:103A80003DF810BD084810B50068002804D0002299
:103A90000121032002F032F810BD00004023008015
:103AA00000020090B05900B048C800B00A2A10B512
:103AB00011D00B2A0FD00C2A0DD1002B0BD10021D5
:103AC0000F20FFF731FC0448426981018A434261BB
:103AD00082698A43826110BD000200903EB50C22CB
:103AE00004006F4841686846FFF7EDF9A00702D56A
:103AF000019805F066FAA00603D56B46187A05F022
:103B000071FA3EBD10B54078FFF7E8FFFFF777FA8E
:103B1000002010BD3EB5040002E0012001F0D5FFF9
:103B2000FFF7A2F90028F8D002206B461870002099
:103B30005C709870D87001216846FFF7EBF93EBDC4
:103B4000574808B541680122891C6846FFF7BBF950
:103B50006B46187808BD10B50400FFF7F1FF002888
:103B600002D12000FFF7D6FF10BD10B50C000100F8
:103B70004B4824220068FFF7A6F9002C02D0200051
:103B8000FFF7E9FF10BD464910B509682422FFF789
:103B90009AF910BD01B54248012200686946083013
:103BA000FFF791F908BD01B53D480122006869465B
:103BB0000930FFF788F90820FFF7CDFF08BD11B5E0
:103BC00081B0374C0122216868460A31860422CF31
:103BD000010000008C3900A000020000DF444D9D70
:103BE000FFF77BF96B4618781979884208D020686E
:103BF00001220A3001A9FFF770F90820FFF7B5FF8D
:103C00001CBD01B52B480122006869460B30FFF747
:103C100064F908BD01B527480122006869460C30E7
:103C2000FFF75BF908BD01B522480122006869462B
:103C30000D30FFF752F908BD13B504221D4C69463B
:103C400020681030FFF749F920680422143001A9D8
:103C5000FFF743F91CBD01B516480122006869460B
:103C60001D30FFF73AF908BD01B51248012200687E
:103C700069461E30FFF731F908BD01B50D48012234
:103C8000006869462030FFF728F91020FFF76DFF24
:103C900008BD084808B5416801226846FFF71DF9CC
:103CA0006B46187808BD034910B549680C22FFF728
:103CB00014F910BDF85900B0FB4A10B510684378EC
:103CC00004781802F94B2043984203D01068017021
:103CD000090A417010BDF4498000091F08580221EB
:103CE000593002780A430270F14A507C08435074FC
:103CF0007047ED48F8B524300188EE4A91421DD056
:103D000002001288012441889440EB4F012904D11C
:103D1000FD68A5432C43260003E0FE68A643344318
:103D20002500E6498088096846F31AE88905800A73
:103D30000843FD6001D01DF008ECFE60F8BDDA4AD2
:103D40008000121F105840308183D2E770B5050003
:103D5000DB4C09D10022DB48110046F353F8002860
:103D6000206001D020210181A8002158002908D01D
:103D70000A898918CC4A121F125811672058082145
:103D8000017370BD70B50400C068C74D012180008B
:103D90002D1F285800264166E06880002858466696
:103DA000E068800028580B23D83002689B021A4331
:103DB0000260E068800028580823D83002681A435F
:103DC0000260E068800028584B05D83002689A43AA
:103DD0000260E06880002858D8300268DB210A4879
:103DE00001000000883B00A0000200002BACF32083
:103DF0000A430260E068FFF7B3FFE168072089002B
:103E000069580866E068FFF770FFE068002802D193
:103E1000296817200866E06880002858AA49866645
:103E2000E068002804D1AB4A0832118051809180AB
:103E3000A84A0B0A0E32117053709170090AD170A2
:103E400081000E3A5158002901D00D2100E00C21CB
:103E5000FFF77FFFE0689F498000091F0E50E06870
:103E60000521820095488258D170E1688900415847
:103E70008E70E168890041580E71E16889004058F0
:103E80004671002070BDF8B504001422914F6243C2
:103E90009248A5003F1F0026032911D1002C0AD10A
:103EA00046F31CF8202138600181010024310020F4
:103EB00002F061FE14E0101846F310F878510FE09C
:103EC000052904D1002C08D084481438F3E70229CE
:103ED00001D0082904D1002C2ED145F3FFFF386012
:103EE0007859002827D0002C25D13868734C0189D7
:103EF000411848780B7802021A43241F2068C0300A
:103F0000828248780A7803021343201D0268D5781C
:103F10000122AA40521E9A1803680068DB781A41F1
:103F20008270CA7820688030C28122683000D166F1
:103F30000221FFF70EFFF8BD68481430BBE70122ED
:103F400070B5D2079378634C80000C3C22588A42AB
:103F50002FD0002921500DD0002001228500655965
:103F60008D4204D0461C1500B5401D4221D1401C95
:103F70000128F3D351480C3802788A4219D00170D5
:103F8000514A3630002909D0C17883780802184395
:103F900090420ED001F0ADFD012008E04178037899
:103FA00008021843904204D001F0A3FD0020FEF760
:103FB000D1FE70BDFFB581B00400029800287BD00F
:103FC000E068002878D1029D0498E88020202881AC
:103FD000121D2035100A2A70687000200126A87072
:103FE0001DF090F90090E0680021FFF71EEE5B2BBA
:103FF00001000000843D00A00002000032542D505A
:10400000A8FFE068384F8000083F385800280ED0DD
:104010000498032805D1291D002002F0D0FD0028B6
:1040200005D100210B2208000B0002F038FC049897
:10403000022874D0032821D005285BD0082817D186
:104040000320E870E06814214143294808180299C8
:1040500045F377FFE068244A8100121F5258002A76
:1040600006D17958002903D10221FFF716FF002657
:1040700000981DF055F9300005B0F0BDFE20E87045
:10408000291D002002F09BFD0028E0680BD01423BE
:10409000584317494018029945F375FFE16800201D
:1040A0008900785006E0142141431148081802990C
:1040B00045F347FFE0680C4A8100121F5258002A5E
:1040C000D6D179580029D3D10321CEE72FE026E0BD
:1040D000A86600B0DCFE000080000080FFFF00004A
:1040E0000002009044C800B0C46600B0B45B00B0E9
:1040F00078FF00B00220E870E06814214143FE48D8
:104100000818029945F31DFFE068FC4A81005258E7
:10411000002AADD179580029AAD10521A5E70420AC
:10412000E870E06814235843F34940188FE70020F3
:10413000A2E710B504001DF0EFF8F04AA1001C3A08
:10414000EF4B54586366525817231366EB4B00220B
:104150000C3B5A501DF0E4F810BDFEB5840006007B
:10416000E64800251C3801590D66025901215166A7
:104170000059E24F45663F1D3859002802D045F3EB
:104180002BFE3D51DC4914227243DC4F0B001433EB
:104190003859D31801930B00143BD3185618002834
:1041A000009307D045F318FE04E0300045F3A0FE6D
:1041B0003851F7E7300045F304FF0028F5D105E05A
:1041C000009845F395FE385145F306FE009845F3F7
:1041D000F8FE0028F4D105E0019845F389FE385136
:1041E00045F3FAFD019845F3ECFE0028F4D13D516A
:1041F000FEBDF8B504001500C0481C38DAF592136E
:1042000001000000803F00A000020000C6BC93ED4A
:104210000600083E15294DD010DCBD4F091F0022B5
:104220003F1D0B0045F3C4ED11DEDFDFDFCA98DF71
:10423000A3DFAEAEDFDFDFDFAA2ADF00B448123033
:104240001C293ED009DC17295ED019297ED01A29F5
:104250002FD11DF06BF8756129E01D2940D01E2972
:104260004DD0202973D04629F2D1E0680028EFD143
:10427000A7480068002800D00120F8BD1DF056F8BE
:104280000500E0688100795800290FD1FFF77CFD17
:10429000E06881007958002903D128001DF04AF810
:1042A000EAE7002802D10121FFF767FD28001DF091
:1042B00041F898E0E1688900405802218068084090
:1042C000F8BD69782A78090211430170090A417022
:1042D000E978AA78090211438170090AC17082E065
:1042E00041780278090211432970090A6970C1787E
:1042F000827808021043A870000AE87073E0E06852
:104300000121FFF730FE6EE0814E834A0C36308883
:104310000F2801D99042AFD1E068002863D1A88866
:104320003080E98871802B899042B3805BD0FFF7A1
:1043300078F87A4B1A683088012181400A431A6064
:104340000006000E0121FFF717F84CE000E043E003
:10435000E068002847D107E0E068002843D16C49B5
:104360000C39096800293ED0FFF7EDFE3BE0E1681B
:10437000002938D100681721016634E0E068FFF7B2
:10438000F6FE30E0E16800290FD1717800290CD0E9
:10439000634900685E4BC0308182E0688000183B52
:1043A00018580170090A41707270E06881007958EC
:1043B000002918D00121FFF7E0FC14E0E068002894
:1043C00011D15248143881681430806809184F4858
:1043D000143080680818F8BDE0684D498000083145
:1043E0000D5000E035610020F8BDF8B50025A800AB
:1043F00047491C390A581023566EF2431A430B588A
:104400005A6608584030007E002D7ED1283FE9488A
:10441000010000007C4100A00002000023EBCEEA76
:104420000024F1073FD040073DD43E490022091D3A
:1044300008680389C418637827781B023B433E4F02
:10444000BB4204D901212800FFF7A1FC2AE0022386
:10445000037334480021001D0768072208000B0081
:1044600002F031FA0020FFF799FC2E48001D006889
:10447000002803D001212800FFF789FC3889001D9E
:104480003881E078FE2801D10120E070E078F880E2
:104490002348244928307861E37808310C680022E9
:1044A0003900A0470124B00754D51E4F00213868B9
:1044B000002816D001894118091D002002F089FB4F
:1044C000002802D00120391F0860164824380169ED
:1044D0003868002901D0884701E045F391FC0020AD
:1044E0003860230400211B0C0622080002F0EBF9BF
:1044F0000B4C200045F379FD002809D1200045F33D
:1045000074FD002804D1200045F36FFD002821D060
:104510000449091F0968002916D00B220EE02DE07E
:1045200078FF00B0C06600B0EFFEFFFFFFFF0000A5
:1045300040230080DCFE000005040000002108008C
:104540000B0002F0C0F905E0C0880106090E280042
:10455000FFF7B7FC0C490868006EC0060ED5F006E0
:104560000CD50A0001201032106009680720086687
:104570000021092208000B0002F0A5F96D1C012D95
:1045800000DA3EE70120F8BDA46600B070B5050072
:104590000C0009D102E0012001F0C9FA28001DF049
:1045A000A3F90028F7D011E0641E28001DF09CF943
:1045B00000280BD1012001F0BAFA002CF4D11249E5
:1045C000A8000A58521C0A50002070BD012070BD7E
:1045D0000E4B30B501215A6881400A408000002A04
:1045E00005D1094980310A58521C0A50FEE7064C91
:1045F000803C2258012A02D15D688D435D60521EC5
:104600002250012030BD00005CCF00B0C02A0080E5
:1046100030B500240D4B2200D5005D594976BD7A96
:1046200001000000784300A000020000D70370578B
:10463000002D0ED1D40018510A4B9200D318D96026
:1046400000030321000B890740180749511808602F
:1046500030BD521C042AE9DB012CF9D0FEE7000032
:104660005CD000B0C09B00A8009800A8FF4840683C
:10467000016F1022114301677047FC484068016FC9
:1046800010229143016770470020704770477047C0
:10469000F6484068816B090C01D000207047816B9F
:1046A000490504D5816B0904090FFBD100E0806B3B
:1046B00001207047ED484068406B7047EB494968FE
:1046C0004A6E82434A667047E84949684A6E024327
:1046D0004A667047E5494968CA6E0243CA66704730
:1046E000E24949688A6E02438A667047DF4840683B
:1046F000806B8007C00F7047DC484068C03041685D
:104700003722914341604168012211434160704763
:10471000D6484068C03041680822914341607047E4
:10472000D2484068C0304168082211434160704758
:10473000CE484068C03001680122114301607047D3
:10474000CA484068C03001684908490001607047A4
:1047500070477047C5484068416801229204114380
:1047600041608168121191438160FF30401C4168B3
:104770004908490041607047BC484068C11DF93193
:104780004A6801231A434A6041689A049143416090
:1047900081681211114381607047B4484068FF304E
:1047A000401C41680222914341607047AF48406815
:1047B000FF30401C41680222114341607047AB4802
:1047C0004068FF30401C01680122114301607047BE
:1047D000A6484068FF30401C016849084900016054
:1047E0007047A2484068FF30401C0168082211430E
:1047F000016070479D484068FF30401C01680822F6
:1048000091430160704799484068C03001680122B7
:10481000D20711430160704794484068C030016876
:104820004900490801607047904840683080799A93
:1048300001000000744500A000020000CEFBAE277E
:10484000FF30401C01680122D2071143016070470C
:104850008B48406880680003C00F704788484068F4
:1048600081680122D2041143816070478448406806
:10487000FF304130416A89088900416270478048B1
:104880004068FF304130416A0422914341627047E1
:104890007B484068FF304130416A04221143416245
:1048A000704777484068FF304130016A0122114368
:1048B0000162704772484068FF304130016A490820
:1048C0004900016270476E484068FF304130016A1C
:1048D0000122D20711430162704769484068FF30E6
:1048E0004130016A490049080162704764484068E4
:1048F000FF304130806A0005C00F70476048416852
:10490000092080010818C169012292031143C16185
:10491000C16952001143C161C16952001143C161B3
:10492000704757484168092080010818C169012271
:1049300092031143C161C16952001143C161C16950
:1049400052009143C16170474D4840688168102210
:104950001143816070474A48416809208001081866
:10496000C169012252041143C161C169D2001143DE
:10497000C1617047424905224968D2018918CA6954
:10498000382340079A43800E0243CA61C869012256
:104990001043C86170473A4A0023D3561F21C018FC
:1049A0001F2800DA01000806000E70470D2804D801
:1049B000334900228A56002A00DBECE77047F0B545
:1049C00093B0304C2068030960681B010109A0689E
:1049D00009010209E068120100090001C01C1290DF
:1049E0002069491C050960692D0100090001401D6D
:1049F0001190A069921C00090001801D1090E069CF
:104A00002D1D0609206A36010009000108300F90AB
:104A1000606AF61D0009000109300E90A06A0009C5
:104A200000010A300D90E06A000900010B300C9083
:104A3000206B000900010C300B90606B70F771184F
:104A400001000000704700A0000200003A13109A15
:104A50000709A06B3F01000900010D300A90E06BCF
:104A60000D37000900010D308646F02081431031DA
:104A700009911299854340350895119D82438143E0
:104A800020323031854350350795109D834385434F
:104A9000944603E0005A00B05CD200B05035069551
:104AA0000F9D0C9A8543503505950E9D8243854395
:104AB000503504950D9D50328543503503950B9D1F
:104AC00002928543503501950A9D72468543824383
:104AD0008643874350351F200002009513258343EA
:104AE0002D025B192360099B814383435B1963603B
:104AF000634683435B194919A360E160089D503206
:104B00000B218543490296466A182261079D50365B
:104B100085436A186261069D864385436918A161D1
:104B20000321C9027218E261059D503785436A1856
:104B30002262049D874385436A186262039D854310
:104B40006A18A262029A82435218E262019D85436A
:104B50006A1822637A186263009D85436A18A2630B
:104B600072468243511800250700E163AE00A05948
:104B7000C004C00EFFF719FFA159C006C00CB9430D
:104B80006D1C01432D062D0E102DA151EED313B037
:104B9000F0BDF0B588B0FF490A6A1206130F4A6AE1
:104BA0001206120F120113438A6A1206120F120222
:104BB0001343CA6A1206120F120313430A6B12063A
:104BC000120F120413434A6B1206120F12051343FD
:104BD0008A6BC96B1206120F09061206090F1343DE
:104BE00009070B43EC494A68D11DFF31FA310C69C2
:104BF0000B610C6B0B630924A4011219D468D360F8
:104C0000E44BDC682406260F04969C6835012406D4
:104C1000240F03942C431D692D062E0F35023703F4
:104C20002C43059700962600A6465C693E43240661
:104C3000240F0194240426430694019C27059C69B3
:104C40003E432406240F2506DC692E435C73C134E1
:104C5000010000006C4900A000020000FD0A12C71C
:104C60002406240F24072643029607965B68BC4659
:104C70001B061F0F039B1E013B003343049E059F31
:104C800036023343009E3B4336041E4367463E4391
:104C90002E432643072803D0062801D00A2809D12D
:104CA000906802989060C8680798C860C86ACE6229
:104CB00008B0F0BD0528FBD19068019E7046360310
:104CC0003043069E3043664630432843204390607D
:104CD000CA68C860C86A06980343604603432B430A
:104CE0002343CB62E4E7F0B5AF48016842680907A7
:104CF0001207090F120E11438268036B1207120D7F
:104D00001143C2681207120C114302691207120BF9
:104D1000114342691207120A1143826912071209EC
:104D20001143C2699446120711439646026A14075A
:104D3000426A240F1207120E1443826A1207120DE0
:104D40001443C26A1207120C14431A07120F1504F7
:104D50002C43456B26002D072D0A2E43856BC06B17
:104D60002D072D092E430007064390484568E81D8E
:104D7000FF30FA3047684160876886601605344323
:104D8000120614431A07144309229201AA18136841
:104D900011605368546062461207120F13011343E7
:104DA000140223431403234314042343140523430D
:104DB0001206134372461343426A4162816A836258
:104DC000F0BDF0B5784908684A69C004C50E486866
:104DD000D204C004C00E400105438868D20EC0044E
:104DE000C00E80020543C8685206C004C00EC0034E
:104DF00005430869CB69C004C00E0405254315436B
:104E00008A69DB04D204DB0ED20E5B011A430B6A03
:104E1000AC46DB04DB0E9B021A434B6A4D6BDB0492
:104E2000DB0EDB031A438B6AED04DB04DB0E1B0590
:104E30001A43CB6AED0EDB04DB0E5B061A430B6BE9
:104E40006D01DB04DB0E2B438D6BC96BED04ED0EA6
:104E5000AD022B43C904C90E4701060093A66EE3B9
:104E600001000000684B00A00002000009E2AC7ADB
:104E70003E4387023E43C7033E4326434006064364
:104E800048010C000443880204434D48CD034068A8
:104E90002B430100FF302C43FF30801C45696546E1
:104EA000456187698261C769C361436B33004663AB
:104EB000866B8363C66BC3630800092189014018B0
:104EC000016905614169426181698461F0BD10B584
:104ED0000400FFF712FF2000FFF76FFEFFF77BFFD4
:104EE00010BD37494968FF31FF31891C0A6A000744
:104EF00012091201000F02430A62086A0F2212030C
:104F00009043086270472E494968FF31FF31891C80
:104F10000A6AF02300079A43000E02430A62086AF5
:104F20001A0390430862704730B50400244D0428EA
:104F30000CD21120FFF758FD6968092292018918E7
:104F4000C9698904C90E884200D204246868FF3008
:104F5000FF30801C016A0F22120291432207120DBA
:104F60001143016230BD164A10B553680522D201C3
:104F70009A1813691F246406C006A34380080343DC
:104F8000136110696311C9069843C9090843106188
:104F900010BD0B4A10B553680522D2019A18136947
:104FA0001F24E403C006A343000B034313611069ED
:104FB0006311C9069843490C084303E05CD200B072
:104FC000005A00B0106110BDF94A10B552680523AF
:104FD000DB01D21813691F246401C006A343800DAE
:104FE000034313611069C90640094001C90E084313
:104FF000106110BDEE4A10B552680523DB01D218CE
:1050000053691F246401C006A343800D0343536109
:105010005069C90640094001C90E0843506110BDDE
:105020000C2010B5FFF7D5FC04001120FFF7D1FCD0
:105030002100FFF7DFFF1220FFF7CBFC0400132055
:10504000FFF7C7FC2100FFF78EFF1420FFF7C1FC1C
:1050500004001620FFF7BDFC2100FFF79AFF172080
:10506000FFF7B7FC04001920FFF7B3FCB9F2A47EE8
:1050700001000000644D00A000020000101A720A36
:105080002100FFF7ABFF10BDCE4905224968D201D0
:1050900089180A699205D20E824206D30A69D2069D
:1050A000D20E824201D8082070470A691203D20E3C
:1050B000824206D30A695204D20E824201D80420E9
:1050C00070470A699200D20E824206D30A69D20161
:1050D000D20E824201D8022070474A699205D20E50
:1050E000824206D34969C906C90E814201D801200E
:1050F000704700207047B34949688031CA6AFF236E
:10510000E13300079A43C00D0243CA627047AD49BC
:1051100000B549688031CA6AC30652095201DB0EE4
:105120001A43CA62FFF7B0FF0006000EFFF7E3FF65
:1051300000BDA4494968C0314A69FF23E133000733
:105140009A43C00D02434A6170479E4900B54968C1
:10515000C0314A69C30652095201DB0E1A434A6143
:10516000FFF792FF0006000EFFF7E3FF00BD954931
:105170004968FF3141314A6BFF23E13300079A430D
:10518000C00D02434A6370478E4900B54968FF313C
:1051900041314A6BC30652095201DB0E1A434A637E
:1051A000FFF772FF0006000EFFF7E1FF00BD854923
:1051B0004968FF31491C4A69FF23E13300079A43DC
:1051C000C00D02434A6170477E4900B54968FF310E
:1051D000491C4A69C30652095201DB0E1A434A614F
:1051E000FFF752FF0006000EFFF7E1FF00BD754913
:1051F0004968FF31FF31891C0A6A0F235B060007EB
:105200009A43C00802430A6270476E4900B5496874
:10521000FF31FF31891C0A6A1F231B059A43C3060D
:10522000DB091A430A62FFF72FFF0006000EFFF7A3
:10523000DEFF00BD70B505000D20FFF7DFFB614903
:105240004E68092189017118CA699204D20E9042F0
:1052500001D2012200E000225A480024401C035DD4
:10526000AB4204D0641C2406240E022CF7D3086A37
:1052700018255543534A000C000408325ADD81E8D2
:1052800001000000604F00A000020000E4F2CCB773
:10529000535B18430862486A000C0004AA1853883C
:1052A00018434862886A9388000C00041843886297
:1052B000C86AD388000C00041843C862086B1389BD
:1052C000000C000418430863486B5389000C000469
:1052D00018434863886B9389000C00041843886363
:1052E000C86BD389000C00041843C8630520C001B3
:1052F00030180368168A1B0C1B0433430360436891
:10530000568A1B0C1B04334343608368968A1B0C2C
:105310001B0433438360C368D28A1B0C1B041343F2
:10532000C36030232C4A634338329A18535B0C6AAB
:105330001B042404240C23430B62521953884C6A27
:105340001B042404240C23434B6293888C6A1B04A3
:105350002404240C23438B62D388CC6A1B042404CA
:10536000240C2343CB6213890C6B1B042404240CF0
:1053700023430B6353894C6B1B042404240C2343E9
:105380004B6393898C6B1B042404240C23438B6391
:10539000D389CC6B1B042404240C2343CB63118AD4
:1053A000036809041B041B0C19430160518A4368FC
:1053B00009041B041B0C19434160918A836809048A
:1053C0001B041B0C19438160D18AC26809041204B2
:1053D000120C1143C16070BD005A00B055494A68B3
:1053E000092189015118CA691F235B02C0069A432B
:1053F000800C0243CA61C869012292049043C861CB
:1054000070474C494968C0314A690F239B03000724
:105410009A43800B02434A617047464900B5496888
:10542000C0314A691F235B029A43C3069B0C1A438F
:105430004A61FFF733FE0006000EFFF7E2FF00BDF2
:105440003C494A68092189015118CA69FF23E1339F
:1054500000079A43C00D0243CA617047354900B541
:105460004A68092189015118CA69C30652095201C3
:10547000DB0E1A43CA61FFF711FE0006000EFFF7AC
:10548000DFFF00BD10B504000D20FFF77F889E549C
:10549000010000005C5100A0000200009AE96B07C7
:1054A000C1FAFFF7A5FF1620FFF7B1FAFFF7C1FE1B
:1054B000E00614D50120C007C07CC1070FD000074B
:1054C000400F02282AD0032809D11620FFF7AAFA94
:1054D000FFF78EFF1620FFF79AFAFFF7AAFE1620B5
:1054E000FFF795FAFFF7C4FF1620FFF790FAFFF7D2
:1054F0009EFF1820FFF78BFAFFF71DFE1620FFF71F
:1055000086FAFFF736FE1620FFF781FAFFF750FE06
:105510001620FFF77CFAFFF76BFE10BD1120FFF796
:1055200081FAFFF765FFDAE7084881680122120770
:10553000914381608168C205914381608168521006
:105540009143816070470000005A00B0802A0080BB
:1055500070B506000C0015001BF042FF604A3101D7
:105560008918002D03D0002C06D1091D04E0002C61
:1055700001D0083100E00C310C681BF035FF200031
:1055800070BDFFB585B014000D001E001BF028FF94
:105590000190534829010818010008310F1D002E01
:1055A000049105D0002C01D0010006E0011D04E0AB
:1055B000002C01D0049900E03900494B09681A0019
:1055C00060329646121D0392121D9446121D002E43
:1055D000029204D0002C724605D1039A03E0002CFD
:1055E000624600D1029A059B12681500002E03D076
:1055F000002C06D1001D04E0002C01D0049800E02E
:10560000380003600598904202D9059D012727E0E4
:10561000914244D10598814241D9314B012700255F
:105620002800002E08D0002C02D00101C9180CE07F
:105630000101C918091D08E0002C03D00101C91897
:10564000083102E00101C9180C310968A94200D9EA
:105650000D00401C0628E4DB954220D0002F1ED010
:10566000002E04D0002C704605D1039803E0002CD6
:10567000604600D10298002F056010D0002C09D0A0
:10568000002E03D0280000F078FA08E0280002F08D
:10569000F8FD04E0002E02D0280002F0D634580AAB
:1056A00001000000585300A0000200006E01D5BAAE
:1056B000D9FD01981BF0A2FE280009B0F0BD0E48EC
:1056C00010B50068002801D0FFF738FF10BD012297
:1056D000130060E7012200235DE7002201235AE75F
:1056E0000022130057E7012211003BE700220121AD
:1056F00038E700009CD200B0506600B010B502F050
:10570000BDFE10BDF949FF22C832888B1042FCD182
:105710007047F8B5F64C6069002802D01BF06AFEAD
:10572000FEE71BF067FE606100210120FEF788FFA5
:10573000002810D0EF4EB488012080020440B088C9
:10574000EC4D3527A0433F012035B84204D1287DD8
:10575000012108432875F8BD022000F01CFB002839
:10576000F9D03C43B480297D012001432975F8BD5F
:10577000DF4810B5446900214161FF210170DD4817
:105780002030017D4908490001750120FEF77AFFAC
:1057900020001BF033FE10BD70B5D54C60690028A9
:1057A00002D01BF027FEFEE71BF024FE6061002103
:1057B0000120FEF745FF00280DD0CE4DAC8801201A
:1057C00080020440A888A04305D0012000F0E3FA3D
:1057D000002800D0AC8070BDC54810B544690021D8
:1057E0004161FF2101700120FEF74CFF20001BF0FA
:1057F00005FE10BD70B5BE4E7069002802D01BF0CA
:10580000F9FDFEE71BF0F6FD706100210120FEF7B7
:1058100017FF002814D0B74DAC8801208002044047
:10582000A888A04382280BD02888F080002000F0B0
:10583000B2FA002804D0A888308182200443AC80CA
:1058400070BDAB4810B5AB49028944698A80C288F3
:105850000A8000214161FF2101700120FEF712FF43
:1058600020001BF0CBFD10BD70B5A14D686900286C
:1058700002D01BF0BFFDFEE71BF0BCFD68610021FC
:105880000120FEF7DDFE00281BD09A4EB4880120CF
:1058900080020440B088A043022812D0FDF7F7FA36
:1058A000002803D0012803D13F2002E05EE1A1B22D
:1058B00001000000545500A00002000077F90BCA57
:1058C0001A2000E07F203188E9803080B08828816C
:1058D00002200443B48070BD8A4810B58A49028909
:1058E00044698A80C2880A8000214161FF210170D9
:1058F0000120FEF7D1FE20001BF08AFD10BD70B51F
:10590000804C6069002802D01BF07EFDFEE71BF092
:105910007BFD7B4D6061AC88012080020440A8883B
:105920007A4EA043B04206D0042000F03EFA002890
:1059300001D03443AC8070BD724910B54869002273
:105940004A61FF220A701BF063FD10BD70B56D4CFB
:105950006069002802D01BF057FDFEE71BF054FDE4
:10596000606100210120FEF775FE002810D0644D13
:10597000AC88012080020440A888654EA043B04254
:1059800006D0042000F011FA002801D03443AC8086
:1059900070BD5C4810B5446900214161FF21017070
:1059A0000120FEF779FE20001BF032FD10BD70B51E
:1059B00005000E0002F06CFD534C2034258102F0EE
:1059C00067FDA68002F064FD70BD70B5050002F0B1
:1059D0005FFD4D4C2034258102F05AFD207970BDC9
:1059E00030B505000C00FFF797FE454B20331D81B5
:1059F000FFF792FE9C80FFF78FFE30BD30B50500AB
:105A00000C00FFF789FE3E4B20331D81FFF784FE1B
:105A10009C80FFF781FE30BD10B50400FFF77CFECF
:105A2000374B20331C81FFF777FE988810BD10B5E7
:105A30000400FFF771FE324B20331C81FFF76CFE30
:105A4000187910BD70B504000D00FFF7BEFF2843A4
:105A500001002000FFF7ABFF70BD70B504000D0022
:105A6000FFF7B3FFA84301002000FFF7A0FF70BDC0
:105A700024484178002909D12649096801220902F0
:105A80004270090F02002032515C817080787047AB
:105A90001C4910B5C878002815D108611D48406818
:105AA0000A008007800F103210230124002807D03D
:105AB000012803D0022803D0032803D12CD701EDFD
:105AC00001000000505700A0000200008311B577CC
:105AD000136001E030201060CC70086910BD1248DE
:105AE000803000880006000E704700B5FFF7F7FF12
:105AF000022805D10C4840688007800F012800D09B
:105B0000002000BD094B59683822914310400843DA
:105B100058607047003800A8C85A00B000080090CC
:105B20005053000050130000002000800029008026
:105B3000A84B59680F2292019143104008435860C6
:105B4000E7E710B50C00FFF7F3FF2000FFF7DAFFDF
:105B500010BDA14810B5446900214161FF210170C9
:105B60000120FEF7A3FD20001BF05CFC10BD70B50A
:105B7000994C6069002802D01BF050FCFEE71BF036
:105B80004DFC606100210120FEF76EFD002811D060
:105B9000924DAC88012080020440A888B526A0431D
:105BA0003601B04206D0022000F009F9002801D0E9
:105BB0003443AC8070BD10B502F043FB10BD884883
:105BC000C16889008908C160C16803229207114336
:105BD000C160810C7F488030416182490161824906
:105BE00041610521016194E7804800B50068002803
:105BF00001D0FFF7E4FF7E491620C86048607D4869
:105C00008168C2051143816000BD7B4910B50968F8
:105C100044F33CE98905800A084301D01BF02AEDD2
:105C200010BD76E775E775480068000701D50120CB
:105C30006FE700206DE76848C0686AE7F7B586B08F
:105C400004000D001BF0EAFB009000210120FEF78C
:105C50000BFD002854D003216200080090400490FE
:105C60002000083840000E008640039020001038C5
:105C7000059242000B00934002922200183A520013
:105C800091408E4601210F00874001935C480B0034
:105C9000A34094465A4A4030002D39D0082C04D2F3
:105CA0001568049EB543156012E0102C03D25568A8
:105CB000B54355600CE0182C04D2C569019EB5436C
:105CC000C56105E0202C03D2056A7646444EA84003
:105CD000010000004C5900A0000200004408B72A4F
:105CE000B5430562089D002D15D0102C03D2946891
:105CF0001C43946002E0426A3A4342628268022393
:105D00001A4382603F4A80325068DB051843506076
:105D10003E48416055E03B4A803210680821884384
:105D200010604EE0082C09D21668059DAC46049D13
:105D3000AE436546A9400E43166021E0102C0AD2FE
:105D40005568AC46039DAE466546B5437646B140C0
:105D50000D43556014E0182C09D2C669029DAC466B
:105D6000019DAE436546A9400E43C66108E0202C64
:105D700006D2056A7646B5436646B1400D430562D4
:105D80000899002917D0102C03D29168994391608B
:105D900002E0416AB9434162816802229143816015
:105DA000184A80325068012109068843506017491B
:105DB0000020486005E0134980310868082210433C
:105DC00008600120FEF77CFC00981BF035FB09B051
:105DD000F0BD10210A2803D2044940003031095A8D
:105DE0000348018001209EE600290080C85A00B0C7
:105DF00000080090002A0080170000FF102000001B
:105E0000506600B0C0220080009100A844C800B0D5
:105E10000020008000020090044903480860044903
:105E2000001F007808707047085B00B0F05900B0A0
:105E3000EC5900B070B505002924FFF7A2FE200040
:105E4000FFF7D7FD29002000FFF7C5FDFFF78BFE08
:105E500070BD704710B50400FFF793FE002C0AD008
:105E6000FFF72AFE000706D42C211920FFF7B3FD07
:105E7000FFF779FE10BDEE211920FFF7ACFD602180
:105E80001A20FFF7A8FD6C212820EFE710B5FFF7D7
:105E900003FE052806D0062806D00A2806D17D2153
:105EA000090205E0324903E0324901E00121C9035A
:105EB000314A93681B041B0C0904194391609168D3
:105EC00002231943916091680424214391600728BB
:105ED00002D190689843906010BD01205178B42D94
:105EE00001000000485B00A000020000B0E009973C
:105EF00010B5FFF7B9FF26480168C20B11430160D6
:105F00000168490849000160000C10BD70B5FAF73E
:105F1000D3FE1F49CA0B0028086805D0104308604B
:105F200008680122104304E0104308600868400834
:105F3000400008600020FFF797FF144C403CA06B26
:105F400021050843A063A06BC9100843A063A56B9B
:105F5000FFF7ACFD052805D0062805D00A2805D195
:105F60000C4804E00C4802E00C4800E00C48290E04
:105F700009060143A1630B49086802221043086027
:105F8000080C70BD143B0000AB7A0000402100807B
:105F9000002800808509040020DF0300705E0400F3
:105FA00068310400002C008070B5FFF77FFDFC4BCA
:105FB000C1005A58FB4814010DD4C468FA4D2C4056
:105FC000C4604468A400C46802D501252C4301E0E4
:105FD00064086400C46044683D25AD062C40AA43B3
:105FE000144344608268CB185B68920E92069B0152
:105FF0009B091A438260436801229206134343605F
:10600000836813438360E648E84A84304358D3608A
:1060100008184068906070BD10B5FFF747FDE44A6E
:10602000D16AE44B80001940DD4B58331858E14BDE
:10603000DB4318400143D16210BDFEB504000020CF
:1060400001901BF0FFF9DC4E0090B068844237D01D
:10605000F069002804D0002C02D1012001902FE02B
:10606000D64F3D6A1020054007D1386A10210843F9
:1060700038627D20C000FFF7DCFDFFF795FFC948BF
:10608000012241685207002C07D011434160C168CA
:1060900001221143C160B2600CE091434160C168CC
:1060A00049084900C160416801229206914341605C
:1060B0000020B060002D03D1386A10218843386277
:1060C00000981BF0C3F90198FEBDFEB50500002045
:1060D00001901BF0B7F9B84F0090F868854229D0BD
:1060E000F869002804D0002D02D1012022FAF5FE23
:1060F00001000000445D00A000020000A918D7E7DD
:10610000019021E0B34C266A01200006064008D128
:10611000206A01210906084320627D20C000FFF7A4
:1061200092FD216A0820002D03D001432162012045
:1061300002E0814321620020002EF86004D1216A30
:10614000012000068143216200981BF089F9019823
:10615000FEBDF8B5002506001BF07EF99B4C0090B3
:106160002069864231D0E16996489B4F002903D0CF
:10617000002E03D1012528E0002E19D0416A012606
:1061800031434162FFF79CFC94494000085A642364
:1061900058430009F8627D21C90043F3B0EE310095
:1061A000002800D001003963A661666126610CE019
:1061B000416A4908490041627D208001F862082057
:1061C00038630020A0616061206100981BF048F9ED
:1061D0002800F8BDF8B5040000251BF03DF97B4E02
:1061E00007007069844223D0F069002801D0002C98
:1061F00007D0B369734802214022002B03D1002C41
:106200001BD0012514E0002C17D00400806A08433D
:10621000A062A06A1043A062FFF752FC062805D9CD
:10622000A06A3C2188431C210843A06201207061C0
:1062300038001BF015F92800F8BD836A9343836288
:10624000826A04239A438262826A8A4382620020BD
:10625000EDE7F8B5040000251BF0FEF85B4E0700E3
:10626000B06984421FD0F069002801D0002C04D00E
:106270007069002803D0002C01D1012513E0FFF73D
:10628000D5FE5048816AC20C002C04D011438162B3
:106290000120B06107E0914381620021B161C16AD0
:1062A00004229143C16238001BF0DAF82800F8BDDF
:1062B000F8B5040000261BF0CFF8444F0090F869B1
:1062C00084423DD0B8683F4D00280BD0F8680028C4
:1062D00008D03869002805D07869002802D0B8694C
:1062E000002803D1002C13D0012629E0002C0FD068
:1062F000A8690F2109040322884352049C8725487A
:1063000001000000405F00A0000200005DF0695A3B
:106310008018A861286A884380182862FEF732FA3C
:1063200001200CE0FEF735FAA86900090001801C85
:10633000A861286A00090001C01C28620020F861D9
:106340000620FFF70CFA01F0A4FF0620FFF70AFA77
:1063500001F0DDFF00981BF08DF83000F8BD2048FB
:10636000C069704770B5040000251BF07FF8060077
:10637000FEF7F0FA002801D0002C0AD1FEF7EAFA65
:10638000204306D01648C06901E0FEF73BFA00281A
:10639000FBD030001BF06EF8280070BD10488068FC
:1063A00070470F48006970470D48406970470C48B6
:1063B0008069704710B50024FEF7CCFA002800D0A1
:1063C0000124200010BD000050000004002F0080B8
:1063D0000300FCFF8026008000210080F9FF000000
:1063E000285B00B000280080403D0080009400A899
:1063F0000000000470B51D4C2068002811D1FFF783
:1064000069FB0500FFF766FB19494000085A194A65
:10641000E900515864235843C90F491C43F378EDF0
:10642000206070BD114901204860704710B501F02F
:1064300087FFC7E770B5040000251BF017F80B496C
:10644000896800290DD10C490C220B68002C06D05C
:1064500093430B600A6804231A430A6001E09343E4
:106460000B601BF007F8280070BD0000285B00B02F
:106470000000000450000004002F008070477047A7
:10648000F8B58A48017801297ED0012101701AF0FF
:10649000EDFF00908648422143F3D8EB0121844A66
:1064A000C90700200B781354491C401C0A28F9DB4B
:1064B000804900200B781418491C401C0B28A3723B
:1064C000F8DB7C48903801785175017991754179F4
:1064D000D175017A1176417A5176017B9176407BB4
:1064E0007449D076803900200B781418491C401C60
:1064F0000A282377F8DB6F4950390A7E6C48203030
:1065000082710A7FC271497F01726A49BD85269CEA
:10651000010000003C6100A000020000552F988798
:1065200030390A7842724A7882728A78C2720A795D
:1065300002734A7942738A7982730A7AC2734A7AF9
:1065400002748A7A42740A7B82744A7BC2748A7BA0
:106550000275CA7B42750A7C82754A7CC2758A7C48
:106560000276C97C4176584930310A7882764A7879
:10657000C2760A7902774A794277544A137C837744
:10658000927CC2770A7F20300270497F41704E4E64
:10659000042010368446B078EE2800E03EE0FAD1C0
:1065A0006046F070FF20B07000222FE0B078EE2837
:1065B000FCD10C245443464B1959F170080A307130
:1065C000080C7071080EB071FF20B070002903D163
:1065D000B078FE28FCD11BE03B4FE51869681A37FC
:1065E000B078EE28FCD1384813300B780370491C82
:1065F000401CB842F9D9364B68681B59C01888420C
:106600000DD8287AB070521C1206120E6245CDD3F6
:1066100000981AF039FF2A4800210170F8BDFF20C8
:10662000B070DDE7284810308078EE2800D131E7DF
:10663000704770B5FBF73BFD2648002200680D212E
:1066400000F3CDFB0120FDF7E0FB234D2C6804E0B7
:106650006068002800D080472468002CF8D1FFF73C
:10666000E1FFFBF71AFDF1E71C4810B5FEF2C0FA96
:1066700010BD10B5134C203C6360E260A160206047
:106680001BF0B2E820611BF0C0E860611BF0CCE8B1
:10669000A0611BF0DAE8E061FEE710B504001AF033
:1066A000EFFE0D4B19680A0000E00968002902D0CE
:1066B000A142FAD101E022601C601AF0E5FE10BD93
:1066C000485B00B02CD300B09002008080000080B6
:1066D0002C010004800E00049C0E000444160004EB
:1066E000004870470F1D0F12704770B57D240500DC
:1066F000010024022000FFF730F829002000FFF7F6
:106700002FF829002000FFF72EF829002000FFF7BE
:106710002DF870BD10B5040001000020DDDBADC018
:1067200001000000386300A000020000A1C7263A63
:10673000FFF71DF821000020FFF71CF821000020C2
:10674000FFF71BF821000020FFF71AF810BD012009
:10675000D5E70120E8E7414A002010B504000C21EC
:10676000414389180B7A002B03D04968A14200D914
:106770000C00401C0228F2DB05212000FEF7F7FF89
:1067800005212000FEF7F6FF05212000FEF7F5FFAA
:1067900005212000FEF7F4FF10BD0C2358432F4ABB
:1067A000012180180172D6E70C2358432B4A00219F
:1067B00080180172CFE72A4909784172294909787E
:1067C0004181704770B50124002800D0264C274D28
:1067D000A868A043A8600220FFF753FAA8682043E6
:1067E000A8602348FFF74DFA70BDF8B50125AD0547
:1067F000204C214E214F012815D160686900884343
:1068000060606068284360603068018CE20D11436D
:10681000018400F355FC3868C18A220C1143C182FF
:1068200000F35AFCF8BD00F34BFC3868C18A4904F8
:10683000490CC18200F350FC3068018CFF22521CCD
:10684000914301846068A8436060F8BD10B5FFF70C
:1068500051FF7321000E0902401810BD545B00B0B7
:10686000A1E50004A0E500040100000480210080EF
:10687000DC0500004023008064EA000434EA0004E0
:1068800010B537F39FFB10BD10B537F35EFB10BD9D
:10689000704710B504000020C0432060464880794E
:1068A000042805D003281AD1002024F33FF92060E2
:1068B00042480068401C0BD0012024F337F92168BE
:1068C000884203D2012024F331F900E0080020605F
:1068D0003B488178002904D00079002801D10020AC
:1068E00010BD012010BD704710B50A78012A0BD0E9
:1068F000022A09D0032A1BD1012819D13148007876
:10690000012813D0022202E0012804D10122002133
:1069100008000B0008E003280AD188784B780002B1
:10692000034300210122080000F077F838EAD4730D
:1069300001000000346500A000020000B83FF84AE2
:10694000012010BD002010BD38B500240878F128C2
:1069500007D0F22805D10320009001206946FFF7F7
:10696000CDFF200038BD70B5050038F3A2F900282E
:1069700003D104F052FB002801D0012400E00024E0
:10698000002D02D038F387F900E00020204370BDCD
:1069900010B506F0ABFE10BD102010B504F042FBA0
:1069A00010BD10B50C4C6078002803D001F3ECFD4D
:1069B000002060700120FBF7CBFB002801D102F022
:1069C000DCFB02F06EFAFDF747F810BDD0D10004F1
:1069D000E0E900046CE600046C5B00B0F8B50D0063
:1069E000060000200090180017001C000D3000F376
:1069F0008DFA0028009018D0002D04D0FC490160C9
:106A00000572466004E0FA49491E0160FF210172E7
:106A10004472220039000A3043F39AE8F5480168CD
:106A2000684600F382FA0020F8BD0120F8BD38B5B1
:106A30000D0011001A061C00120E012D6B4604D128
:106A400019705A7000216A4604E01A70220A6B46D7
:106A50005A706A460223FFF7C1FF38BDF8B500241B
:106A600006000F001AF020FD0500E3483101081868
:106A7000037B43F35CEA050E0E0E04050E000124B1
:106A80000021017341700800FBF7F5FB0021FBF7C3
:106A9000DEFC28001AF00CFD002C07D0002F05D0DA
:106AA0002022012130000223FFF7C1FFF8BDF1B51C
:106AB0000020FBF7E0FB05000098D04E0101CE4816
:106AC0000C182079FF2828D16079002819D0FF28D8
:106AD00017D0A068FBF777FB6179FE2901D1C8497F
:106AE00002E07D23DB00594388420AD20D1A012DB2
:106AF00007D9FBF764FB07003800FBF764FBA842EB
:106B0000FAD9306800220B2100F37DF900980121A9
:106B1000FFF7A4FF00206070F8BD2800FBF7C1FC60
:106B200001002079FCF73BFD6079FF281DD000288B
:106B30000BD0FBF744FB06003000FBF7C8A1CCB23A
:106B400001000000306700A0000200004CD746F7AB
:106B500044FB61797D23DB0059438842F6D9280044
:106B6000FBF7A9FC002801D1012100E000212079D8
:106B7000FCF71FFD00980121FFF77AFFF8BD306890
:106B800000220B2100F349F9F8BD70B506009F49BA
:106B900000014418085C257B002817D0E0880028F5
:106BA00008D0A068FBF719FBE1887D23DB0059437F
:106BB00081420BD8002D03D0032D07D1012070BDD9
:106BC0000021042230000B00FFF73BFF002070BDC6
:106BD00010B50400FBF74DFE8C4821010818017B1D
:106BE000002909D0032906D14078002803D10021CB
:106BF0002000FFF73DFF10BDC0780028FBD000212A
:106C0000042220000B00FFF71CFF10BDF7B5002089
:106C10000C0082B0FBF739FB02997C4A0700230085
:106C200009017B4D002601208C1843F38AE90C0AE8
:106C3000070C0E13373A3E54640A790A50540498EC
:106C4000E08005B0F0BD5654FBE7A1780029F8D0EC
:106C5000E070F6E707002073E078002817D002986C
:106C60005A2201210023FFF7ECFE6770E6702868C6
:106C70001D216A4600F3D1F86B46D8880128E0D080
:106C80000020FBF702FB0121FBF7EBFBD9E7012119
:106C9000029820220B00FFF7D4FED2E702202073D7
:106CA000CFE7029800F0CDF8CBE7207B022801D196
:106CB000042020730020FBF7E8FA0021FBF7D1FB4A
:106CC000607800282AD100210298FFF7D1FEFBF757
:106CD00080FAA060B5E76078002802D02079FF280C
:106CE000AFD128680022192100F397F802980121FA
:106CF000FFF7BEFEA5E728680022092100F38DF802
:106D00002079FF280AD03800FBF7D5FB002801D1F5
:106D1000012100E000212079FCF74BFC0121D3E7A1
:106D2000607800288DD00298FFF7CBFE89E70B78BA
:106D30008A78FF2B01D15A2A04D0202A06D1C9789B
:106D4000012903D1052200210B007AE67BEFAD4F2C
:106D5000010000002C6900A0000200008BCE44AAB4
:106D600070470878FF2804D188785A2801D101207B
:106D70007047002070478878202804D1C8780228FE
:106D800001D10120704700207047254900014018BB
:106D90004078002800D001207047F8B515000600A3
:106DA000022945D12878FF2818D11E4800680028FC
:106DB0003ED01E49096888423AD10068002807D0B1
:106DC000012807D0022807D0032831D107240AE080
:106DD000042408E0052406E0062404E00D2801D17F
:106DE000092400E008240020FBF759FA2A7807005C
:106DF0002100FBF701FB00281AD0094832010121CC
:106E0000101881702978017169784171002138006A
:106E1000FBF731FB0120F8BDEC130000E0A63400C5
:106E200070D300B0880E000440420F00800E0004B2
:106E30000020F0E702001301234A10B59A18937856
:106E40000120002B06D01279FF2A03D01000FCF796
:106E5000BAFB002010BD70B505000020FBF71FFA3B
:106E60000600194829010C18207B022823D1032091
:106E700020737D20C000FEF722FF6078002819D023
:106E80002079FF280BD03000FBF71FFB002801D131
:106E9000012100E000212079FCF795FB02E0FBF7DF
:106EA000A2F9A060002D05D10848002200681E212B
:106EB000FFF2BDFF70BD00212800FFF7E3FDFBF7E7
:106EC00092F9A06070BD000070D300B0880E00047D
:106ED00038B58D21564D4901280042F314EF55492C
:106EE000554842F310EF554C56492268080000926D
:106EF000534A514B0C38FEF27BFE524922681C3932
:106F000008000092504B514A3430FEF271FE226864
:106F10004C4900924D4A143908002B002032383079
:106F2000FEF266FE38BD704710B5FAF75FFF002825
:106F300001D0002201E00022D24342480021243047
:106F400043F350F8002806D13E4924390868401C14
:106F50000860002010BD28210181283070A6A3EA16
:106F600001000000286B00A0000200007F26FA1735
:106F700010BD3C4909680847374800221100183005
:106F800010B543F339F8002806D13349243948684D
:106F9000401C4860002010BD28210181283010BD10
:106FA000283810B542F3FEFF10BD2F231B015843B4
:106FB0002D494018817B491C81732021018120309B
:106FC00070472F231B01584327494018817B491ED6
:106FD000817370472F231B015843234940182030E9
:106FE00070472F231B015843204940182030704719
:106FF0002F231B0158431D494018817B491C817375
:1070000020210181203070472F231B01584317494D
:107010004018817B491E817370472F231B01584301
:107020001249401870470C4900201C390968002992
:1070300002D088680006000E70470D480009000164
:10704000704700008CB600B0F05700003C7000B0F4
:10705000980E000420E500B09C5B00B02C9500B0B9
:1070600038E600B078FB000480D300B050DC00B0FC
:107070000CDF00B070B501253A4C2D07E560FCF738
:1070800044FD39480021006843F310F8A068284304
:10709000A060012070BD10B500F03DF806F047F883
:1070A00000F013F8314801681322114301603049A0
:1070B0001C20FAF799FE2B48816801221207114320
:1070C000816006F06DFB002010BD00B52948142139
:1070D00087B042F3F8ED27481421143042F3F2ED63
:1070E00001220021042003AB07C302002248FF2134
:1070F00091316B4607C3A838204A002320A1FDF236
:10710000E1FB0004000C04D11A4820A12830FCF255
:107110006BF907B000BD38B5204D1F48204C2860E2
:10712000226800921F4A291D0800130018304033BE
:10713000FEF268FD226800921B4A29000C3108000B
:1071400013001C304033FEF25DFD226829000092DE
:10715000084A143108002B68203A2030FEF252FD14
:1071600038BD0000009000A8845D00B066948029BE
:1071700001000000246D00A00002000066DE24670C
:1071800000F003A92D6C0000502101B0600501B092
:107190009FD20000426C654D62785461736B0000B1
:1071A000426C654D6278466C61677300DC6600B0C6
:1071B0004CC800B0980E0004F00601B0300E01B0CB
:1071C000F8B5F9480569681C3DD01020FFF2C6FEED
:1071D0000028009037D0F549002402C0FF220A2180
:1071E00042F3D6EC24E0E80720D0601E0D281DD81D
:1071F000A0000019083800D5002001001A314F29DD
:1072000003DD4F210E2C00D03520009A091A121DE3
:1072100041188C4608E04607C108760F0127535CE9
:10722000B740BB43401C53548445F4D86D08641CDC
:10723000002DD8D10098001D07F05CFADC480168E9
:107240006846FFF29AFEF8BDD749012010B50870D4
:10725000FFF7B6FF01F345FB012007F029FA10BD47
:10726000F8B505000600D04F0C0038781C3E002809
:107270000AD0D0480079C0070BD00020FFF799FD55
:10728000002806D0032C04D03000F4801AF048EB1C
:10729000F8BD0020FFF7BAFC1AF046EB6A7AF868EE
:1072A000921C2300310042F3FFFEF8BD10B501F33C
:1072B00090FCBD490400C8684968884203D1002297
:1072C0001421FFF2C8FD02212000FFF7C9FF10BD05
:1072D000F1B50098C17A857A047A406809020606F9
:1072E0000D43360E6846FFF23CFE2A0021003000B6
:1072F000FFF7AAFCF8BDF1B500270098AB4A01687A
:107300008588C6880C32914203D1052107F073F9B4
:10731000F8BD806824210400283C2181001F290A2F
:1073200005704170310A8670C170A2480079C007AB
:107330002CD00020FFF73DFD002827D00098806862
:10734000C278817812021143427903791202477898
:10735000134302783F023A43964F921E3F8812062B
:10736000120E8F420DD1934F7988994209D17B79C2
:107370003900934205D1801D891D19F048F08D8C8C
:1073800001000000206F00A00002000092369ADA8F
:107390000FFF002803D06846FFF2EDFD29E001272A
:1073A0000020FFF73DFC00982A0B2D0581682D0D6C
:1073B0002800012306F035FF6846FFF2DCFD7F4818
:1073C0000078002805D10520E08020001AF0B2EAFC
:1073D000F8BD7E480168002903D0200088470028B6
:1073E000F6D11AF0ACEA012F09D17748007980076D
:1073F00005D577492000096828308847F8BD7548C9
:107400000078002809D074490888401E0880734914
:10741000E80040184188491C41806848321DC06816
:107420002100052342F34AFEF8BD1CB5C18802299C
:1074300035D02423421C052918D0082913D10381F3
:107440009A5CC15C120211430905090D644A8B0064
:107450005918535C002B06D0891801228A56002A3D
:1074600001DD521E4A7042F3B1FD1CBD0489038147
:107470009A5CC15C120211430905090D80393F294C
:10748000F1D95849048109782830012901D050499F
:1074900000E055490968884701F3BAFB1CBD0100AB
:1074A0001C310191097A3E29DDD005290BD1042038
:1074B000FFF25EFD42490090783901604B48016857
:1074C0006846FFF264FD01A8FFF255FD1CBD10B532
:1074D00080884749884202D1FBF799FB10BD444997
:1074E000491C884202D1FBF784FC10BDFBF7BEF9B2
:1074F00010BDF8B504000F000578407800260002A2
:1075000005432805000D8038402817D31420FFF2CA
:107510002FFDFF21FF31009001608580E278A17886
:1075200012021143C1800021C181241D4773846070
:107530002E4801686846FFF22AFD04E03900200069
:1075400000F0C9FB06003000F8BDF8B50D001B4E79
:107550003178002901D16869F06028894419E888E8
:10756000082806D01DDC012850D0022842D003286C
:1075700074D10C20FFF2FCFC002800906ED0FBF7C9
:1075800075F90F490098183901606278CED0D4623D
:10759000010000001C7100A000020000EC2D3D6AFB
:1075A0002178120211438180856015480168684680
:1075B000FFF2F7FC64E0092832D00A2824D0112811
:1075C00056D1FBF75DF901212000FFF79CFF57E042
:1075D0007C0E000401140000E4A63400A05C00B09E
:1075E00078E6000494F500049BE50004A8E5000497
:1075F000489D0004109E000498E500049CF50004DA
:10760000E0A6340080FE0000FBF73AF900212000DC
:10761000FFF779FF002833D0280042F3E1FC2FE088
:10762000002901D1FFF724FE7168F068884227D154
:10763000A0780930FFF2A6FCFF4900900160627853
:107640002178120211438180A1788171A278E11C16
:10765000C01D42F3BAEA0098FFF743FF009807F015
:1076600002F9002804D1F54801686846FFF299FC48
:10767000280042F3B5FCF06800221421FFF2FFFB62
:107680000020F8BDFEB500220500FF21EC48D243E2
:10769000193142F3CFFC07005BD0A8880005000D2C
:1076A00000900020FFF7C6FA0320F88024203C1841
:1076B0003881A8882070A8881C23000A6070E88898
:1076C000A070009881000918DE480E187078DE4915
:1076D000401C70700098584340184079FFF7BBFC7D
:1076E0000189DA4A08180190A968401A80180290A6
:1076F000EA88824201D8E01C0AE0029AE01C42F3C8
:1077000064EAE8880299421A029801992018C01C7C
:1077100042F35AEACE480078022803D17078401E1E
:10772000707010E000981AF018E9002812D07078F4
:10773000401E7070009801F32EF92070009801F33C
:107740002AF9000A6070EA88390000200323FFF755
:1077500006FFFEBDBF480168002903D038008847F6
:107760000028F6D100981AF0FCE8002806D07078BE
:10777000401E7070380042F333FCFEBDA278B6485C
:10778000D21CC0683900082342F3A2FCFEBD71B5CB
:1077900081B0019AB04E908894680B281A3374D443
:1077A00001000000187300A00002000018C583D774
:1077B00039D2A94983001B1859188B78002B32D075
:1077C000FF23F73300921360009A2389D3800A794C
:1077D000521C0A71A3490978012905D0A4480168FF
:1077E0006846FFF2E8FB1BE021891C230D19584372
:1077F0009A4940189F49407909688847009AA978B2
:10780000D180AA78E91C42F3EAE9009801F3B4FDBB
:10781000200042F3EFFBF06800221421FFF239FB55
:10782000002001907CBD200042F3E4FBF0680022C0
:107830001421FFF22EFB01980028F3D001A8FFF2DB
:10784000AEFB7CBDF1B500998A884E7B1005000D1A
:1078500005000B2822D2920B00D00020864AC300DC
:107860009C182279002A19D0E5808A888968120B31
:10787000002306F0EAFC002E02D16079401C607102
:1078800078480078012805D0794801686846FFF2F9
:1078900092FBF8BD009801F352FCF8BD8868774967
:1078A000096888476846FFF27AFB002EF5D101216E
:1078B0002800FFF719FDF8BD31B50098664D8088A6
:1078C0000005000D84002418295D002912D06849A4
:1078D000096801F3B9F96548017800290AD06119EE
:1078E00001228A56032A05DA4078002802D100983E
:1078F000FFF7D2FE6846FFF252FB38BD01B559488A
:10790000007802281CD0009881888A0B01D00021C1
:1079100001E00905090DCA00574951180A79002AE2
:107920000BD08279002A08D14A79521E4A71808888
:1079300001210005000DFFF7D7FC6846FFF22FFB81
:1079400008BD31B500984C4A81880905490C525C44
:107950004449002A097817D0022912D048490978E9
:10796000002903D047490988002902D0FFF7E1FC2C
:1079700038BD454A454C11788B00491CE0501170C8
:1079800038BD01F30AFC38BD8068012901D04049A7
:1079900000E03A49096888476846FFF200FB01F3B6
:1079A0004BF938BD01B5009880680028EA90C07C8A
:1079B00001000000147500A000020000013D5DA759
:1079C00007D042F321FB2E480022C0681421FFF2A9
:1079D0006AFA0098808819F0D4EF002803D068462E
:1079E000FFF2E7FA08BD009801F3B0F908BD10B541
:1079F000234CE068002817D100212BA0FFF207FAE2
:107A00006060A2681A21FFF24EFA294A60682021BC
:107A1000FFF249FA274A60680421FFF244FA6068DD
:107A20002549E0602348086010BDF0B5002185B00D
:107A300022A0FFF2ECF9124DA860FFF7D8FF214F0A
:107A40000421388801F3C3F801F3D2F8114E002461
:107A5000FFF2E8FA024B039002681233D11A33E0C6
:107A600092130000E4A63400905B00B0109E000466
:107A7000B4B40004D202000098E500047CE60004DF
:107A80007C0E0004FCA93400ACF50004489D000401
:107A90009CF500049BE50004A8E500049CE50004B7
:107AA000E09D000494F5000462745F7364696F00E4
:107AB000DB700000BB6F0000B0EC000462745F6814
:107AC00063690000A4E500049A426FD024DCAC494D
:107AD000531A8A427CD017DCAA4BD11A9A4267D03B
:107AE00009DCFF3AF63A70D0032A6FD0092A54D144
:107AF000FFF7B2FE35E00129F1D0062967D0092948
:107B00004BD101F3C4F82CE0133B42F360EA084D7B
:107B100073787F8446469C4648294AD023DC342922
:107B200065D015DC01296FD002296ED0032934D12C
:107B30000820FFF23BFA92490290363101609249E7
:107B4000097801719148016802A8FFF23EFA24E029
:107B5000452971D0462970D047291ED10321FFF74E
:107B6000A7FB039474E7692968D009DC4F2976D014
:107B70005C2975D0682910D1022106F064FDF0E778
:107B80006A2919D0722908D1EB6869688B4204D13F
:107B9000020017211800FFF286F903980028E1D0AF
:107BA00003A8FFF206FA53E70221D8E74EE00FE000
:107BB00063E0FFF7B5FBD4E782694169294E662788
:107BC00001000000107700A000020000F5D5E31AC4
:107BD000001D019200910FC819F0E4EEE7E750E0B4
:107BE00052E057E030780028E1D06E480088002845
:107BF000DDD068497D2000224F31C00030F374FB96
:107C0000D5E701F342F9D2E706F079FD01F33FFA37
:107C100055E08179808801F3BDF9C8E72BE018E0D1
:107C20008179808801F38BF9C1E780880100803970
:107C30003F2902D806F055FDB9E701F3EDF90399A4
:107C400000228888891D19F0B2EEB0E716E024E022
:107C500038E0007901F33EF8A9E700793070A6E733
:107C6000514A0189118080880421388000F3B9FFCE
:107C70009DE716E01BE001F3C2F898E7FFF7A5FDCA
:107C800079E7FFF7A3FE76E7FFF72AFE73E7FFF732
:107C900049FE70E7FFF769FE6DE744490079087017
:107CA00085E706F0CCFA03A8FFF28DF97FE740687C
:107CB0002969884292D02861287800288ED0FFF761
:107CC000B1FA74E706F0F7FC55E7010000200B2934
:107CD00006D2374AC90089180979002900D0012045
:107CE0007047344810B541693348344A81600021F7
:107CF000016141618161C16102624162FFF246F846
:107D000006F0C0FD10BD0100002000290AD1294A5B
:107D1000D168002906D01378002B03D05268914215
:107D200000D101207047F3B50124060081B08578A9
:107D3000C078000205432002854200D80024002CB0
:107D400025D11C48C1684068814203D102980028AF
:107D500000D10124002C15D000221948110042F353
:107D600087F9002803D1212000F320FF0FE0022132
:107D7000C1802421471801812A1D3100380041F3B8
:107D800042EF00E037000299380006F04DFC200079
:107D9000FEBD000089130000FF01000098E500040B
:107DA000E4A63400AAE50004A8E500049FE5000469
:107DB000489D00047C0E000468E600B0DB70000003
:107DC00074C800B0002101600120704752003FFCE0
:107DD000010000000C7900A00002000032CCE14755
:107DE000002101600848006B8001C00F7047064801
:107DF00040300079C00701D1012070470020704752
:107E000002484068C07A704770DA000470DC0004F1
:107E100070B50124394D6406EC6039480021406892
:107E200042F38AF9AC603748807EC00704D13649F6
:107E30008888621390438880012070BD012B10B5A3
:107E40000BD1324842F3A9F9314800688047002835
:107E500003D13049012009688847002010BD2E4811
:107E600008B502680092264A2C4B103211000839DE
:107E700008001030FDF20CFF08BD2448142110B595
:107E800041F366EF06F064FD254800214068C172A9
:107E90001B48026823488260234A0261234A8161A9
:107EA0004261234AC16102624162224909688162DA
:107EB000002121A0FEF2BFFF22491A4A08601A21C0
:107EC000FFF205F8204B174801211B680D2289029B
:107ED000303098471348FEF263FF002801D001209C
:107EE00010BD1A491920F9F7C5FF0028F8D1034938
:107EF000012040068860002010BD0000009000A80E
:107F0000D05B00B090DA0004C02800A878DC000440
:107F10005CEF000468F00004980E00048CCC00B004
:107F200070DC0004E0E600B0451034004910340075
:107F3000697900002CF000046863695F6D75785FF3
:107F4000666D00003CED000464F000043D79000023
:107F500070B501248A4D6404EC608A4800214069B0
:107F600042F3EAF8AC60012070BD10B50AF00AFED9
:107F7000002010BD08001100012B10B502D1824A6B
:107F800012689047002010BD002070470020704705
:107F9000FEB50020010001907CA0FEF24CFF794C60
:107FA000606109F065FF002179A0FEF244FFA06145
:107FB00062691A21FEF28BFF2600784F1C3600F012
:107FC0003DF9774C774D01E020688047386880475D
:107FD0000028F9D1286880470028F5D13FBFC97C27
:107FE00001000000087B00A000020000C6245FFA28
:107FF000421E009271480122072101ABFBF2B6FA42
:1080000000240CE0E00085196A680A4206D0325864
:10801000200090476968019888430190641C019989
:108020000029EFD1D5E71C3010B5417A092901D0DC
:10803000082917D1624900244472096888476148B9
:108040000068804754488168491E81600178002992
:1080500005D00470806900221421FEF242FF5548C9
:108060000068804710BD70B505004B4E0C00B0692C
:1080700000280ED029682200022342F35BF8002872
:1080800003D0F068844200D9F4604D4928000968A3
:10809000884770BD01004948002210B5FBF2F6FA8E
:1080A00010BD1CB50020020001900090434807213C
:1080B00001ABFBF25BFA002804D10198400700D025
:1080C00001201CBD00201CBD38B505000C00FCF2D1
:1080D00007FD0022D24300923848230001222900E4
:1080E000FBF244FA38BDF8B501250600364CAD0266
:1080F00019F048FA284F00213A69AA1A04E02378B7
:10810000EE2B03D1641C491C8A42F8D8691A002E50
:10811000396101D0691A316019F038FA3869F8BD4F
:1081200010B504002748006880471B482149427861
:10813000944202D10868804710BD447008688047A7
:10814000002CF9D0012C04D17D24E401FBF758FD6B
:1081500003E07D242402FBF759FD03212000FDF7F5
:108160007EFB03212000FDF780FB03212000FDF7AB
:1081700079FB03212000FDF77BFB10BD10B509F052
:10818000A9FE012010BD08B56846FFF7ACFF01202D
:1081900008BD0000009000A8F45B00B07CF0000473
:1081A0006E6663006863695F6D75785F6E66630015
:1081B000C4F20004D0F20004C8F20004104100042C
:1081C000BCF10004CCF20004683C0004254810B562
:1081D0000068C00604D5FFF764FF002836D007E02A
:1081E000FFF75FFF002803D11F48C07C6D8F6AC670
:1081F00001000000047D00A000020000DFDC818A95
:10820000002801D0002010BD06F0AFFE0028FAD0F3
:1082100006F069FE0028F5D106F060FE0028F1D1D5
:1082200019F0E6EB0028EDD107F0FCFF0028EAD0BA
:1082300006F0F9FD0028E6D00AF0E2FE0028E2D0C0
:108240000F4800780028DDD106F0EDFD012803D1AC
:108250000AF0BAF8002803D006F0E5FD0228D1D1D3
:10826000012010BD10B5FFF7BBFF002801D009F0B9
:1082700097FC10BD70470000985900B08CF200B018
:108280002D5E00B0F8B5150006000A4C30202178AC
:108290001A004843084B069FC018491C30602170E3
:1082A00000922B003A00611CF9F2F8FC0006000E67
:1082B000F8BD0000940E000440EB00B070B505005E
:1082C000824A834E1178C807000F3358AB4201D160
:1082D000801907E0491CC807040F11703059A842E3
:1082E00002D1A019406870BD6421280041F3A6EEB8
:1082F0007849020000204300CB5A934202D2401C2E
:108300000928F8D3A1193551486070BD70B5050032
:108310006E4A6F4E51781036C807000F3358AB4283
:1083200001D1801907E0491CC807040F517030596A
:10833000A84202D1A019406870BD6421280041F311
:108340007EEE64490200002032314300CB5A934252
:1083500002D2401C0C28F8D3A1193551486070BDD9
:108360005E485D4A4168114341605D4AC1681143FE
:10837000C16070475B4870B5006800281ED0FDF7EB
:108380003FFC0500FDF74CFC0400FCF7E2FBFCF7AA
:10839000FAFBFCF72CFC2800FCF793FE2800FFF703
:1083A000DFFFFCF737FF2000FDF752F92800FDF74B
:1083B00031F80520FCF7F6FBFCF7B8FB70BD70B593
:1083C000040019F0E9F805002000FFF777FF4149A4
:1083D0006A310C5C2000FCF77EFE3E4960001231E1
:1083E000085A642444437D21A002C90041F326EECB
:1083F000401E052141F322EE3B49401C8AFD884F77
:1084000001000000007F00A0000200002B343F3775
:108410000860280019F0CEF8200070BD70B5040087
:1084200019F0C4F805002000FFF752FF2E496A3109
:108430000C5C2000FCF76BFE2B4960001231085ADF
:1084400064244443280019F0B5F8200070BD70B5CD
:10845000040019F0ABF805002000FFF761FF224986
:108460007A310C5C2000FCF763FE1F4960004A3142
:10847000085A64244443280019F09CF8200070BD79
:1084800070B5174CA068002829D16068002816D163
:10849000FDF7C0FB05280DD0062808D012498B3106
:1084A00007280BD00A2809D10800203004E00E4824
:1084B0009B3001E00C48BB30606000E061606068A8
:1084C0000949407A08390D5CFDF7A4FB0C494000CE
:1084D000085A64235843290041F3BAEDA06070BDE7
:1084E000405C00B0A0ED00B03802000410325476B9
:1084F0000027008022436577506600B044C800B072
:10850000000000047047002811D08807800F0ED0AB
:1085100001280CD0022801D0032808D13B488168EB
:10852000090104D5816801229206114381607047D8
:108530001123374A1B02002910D0012917D0022924
:1085400015D0032912D1510D002890681FD0332374
:108550001B02984390609068084306E000289068EA
:1085600002D0FF21491CF7E798439060704700282C
:10857000906809D0984390609068012149020843AF
:10858000906090680901E7E711214902FFE78843FD
:10859000EBE7F0B50D00C10701D10C2801D912207D
:1085A000F0BD0024400884462BE029786D1C2A7811
:1085B0006D1CFF2A03D10020FFF7BAFF1EE0002345
:1085C000180009E04700BE19B7788F4201D1012396
:1085D000F270401C0006000E0E4E37888742F1D81C
:1085E000002B0BD1300003885B001B1899700188A9
:1085F00049000918CA700188491C0180641C2406BE
:10860000240EA445D1D80020F0BD00000D52E7B3E0
:1086100001000000FC8000A000020000ACE4E44483
:10862000002F008040230080C0ED00B0FF22120226
:108630000240010612021143FF2212040240120AF4
:108640001143000E084370470349FF22C432888B50
:108650001042FCD17047000000080090F8B50024DB
:1086600025000F4E0F4F1049A000355009583020FB
:108670006043C019C46081600C4901610C494161CB
:108680000C4981610C49C1610C4901620C4941628C
:108690000C498162FEF2ACFB641C022CE3DBF8BDEA
:1086A000F0EC00044CD8000400ED00045FFB330044
:1086B00093FB3300D5FB3300F3FB33000BFC33009B
:1086C00075FC330055FC33000C48002110B50160E7
:1086D0000B4802680B488260C1600B4901610B497D
:1086E00041610B4981610B49C1610B4901620B4931
:1086F00041620B498162FEF27BFB10BDE4EC000499
:10870000E8EC00041CD80004F5F933001BFA330030
:1087100035FA330043FA330061FA330099FA330033
:108720007FFA33000278FA49401C0A700278401C34
:108730004A7002784078000202430A81704710B5FF
:10874000F34C0020210062784B690989012A07D087
:10875000022A0BD0032A08D18B4206D3606103E0C2
:108760005A06520E8A4200D2012010BDE94BA2697E
:108770005A43E94BD218A2611A408A42F4D810BD7C
:1087800010B537F3A5FE10BD10B537F3C8FE10BD08
:1087900010B537F3E8FE10BD70B5E04D287800281D
:1087A00033D10021DEA0FEF26EFBE04C00212061FF
:1087B000DFA0FEF268FB60610021E0A0FEF263FB37
:1087C000E0600020A061206900222021FEF2A7FBCA
:1087D000206901222B21FEF2A2FB606900222021E8
:1087E000FEF29DFB606901222B21FEF298FBD64A26
:1087F000E0682021FEF293FBD448442141F3FAEAD9
:108800000120D4492870D2480860002070BDF0B51E
:1088100085B0D1480078002878D137F33DE2DD6695
:1088200001000000F88200A000020000580C5AF974
:10883000BFFE0024E443CE482200002141F354FC53
:10884000CC4F22003860CA48002141F34DFCCA4990
:10885000BB4E086038686A4601890818000C009011
:1088600030692521FEF265FBC3486A46006801892C
:108870000818000C009070692521FEF25AFBBF48D1
:108880001A210180A9490024091D84800181C48026
:10889000012144814180B94A30692621FEF249FB19
:1088A000B74D3A20E880B54A70692621FEF241FBB7
:1088B000B4483A21C1803968F0230A892A815F00CF
:1088C0006B810122AF812A80AB4A6C8012681589C6
:1088D000058143818781048044801089821808893A
:1088E000411801A837F38DFF6B461879F72108402E
:1088F000A54901AA0978C909C90008431871F06897
:108900002521FEF216FBA14B00221B68022110005C
:1089100098479F48006801880322D2029143018052
:10892000002005B0F0BD70B59A4D954C2868002820
:1089300012D1421E98485C2141F3D6FB03212860E6
:10894000C1802030C170286824210181002161800C
:1089500029210028A1800ED02868A188018185499D
:1089600001220968042308607548006941F30AFC84
:108970006088401C6080002070BDF8B5012204238F
:108980006F487C4900690968FEF2C7FA7C48418853
:10899000002948D07F4D24212C68624B21814188D9
:1089A000C088EF274143891CA1806D4924340A798E
:1089B00022704979E01C0907090F617029688988CC
:1089C000A1700121E17021790A0912010832DF2129
:1089D0000A409978CE07B60E32439606F60F3A4013
:1089E000360132438E075206F60F520EF60132431D
:1089F000D609BF27B6013A403243491C4270880766
:108A0000800F9870601D37F3C5FD286800268088A8
:108A1000A41C0655296861488A880068D21C032373
:108A200041F3B0FB2E600020F8BDF8B5E465FEA16F
:108A300001000000F48400A00002000041F48489D9
:108A400000263D49009608695B4F401C0861594863
:108A500035000068002821D1380041F3B1FB554CA6
:108A60002060396800290AD05449096888473800CD
:108A700041F3A6FB206030480021012501712068E8
:108A800000284AD0444A00215180018901260B1850
:108A90009B78C91C8380918001813EE03E4980889B
:108AA0004A88C9885118891C814235D9424841F306
:108AB00087FB0400386800280BD040492000096873
:108AC00088473D4841F37CFB04001B4800210125F9
:108AD0000171002C21D020890126001982782E48AE
:108AE000A280808820810119324800688788038924
:108AF000BA181204DB19120C1B188280FF203130C7
:108B0000824200D9FEE7A288180041F3C2E82B494F
:108B100020000968884700E0012626481E4A0068B0
:108B2000D28881880024891A891E0F043F0C002EE8
:108B30007DD001890E187EE0505C00B00D661900F2
:108B4000FF7F000098EC00046D6465765F736263DC
:108B5000456E630008D700046D6465765F736263D9
:108B6000446563006D6465765F62745F70636D0079
:108B70007D310100C4D600045D8200007CE6000463
:108B8000B4EC0004B45B00B0A0EC0004A4EC00045E
:108B9000B8D60004FCD700040CD80004E7E90004B0
:108BA000A4F800046CEA0004ACEC0004905B00B094
:108BB000840E0004A8EC000498D60004B0EC000475
:108BC0003019FFF7F5FD002834D03019407837F31D
:108BD00013FEC24A1179002906D1401C8007800F7C
:108BE000D0700120107116E0D178814203D1491C68
:108BF0008807800F0EE0491C8907890F814206D142
:108C0000401C8007800F00270125D07020E0401C09
:108C10008007800FD070A41C30190600FFF7CCFD30
:108C2000002805D0300037F3A3FCAD4F0BE018E06F
:108C3000012505E0641CAB4840880019A40E1FB054
:108C400001000000F08600A000020000B51C3A34CC
:108C5000B842BFD9A748874204D1FFF78EFD00284C
:108C600000D0A64FA4494888001948808988081870
:108C7000A349096808819F48A24C87420ED1002D64
:108C80000CD19B480121C180C168491CC1609C482E
:108C90002168006808600120009023E0974887421F
:108CA00001D0002D02D00120009003E09649086811
:108CB000401C08608E480021C18094484A1E41F340
:108CC00027FA934E306001890D18392181800A00FE
:108CD0009049280040F3E6EF280037F353FC216861
:108CE000306808608C4E216870690122052341F3C9
:108CF0005DFA7F4DE888002809D18848406B00283C
:108D000005D18748FDF25EFC84492031C881824844
:108D10002168406901220523FEF213F9009800281A
:108D200013D07549764E4888CA88801848808A884A
:108D300012183068028149888288914205D17949A8
:108D4000096888470020306018E06D480268002AF2
:108D500014D0694E93887088F1884018801C98421E
:108D60000CD910898118B088108177888018DB1B96
:108D7000938000237380928840F394EF6A48664F93
:108D80006A494289F86809680823FEF2DAF8FFF7B1
:108D9000DEFD206801890E186869401C686128782A
:108DA000002813D0E888012805D15D483200310041
:108DB000FDF20BFE0AE056480068002801D041F39E
:108DC0007DF9574832003100FDF299FD4A4821688B
:108DD0004289F868082341F3E9F9FFF7E2FD002032
:108DE000F8BD10B504000020E20702D00800FFF72C
:108DF000F1FC4F490978012914D1210701D5FFF76A
:108E000024FD610601D500F02BF8210601D500F004
:108E100043F8A10501D5FFF71CFE6107890F01D0BA
:108E200000F001F810BD70B50025414E30780128E2
:108E300012D14048384C05702069FEF272F8606922
:108E4000FEF26FF8E068FEF26CF825614EE8679874
:108E500001000000EC8800A00002000072053869E3
:108E60006561E560E561357037F3C0FB3748056043
:108E7000002070BD70B50024334E224D307800289C
:108E800008D12A480022C0682821FEF270F8AC7090
:108E9000EC702C7101203070204804602C48046074
:108EA0002448FDF28DFB00206C6170BD70B5264D2D
:108EB000287801280FD11D4C0022E0682921FEF2FC
:108EC00056F8206900222A21FEF251F8606900223A
:108ED0002A21FEF24CF800242C701E4D2868002830
:108EE00002D041F3F5F82C60134C0A4D2868002895
:108EF00001D021688847184841F376F90028286096
:108F0000F4D170BD505C00B0FFFF00000CD800042D
:108F1000FF070000A8EC0004A4EC0004BCEC000473
:108F2000B45B00B0A00E000490A4340008D7000485
:108F3000F843000438410004B0EC0004FCD70004FE
:108F4000A0EC000498EC0004B4EC00047CE60004FF
:108F5000B8EC0004ACEC000498D6000410B536F36D
:108F60008CFD00210800FFF715FB002010BD00005C
:108F700070B5012500201AF38FFC040003201DF3B7
:108F8000E7FA002804D105201DF3E2FA00283BD0BF
:108F9000012138224A43A05C800705D51019C07909
:108FA000002801D1002504E0491C0904090C082906
:108FB000EFD32800FAF79DFFFF4E30680088C50AFE
:108FC000FEF7C7F80400FAF77FFFE907FB48FC4DFE
:108FD00009D00078844210D90020FAF77EFF30686B
:108FE0000188A94308E04078844206D80120FAF7B6
:108FF00074FF3068018829430180082C04D2F149AC
:10900000A0000A58521C0A5070BDF0B5002595B05A
:10901000ED4F2E000CA80295FAF74FFF24220CA961
:1090200003A840F3B4EE00216B46D97308ABE748C0
:10903000E74AD97200781278024302D001226B46C7
:10904000DA73002802D0012008ABD872E1486B46E1
:1090500099730079002801D0012098737AEB891860
:1090600001000000E88A00A00002000086ED86D41E
:1090700000206B46187358739874D874D876987615
:1090800008AB012418711C206043D849085C0328F0
:1090900001D005285ED1082C25D320000838010412
:1090A000090C01910EF304FA01991E235943091882
:1090B00048797F2801D26B469874487A2C2805D0CD
:1090C0003D2803D00D2801D00C2801D1062004E052
:1090D0006B46D87C002802D102206B46D874012050
:1090E0006B46587336E026F363FF642161436D1CC1
:1090F00009183420405C2D062D0E032801D00128CC
:1091000007D1761C403188883606360EB84200D228
:109110000700200005F0FFF9002803D06B46987E79
:10912000401C987601206B461873200017F328FC2A
:10913000002804D120002BF33FFD002802D001209D
:109140006B46D876200002F014FC002802D00120E3
:1091500008AB1871641C2404240C0B2C93D300203E
:109160006B461874002D587406D0B54204D1012006
:10917000102F187400D2587408AB01205D71FDF7F0
:10918000B0FC08ABD871FDF7C5FC08AB0400187241
:109190009748984B00787D215843C90040F394EFDD
:1091A0000006000E08AB98716B46197B08AB1A7C61
:1091B000914227D16B46597B08AB5A7C914221D111
:1091C0006B46D97B08ABDA7C91421BD1197910AB85
:1091D0001A7A914216D1997A884213D16B46187C3B
:1091E00008AB197D88420DD16B46587C08AB597D80
:1091F000884207D1D87910ABD97A884202D1187B3E
:10920000844201D00420029024220CA903A818F063
:109210005BF8002803D0029903A8FAF74AFE15B0BC
:10922000F0BDF1B501242700694E2100F07841F32B
:1092300053FB002814D0442060436F490025401898
:10924000C16B0098401A002801DB05042D0C7079D1
:10925000210041F341FB002808D0708985420DD8D8
:1092600038007179A0408143717107E042A8099EDE
:1092700001000000E48C00A0000200009F1558A42B
:109280003089854204D338007179A0400843707159
:10929000641C2404240C082CD1D3F8BD514910B50A
:1092A000C968401A802802DD0020FAF74EFE10BD82
:1092B00010B530F3F2FC0400FFF7BDFF2000FFF70C
:1092C000EDFF10BD10B5FDF758FF46498A78904272
:1092D00002D94879002800D00120FAF748FE10BDD5
:1092E000424810B500240C38FAF781FE3F480C388C
:1092F0000178002906D0417A002903D0407800285F
:1093000000D001244248047010BD10B5FFF7E8FFFB
:10931000FFF742FEFFF7CCFFFFF7D4FF10BD38B5D3
:1093200004000820FDF2BAFE0028009007D00521B5
:10933000890212C0374801686846FDF2BEFE38BD9A
:1093400038B50028274C01D1012002E0012801D1C5
:109350000020A0710820FDF2A1FE0028009008D096
:109360002D490160A17901712C4801686846FDF220
:10937000A4FE38BD1B48002901D0022100E00321D2
:109380008170704770B504001500FAF726FE0028BA
:1093900010D01C2068431A4940180079002800D0DA
:1093A00001201F49C969002900D00121012C01D1E8
:1093B000FFF7E0FF70BD70B506000D000120FAF761
:1093C000C4FD0020FAF7CAFD064C0120A840E17850
:1093D000002E41D0014348226A43E170114923E045
:1093E00064EA00046C5C00B000080000DCED00B032
:1093F000FFFF0000D7EA0004D8EA00046CD20004A2
:10940000B4B40004BC5C00B0E204000058D3000413
:10941000C35C00B0E0A6340014140000E4A63400DD
:1094200008D7000470CA00045118897E002903D1AE
:1094300021790843207102E0217981432171E0788C
:10944000002800D00120FAF7AAFD2079002800D0DA
:109450000120FAF7ADFD70BD8143E170ECE70B0030
:109460001100012830B408D00D4A0120D47888407A
:109470008443D470547984435471002BE7303566AB
:1094800001000000E08E00A0000200006BFDE61964
:1094900008D0012B04D0022B04D1012030BC94E76A
:1094A0000020FBE730BC704710B530F300FC0149E9
:1094B000C86010BD6C5C00B070B501250E4CAD04E9
:1094C000E5600E480078002802D004F06DFC07E04B
:1094D0000120FDF7E4FAFAF7CCFB002021F38DFC24
:1094E000A0682843A060012070BD03488168012264
:1094F0009204114381607047009000A8C95D00B0DC
:1095000010B50400F8F730FD1C342104090C0028C4
:1095100001D0002201E00022D2430F4840F320FE98
:10952000002805D10D490868401C0860002010BDC6
:109530000189081810BD10B5040000681C3840F3FC
:10954000E5FD0020206010BD11681C39488170477E
:109550001C38408970470000905B00B0B85C00B0D8
:10956000002310B508E09C000C5B844203D11C482A
:109570009A00885210BD5B1C9342F4D310BD30B5E5
:10958000002409E0A500555B854204D1A0008018A5
:109590008170012030BD641C9C42F3D3002030BD9B
:1095A000F7B59446040000260D4F12E029194988AA
:1095B000B94204D101996246FFF7D2FF07E00906DC
:1095C000019A090E6346FFF7DAFF002800D06753BF
:1095D000761C0349B500605B491C8842E6D1FEBD9C
:1095E000FE0F00000100897E0120002900D000202C
:1095F000704701218140FA48014201D001207047A3
:1096000000207047F8B5F74C658BF6482030868807
:10961000E78B0020FDF7B2F9F348006880471FF39D
:109620008FFBF2490020C87308746583ED48203031
:109630008680E783F8BDFEB507000BF38CFF3C681E
:109640000600A588E01D01AA02A921F31FFD6B46B3
:109650001889242819D1A088882358438019C078F4
:10966000E34E0028207A03D1C007C00F20D104E0C8
:10967000C006800F1BD001281AD1FAF7B8FC0028C9
:1096800015D13078012812D812E0DA494BA6B1A0E2
:1096900001000000DC9000A00002000015E641A9D6
:1096A00088420FD10820FDF20DFDD84900900160DD
:1096B000A1888180617A8171D54801686846FDF290
:1096C00010FDFEBD38000AF3B0FE6B461889D14983
:1096D0008842F6D1CA4A0120917BA8408143917308
:1096E000FEBDF8B500210600CB483EF349FA07005D
:1096F000C94801213EF344FA0400C74802213EF361
:109700003FFA050002203900C0433EF301FA2E6003
:10971000266069680020C04308606968062E4860BA
:109720001BD16A68410091606968C8606968086116
:10973000696848616168B94808606168B84848600C
:109740006168B84888606168B748C8606168B748B0
:1097500008616168B648486125E0696888606A68A0
:109760000021D1606A6811616A6851616A680121EB
:1097700091616968C8616168AE4808606168AE4817
:1097800048606168AD4888606168AD48C8606168DC
:10979000AC4808616168AC4848616168AB48886161
:1097A0006168AB48C8612A002100380000233EF3FD
:1097B0002DFCF8BDF7B582B0039840300778202F14
:1097C00000D92027A348BC080068816E0968A1421F
:1097D00003D1C06E0068A04202D02000FFF781FFD5
:1097E0008D4802213EF3CCF900909B4800213EF3C6
:1097F000F9FB01900298019940683EF3DAFD864832
:1098000000213EF3BDF904600500406803993A0069
:1098100040F37AEA804801213EF3B2F904600399EB
:10982000060040683A00203140F36EEA019B0022B6
:10983000310028003EF370FC0406240E28D028686E
:10984000002824DB834829000068C06E3EF306FB35
:1098500000281CDD3068002819DB7E4831000068D4
:10986000C06E3EF3FBFA002811DD0298019A806871
:1098700001993EF310FE009A009901983EF38EFC88
:1098800000983A004168049840F33EEA00E0002462
:10989000200005B0F0BD70B5040008208365EB39E9
:1098A00001000000D89200A000020000E10EFF14A9
:1098B0002060200014308821050040F3CCEA20000D
:1098C0009C306C21060040F3C6EA002128003EF3DC
:1098D00061F9A060012128003EF35CF9E0600221FB
:1098E00028003EF357F92061002130003EF384FB4D
:1098F00060604E4800213EF34DF906004B480121BF
:109900003EF348F905000220A168C0433EF30AF97E
:10991000206830602168296071680020C0430860B9
:109920007168002348607168886072680021D160A6
:109930007268116172685161726801219161716888
:109940003200C86168684049016068683F49416009
:1099500068683F49816068683E49C16068683E49FF
:10996000016168683D49416168683D498161686895
:109970003C49C161A06829003EF352FB2B480021FD
:109980003EF308F90500294801213EF303F90100DF
:109990002068086028606A68354810606A68354841
:1099A00050606A68344890606A683448D0606A6879
:1099B000334810616A68334850616A683248906180
:1099C0006A683248D0614A68314810604A68314854
:1099D00050604A68304890604A683048D0604A68B1
:1099E0002F4810614A682F4850614A682E4890619C
:1099F0004A682E48D0616368002228003EF396FB37
:109A00002000FEF293FB70BD18CF0000000A00A9F1
:109A1000C8F70004BC5C00B0D0EA00047F2000005E
:109A2000C60C000004AA34007F100000549C0004FF
:109A3000B1B946C1ECDEB8FE49302472ABE9A70FDC
:109A4000E7809CE5190521644B60D2273E3CCE3B64
:109A5000F6B053CCB0061D65BC86987655BDEBB309
:109A6000E7933AAAD835C65AF8EE0004DC9C000405
:109A700096C298D84539A1F4A033EB2D817D0377A8
:109A8000F240A463E5E6BCF847422CE1F2D1176B43
:109A9000F551BF376840B6CBCE5E316B5733CE2B16
:109AA000169E0F7C4AEBE78E9B7F1AFE52209E0586
:109AB00001000000D49400A000020000F8F6216428
:109AC000E242E34F38B50500FB4C2000FFF7F7FEFC
:109AD0004C20FDF20BFBF94900900160E168202267
:109AE0004968083040F38EE92069202241680098D7
:109AF000283040F388E92800FDF2D9FB01006846D0
:109B0000FDF203FB38BD38B504002820FDF2EEFA63
:109B1000821D0090E848A11DFFF760FE010000983B
:109B2000E74A026003D000212030817107E0122251
:109B300026210A54FF222021801D40F3F2E8200054
:109B4000FDF2B5FB01006846FDF2DFFA38BD38B51D
:109B5000040018F301F94620005D202801D1D94DF9
:109B600000E0D94D2820FDF2C1FA821D0090A11D10
:109B70002800FFF733FED14A0099D21E0A60A2885E
:109B80008A8001220028D149A08804D08240087A26
:109B90009043087203E08240087A02430A72200070
:109BA000FDF285FB01006846FDF2AFFA38BD31B524
:109BB0000024FCF7C6FE0098C54A016889181AD02F
:109BC00003290DD005290ED0072912D1BE48FEF277
:109BD000B7FABC48FEF2B4FABC490020C87204E0EF
:109BE000FFF770FF01E0FFF78EFF01246846FDF2EA
:109BF00080FA200038BDFFF7AAFFF6E710B5FCF7A2
:109C0000A2FE10BD10B50400FFF2F1F9200004F02F
:109C10002AFC10BD8079AF49002801D0FF2801D16E
:109C2000002000E0012048727047F8B526F3F2F9F1
:109C30000700012464256543785D002821D01C209D
:109C40006043A5494618307900281AD0A34920005E
:109C5000096888470090B078A1490C2358430968E7
:109C600040188088009940F362EA411C00989D4AA0
:109C7000414312680904090C20009047E91960313A
:109C80000880641C2404240C072CD3D99649002096
:109C90000870F8BD48214143944A10B58C1832F33E
:109CA000F9FE00281DD020002FF33EFF04214020A4
:109CB000015500202FF39BFEC01C80012A3AC5F5F8
:109CC00001000000D09600A0000200000C1E9FD9E9
:109CD00080092FF3FAFF8B4B01221B680100200043
:109CE00098470200210002202FF395FF864A0221A7
:109CF000002020F3FBFF10BD70B504002FF31EFF02
:109D000000202FF37EFE2FF3E0FF0100052220004C
:109D10002FF3A3FF7D48804D03787D482D6802789E
:109D20007C4801782000A8473120005DA0857EE6B0
:109D300048214143F8B57248784F0D180124482056
:109D400060436F494618B54218D04420805D05280D
:109D500001D0092812D1F878210040F3F9FD00283C
:109D60000CD06F48005D012808D13100280034F381
:109D70001BFBB08D082CA88508D304E0641C2404C8
:109D8000240C082CDBD32800FFF7B6FF288A26F323
:109D900074F92876288A26F376F96876F8BD10B526
:109DA000040026F341F9642161430818407810BD8E
:109DB000F8B5050048235843514A584C861858486E
:109DC00001274155E078AF40B8430B00E07040F305
:109DD000A8E906041904042828182800FFF7DFFF63
:109DE00001280ED1B07E00280BD14D4803214155EA
:109DF000A078290040F3ACFD002802D1E078384378
:109E0000E070F8BD4420805D052803D0092801D00A
:109E10000628F6D1B07E0028F3D12800FFF788FF8E
:109E2000ECE738432E49E07000208871F8BDF7B5A3
:109E30004821050010004143314A012789180E00CE
:109E40008E463F21490151184A7A8B789446344A0C
:109E50002036145C3A008240002D1CD013438B70D6
:109E60001C233D004343214FDB199F782D4B1B687A
:109E70001B88BD402B4202D1634613434B722849D5
:109E8000012C1AD0019A022A01D1052200E00422F5
:109E90000A5400210BE093438B7063469343204A9E
:109EA000042C4B7201D0052C07D1002111547246AD
:109EB00091850B4A3175517191711949095CFFF710
:109EC00077FF194800688047FEBD0000FE0E7E192E
:109ED00001000000CC9800A000020000CB079D8488
:109EE0009CEE00B0A60F0000A80F00004C9B0004E1
:109EF000449A0004BC5C00B05EF0FFFFC0BD0004EB
:109F0000B4B400044CF7000498EA00042CFC0004EC
:109F100027E9000470CA000458F80004D7E73300AA
:109F20001CEB000404EB00040CEB0004A0F700049D
:109F300050D2000424EB00041CEA0004BCF7000427
:109F4000F8B5060000202FF366FD05000024FF4F42
:109F5000F969884203D0FE4805631AF3BBF9082E5D
:109F6000FD610CD0102E06D01AF3B4F904061AF3D2
:109F7000B1F9000404431AF3ADF9000204431AF3E3
:109F8000A9F92043F8BDF3B5040083B0F14D687919
:109F900001283FD1F04B00201A68C100565A3607FD
:109FA000360F0A2E04D1565A36093601761C5652FF
:109FB000401C0004000C0E28EED3AE8901204002A4
:109FC000864201D9060002E0402E00D24026002041
:109FD0002FF321FD07001020FFF7B2FF310040F3FF
:109FE000BAE878188601DD48B609EE640068008F8B
:109FF000C107DB4800D001210174017C0172AA89EC
:10A00000E989019200912B7CD64D01222D68310007
:10A010000C20A847D4480078002813D00820FDF26F
:10A0200079F8FF215C31029001602178017161783B
:10A030004171A17881710499C171CC48016802A86D
:10A04000FDF277F84DE40121C04A8140507B8843FE
:10A0500050737047BD4930B51023C5488A780068F1
:10A06000002A2BD0C34AC54C557AC34A24781278AB
:10A070002243002D0DD0002A03D1C14A1278012AB3
:10A0800003D930224A700B7011E03C224A7004223E
:10A090000CE02024002A01D04C7001E02D224A70EF
:10A0A000CA79D20701D00C7001E00C220A708979BC
:10A0B000002902D1C18E1943C18630BDC28E9A4398
:10A0C000C28600204871887130BD012181409F48BF
:10A0D000427B114341737047F1B500248DBAAA63E6
:10A0E00001000000C89A00A0000200003FEF2339E1
:10A0F0000098858825F3ACFF06000098A64B016800
:10A100000027CA1A99427ED01FDCA44BCA1A994272
:10A1100068D013DCA24A891837D04E296BD1A14AE6
:10A12000A14B5188994266D08079012863D150783B
:10A13000002828D10800FFF7D2FF5CE0072A20D0D2
:10A14000412A58D1FFF784FD55E01C2A56D009DC7E
:10A150000F2A44D0142A4ED107214156001DFFF783
:10A160001CFF37E0232A2ED0572A44D18288017A57
:10A170008079FFF770FE00988188C07930F347FB43
:10A1800028E08088D7E708001AE064206843801937
:10A190002030007D01280AD11C20684383494018E3
:10A1A0000079002803D182480178491C01706C4A6B
:10A1B00001219078A94088439070FFF755FF28004F
:10A1C000FFF74BFF17E025F378FF009864238088A2
:10A1D0005843375401246846FCF2A9FF0BE0FFF70F
:10A1E00042FDF7E7017D002905D072494A8B6E498F
:10A1F0008A4200D107752000F8BD04E0817980888B
:10A20000FFF7EAFDE6E78088FFF762FDE2E7FFB5CA
:10A210000020A3B000210A000F9005A81C0006C072
:10A2200025F316FF019024981C2300781D90A18827
:10A230001C91E188A2891B92627A594352081A92B2
:10A24000A27A1992E27B52081692584A8918097923
:10A250001890259815910290FF22082103A83FF33A
:10A260007EED16F324F9002801D1012001E016F358
:10A270001EF9040016F31EF96100081AC10F081830
:10A28000C003000C0D900120109018AB197D4A4BB3
:10A29000259A1B6805A898470124250002E0641C44
:10A2A0002404240C642060430199085C002801D137
:10A2B0000B2CF4D30B2C52D100201090D9E13F4944
:10A2C00020000968884700287AD01C988442FBD077
:10A2D0001C206043354940180079159988426FD198
:10A2E00064206043019940182290C07CFB6E5702A5
:10A2F00001000000C49C00A0000200002617FD49D8
:10A30000012810D11A9925983FF364EE22980E0087
:10A3100040691A993FF35EEE8E42EAD16B46987D12
:10A32000401C9875AAE122981A998069884201DB3D
:10A330001A9801E00006000E1B99179001201029C1
:10A340000BD01B99202908D01B99CA1FF93A04D0B9
:10A350001B99CA1FFF3AFA3A00D103201699229A94
:10A3600041180E06928B360E0121102A3AD0202A6F
:10A3700031E080E1BC5C00B000E800046CD2000475
:10A3800028EA000484EA0004ACD20004A4F7000424
:10A39000C0E80004F4E7000464EA000450D20004BA
:10A3A000D7EA0004D8EA0004D0EA0004BB0C00009D
:10A3B0004F0C000009F4FFFF48E90004FFFF000014
:10A3C000B4B4000470EC0004A0AD000434FC00043C
:10A3D00068FC00046BE005D0D31FF93B02D0FF3BC3
:10A3E0005B1E00D10321229A203292785218120665
:10A3F000120E431813920DE0139A8A4205D9139A4C
:10A40000521E1206120E139204E086424AD9761E9C
:10A410003606360E179A934244D8139A179FB218ED
:10A42000BA42E9D83EE0139833E02598219080198C
:10A4300020901799401E3FF3CEED22980F004169FE
:10A440001298401E1F90081817993FF3C4ED8F42D1
:10A450001CD16B46987D0025401C98752199029867
:10A46000884204D122981F994069401801E0209841
:10A47000401E0121490688421A99259003DB7F225C
:10A4800052068018FFE73FF3A6ED1D911F980006C6
:10A49000000E012D129002D112980128C5D2761E0D
:10A4A0003606360E012D02D1012EBCD203E0002D5E
:10A4B0007ED0012D7DD1642060430199461834205F
:10A4C000805D002875D00428FCD02000FF4A0D993B
:10A4D000126890470C901C206043FD49471838795A
:10A4E000002803D1FB4800780028E3D14036B0882B
:10A4F0001A99884201D31A9801E00006E9ACBFDC42
:10A5000001000000C09E00A000020000D2FF43F442
:10A51000000E1790012014901B9810280BD01B9848
:10A52000202808D01B98C11FF93904D01B98C11FDF
:10A53000FF39FA3901D103201490EC492000096851
:10A54000884711901598002804D13879002801D047
:10A5500002200C90E64901200978002900D070897A
:10A560000C990818401E0004000C0B900020089065
:10A5700001200A9061E00020099025990A9801269F
:10A5800008181E904DE01E981799401E3FF32CEDC1
:10A5900011980F0080191799401E3FF326ED8F4246
:10A5A00037D108986B46401C0004000C0890187DB9
:10A5B0000025401C1875CF480168002908D02000EC
:10A5C000884701E064E03BE0002801D0012000E082
:10A5D00000206B46997D401898750A9914980C9A3A
:10A5E000401A0B990006000E891B1018814206DBE9
:10A5F0001998F82807D10C98864215D903E00C99D0
:10A600000998884210D36B46587D0125401C587527
:10A610000AE00998401C0004000C761C3604360C35
:10A6200009900B988642AED90A98401C0006000E8D
:10A630000A900898002803D10A98149988429AD958
:10A640000B2C03D0002D01D1AB484578012D1FD133
:10A65000641C2404240C642060430199085C0028D5
:10A6600001D10B2CF4D30B2C0FD1A3484078002838
:10A6700008D0A24A0021126805A89047002801D0FE
:10A68000012000E00020109005E0012D00D12AE615
:10A690000B2C27D11098002824D11598002821D1FF
:10A6A0001B99012010290BD01B99202908D01B9938
:10A6B000CA1FF93A04D01B99CA1FFF3AFA3A00D1CF
:10A6C0000320259918AB0E911A7D8D4B1A991D68A0
:10A6D0000EABA847002800D00120012810900F9051
:10A6E00000D10124874A03A9126805A89047109851
:10A6F00001281DD1259818AB401C2590197D1A9A68
:10A70000491C0906090E91421D9101D1CCA6EA3CD3
:10A7100001000000BCA000A000020000DA20B22965
:10A7200000211D9118AB197D189A914201D1002189
:10A7300010911A9A02998918814203DD1098012814
:10A7400000D1C0E50F9800287048407815D0002847
:10A7500002D10B2C27D006E06D4A0021126805A813
:10A76000904700281FD06D4B01201B6825AA1DA90A
:10A770009847012817D10B2415E0002813D0644D09
:10A7800000212A6805A8904700280CD02A6807A94C
:10A7900003A89047002806D06B46187F002802D1F6
:10A7A000D87B1D90E7E7239818AB04802498197D87
:10A7B000017027B0F0BDF7B584B005000AF325FF9E
:10A7C0005749040068000F5A88266E438821A05D0F
:10A7D000794303910290605C022805D05148818939
:10A7E000A943818107B0F0BD0220A055069A0599C2
:10A7F0002800FCF271FF0298A05503980019007D13
:10A800000028EFD1380001A91BF38FFD0028E9D003
:10A81000444801780029E5D0434909688A686B46B5
:10A8200019798B001B18DB69D21A9201192392093E
:10A830005B019A42D6D98089E840C007C00FFCF27C
:10A8400021FFCFE7F8B58200060038480D00101848
:10A85000012282560021AA4201DB002404E00222E8
:10A860008256AA421BDC0124C278A24200D00121F8
:10A870000029C47013D0300006F3CDFD00280ED09F
:10A880000820FCF26FFCFF2182310090016086807D
:10A890008471C571264801686846FCF272FCC9E4FF
:10A8A000F3B5002083B001902FF3DDF800900AF398
:10A8B000ACFE01251C246C430F48015D00297ED0AD
:10A8C000201887781B490C2078430968085A1A49D0
:10A8D000000409680016884706000748005D032841
:10A8E0002CD1280002A91BF320FD002826D001202E
:10A8F00025E0000064FC0004B4B40004D1EA0004C4
:10A9000048F7000420E9000490E6000420E9000470
:10A9100038FC00049CF3000430FC0004AD9DC12A07
:10A9200001000000B8A200A0000200002EC80C9494
:10A93000ACF30004E8B500045099000478EA000480
:10A94000FCB50004F4E7000498EA0004D8F500041C
:10A95000002000280CD06B46187AF9490C23584384
:10A960000968085AF7490004096800168847060074
:10A97000F548C419A07D012803D0032801D004287C
:10A9800058D10AF34CFE88216943081816303B2140
:10A9900020F3C8F902000120EC490190A800085CEE
:10A9A000002847D1E849B8004018816C4B1C0BD0F7
:10A9B000009B591AE44B890140339B8889099942CD
:10A9C00002D30021C943816404998E421BDAA17D20
:10A9D00000E043E0032916D00221A175009B002A64
:10A9E00083640ED039200257D74818232030C3562D
:10A9F000921B9A4200DC0121D54A28001268904738
:10AA000016E0012111E003998E4211DDA17D042998
:10AA10000ED0816C491C0BD10221A1750099002A2E
:10AA2000816401D00021E7E7002128000AF36FFBD1
:10AA300039200655C74B31001B68A27D3800984766
:10AA4000280006F3F2FC002808D0C049A800085CE2
:10AA5000002803D031002800FFF7FEFE6D1C2D04F6
:10AA60002D0C082D00D22FE70198002803D0FCF20E
:10AA7000E7FD022803D1FCF2E3FD012807D1B64827
:10AA8000006880470022B54913002DF3D1FC05B0C2
:10AA9000F0BD70B50C21B248B24C81720B214171EE
:10AAA0000A2141740921C171002565712D20A5710C
:10AAB000607020202070A561A57031F383FEAA4844
:10AAC00040213FF318EAA94820213FF314EAA8489F
:10AAD0000068018CC908C9000184018C022211435D
:10AAE0000184C18E10229143C1869F48602140306D
:10AAF00065823FF300EA9F49192088726573E5710A
:10AB000070BD70B50D001400012A07D9401B001953
:10AB1000401E21003FF350EB4443601970BDF8B56F
:10AB20000C00070015001E0025F3BAFA943524170F
:10AB300001000000B4A400A0000200003730D2E4FD
:10AB40006421794308184030818821804189298017
:10AB5000C0893080B7E6F3B583B00398874F0468A7
:10AB6000258A002C65D0200030F3CDFBE169401828
:10AB70000499081A5DD4002620002FF325F8ED0073
:10AB8000785D00283BD0ED196868E16901AA471A91
:10AB9000208A02A96B46FFF7CCFF002F12DC6F68FA
:10ABA0006B461A8904983900FFF7B5FF68600C22DC
:10ABB00001206282A0850020E08204983900FFF71E
:10ABC000AAFF0FE00C2F09DA68686B46E06118896C
:10ABD00060829888A0851888E08204E004992000AB
:10ABE0002FF3F7F8E06120002EF3EEFF0020E0766F
:10ABF0004420025DE16920002FF375F808E0634B03
:10AC0000049A1B68039821009847E069E919486095
:10AC1000A07E002804D020002030867B0121817393
:10AC200020002FF33BFAA07E002801D02034A67329
:10AC300037E7E07E0128FBD1E800385C0128F7D037
:10AC40000020E0762DE7FFB583B048230F0003987E
:10AC50004F4958430C9E40180D9D02902EF3B4FFAF
:10AC60000398C40045480C2E14D901210155380021
:10AC7000484F06D006982FF36EF840496118486097
:10AC800002E00598002809D10C26012500200E902D
:10AC9000B86905E00021002F015504D10298C06970
:10ACA0002FF356F806900E9A3B4C009224682B0026
:10ACB000069903983200A047A8E510B514001A00C1
:10ACC000002C05D1354B1C5C042C01D0052C03D184
:10ACD000334B1B68984710BD33F334FA10BDF7B5FA
:10ACE00084B004000F0025F3E5F9050000202EF3E1
:10ACF000CEFE48216143264A2A4B89181C22624312
:10AD0000D2186423634312795B193425ED5C002D5E
:10AD100012D0012D48D0022D54D0042D06D19D888B
:10AD20005A78010020002B00FFF7C7FF069A390070
:10AD3000200024F35DFB69E549680029D9703E1CB9
:10AD400001000000B0A600A000020000C3D86C59AA
:10AD5000F6D0002AF4D19D885A78010020002B00FB
:10AD6000FFF7B5FF5CE5000098EA0004D8F50004A1
:10AD7000B4C70004FCB5000430F400043CFD00043A
:10AD8000E0F60004470C00002CEB0004BC5C00B0B3
:10AD9000FCED00B038D3000464EA000430D20004B3
:10ADA00060F8000470CA0004B0D10004ACF70004DD
:10ADB00024EB00048CF70004B4B400041800403005
:10ADC000C289418980886D4607C539009B6B069A08
:10ADD0002000FFF742FF23E50020E500FF4E7055FD
:10ADE000986B2EF3C2FFA9194860A9E731B584B06A
:10ADF0000499FB4A08680024801810D045282BD1FC
:10AE00008879012828D1083101A81BF35EFCF54898
:10AE10000C22006801A910301BF3B2FA1CE00AF3FF
:10AE200012FC0499F04D898801221300AD7B8B4000
:10AE30002B4211D088234B4318186030C277EB4A5D
:10AE40000023126800920A00808BE9492DF3F8FA7A
:10AE5000012404A8FCF2A7F9200005B030BD10B50C
:10AE600001680022FF397E3900290BD0DC4BD53335
:10AE7000C91812D18188DF4B8900595C01290CD196
:10AE800082720AE08179002907D081881C23594306
:10AE9000D94BC9188B78D9495A542CF33AFF10BDB5
:10AEA000D74910B509680A8880239A43D54B1B7887
:10AEB000DB09DB011A430A802DF301FC10BD70B5DC
:10AEC000D24AD14C527A2578002A01D00122227030
:10AED00031F3D6FA257070BDFFB581B04823002547
:10AEE0000198CB4F5843C419A17E0298814219D1D1
:10AEF0002E20005D002815D10398012801D10126DC
:10AF000001E00026F643019822F3C5FBC1498842BF
:10AF100008D048235843C419206A80192062E06988
:10AF20008019E06140342079042802D104250220F0
:10AF3000207101A80FC831F374FD042D01D1042044
:10AF40002071B8E5C100B44A091849017FA318551A
:10AF500001000000ACA800A00002000004C16E04C3
:10AF600089188031C97C002914D01C235843A74973
:10AF7000142340188078AE49584309680A5A002AB9
:10AF800008D140184188002904D18088002801D1C7
:10AF90000120704700207047F8B50D001E0407001F
:10AFA000360C0AF35AFBAC88022F4AD10127032E34
:10AFB0002AD1002018F310FD0600287A4006400E22
:10AFC00011283ED18F4821005B302DF35EFA28789E
:10AFD000C107C90F200028F377FE2000FFF7BCFF50
:10AFE00000280FD0382060438019006A002809D05B
:10AFF0001C20604385491423401880788C495843AD
:10B0000009680F52012072E4132E12D18821614386
:10B010000818007D002814D186480078012810D92E
:10B02000E8791322C107C90F2000212320F338F942
:10B03000E8E78148864204D17048A740817B0F43EE
:10B040008773002053E4F8B504000D007B48407975
:10B05000012810D17A4B00201A68C100565A3607D1
:10B06000360F0A2E04D1565A36093601761C56522E
:10B07000401C0E28F0D30820FCF29CF87149009087
:10B0800001602178017161784171A1788171C57188
:10B090006D4801686846FCF29CF828E456481CB5E7
:10B0A0006946006810301BF3A0FB684801680D205A
:10B0B000085667490968884701006846FFF7C3FFDB
:10B0C0001CBD4D481CB5694600681C301BF38DFB48
:10B0D0005E4801680D2008565D49096888470100EF
:10B0E0006846FFF7B0FF1CBD10B5019859494008EC
:10B0F000884202D11BF317F910BD1020FEF770FF34
:10B1000010BD10B52FF3C8F9454820384188912962
:10B1100001D99121418010BD70B50200548A080008
:10B12000012C08D9D5692100401B0019401E3EF3AF
:10B130008EEF4443281970BDF7B584B004001700A2
:10B14000066B456B008A19F318FA384300D00120CA
:10B150000690069A059920002FF302FFD3CCC1B7C1
:10B1600001000000A8AA00A000020000F029D0B948
:10B170004020005D032827D1200020300390C77FA6
:10B180000297608A0190474305983900401BC01917
:10B190003EF366EF7843471967630698002811D09D
:10B1A0000398857F01980095454305982900801BE9
:10B1B00040193EF356EF684380192063009A0299C4
:10B1C000914200D8380095E505992000FFF7AEFFC1
:10B1D00090E5F8B506002EF357FB0A2171430500F0
:10B1E0000C18603C207C012856D1607D002853D08B
:10B1F0003000FDF2F2FC07000100300016F0E2EC36
:10B20000002833E0FCED00B039F4FFFF88EA0004C9
:10B21000BC5C00B0F8A93400BD0B0000FCB5000414
:10B22000B4B40004CAC7000470EA0004E7E90004EB
:10B23000D1EA000450D2000470CA0004FFFF0000ED
:10B24000E0BD000460EA0004D0EA00047F100000C2
:10B250006CD2000428EA0004CF0C000000AA3400DD
:10B260008CEA0004D8F50004AF81190010D0390031
:10B2700030002EF338FB0A20784300214019603853
:10B2800021740174617541753800FDF286FC06E099
:10B29000300016F09CEC02E03000FDF2B6FC00201D
:10B2A00076E438B50C001100049A00920A002100DF
:10B2B0002DF30EFBFD486101006809188888FC4ADF
:10B2C0001278002A04D05622562800D90200100015
:10B2D0008880488138BDF74800884007C00F704714
:10B2E000F44930B50400098800201422114001D02F
:10B2F000012030BDF04D0A224A435219137A022B25
:10B3000002D15288A242F3D3491C0904090C022934
:10B31000F1D330BD0C235843E849401800897047E9
:10B3200000B5008AFFF7F6FF904201D9012000BD69
:10B33000002000BDFFB583B00C000D002035C869AA
:10B340000290287D0190C87E00263700002828D171
:10B35000218ADB4A505410003B388179002920D0E3
:10B36000218A80783FF358FB00281AD0B8F1E5977E
:10B3700001000000A4AC00A000020000E9D10EC949
:10B38000D44A01203B3A518A4003A37E81430120E5
:10B39000002B00D000204003014348040121400C51
:10B3A000C903401850825079297D814200D308009A
:10B3B000012637005071069B059A0398210030F34F
:10B3C0009EFB0090208AC3490A5C521C0A54208AC2
:10B3D00019F3DBF8002804D0A08980088000401C05
:10B3E000A0810298002E00D1E069002FE06105D015
:10B3F00001982875002801D0401E2875B54E218A75
:10B400003B3EB0783FF312FB00283AD07079002819
:10B4100001D0401E7071208AAF49095C052905D111
:10B42000707900282DD00320E0762AE0B179012937
:10B4300027D1A37E01221100002B00D00921A54BAA
:10B440001B5C8B420DD91C235843A4490A23401886
:10B450008078A34958430968085A800701D5A28516
:10B460000FE0059906222000FFF764FF002808D0AE
:10B47000287D401C2875A08D401CA0857079401C3B
:10B480007071009840E4FEB50D001600847E099AA4
:10B490000899002C09D1078A8F4CE45D042C01D057
:10B4A000052C02D103200870FEBD019200913200EC
:10B4B000290030F343FFFEBD10B5040024F322FE43
:10B4C00064216143425C002A04D008182030007DCA
:10B4D000012800D0002010BDF0B587B000217D48C4
:10B4E000804C3B38817001206E4648214143420028
:10B4F0001218091920314D7C6B469D54D2180D7CD1
:10B50000401C00045570897C000C07289170ECD910
:10B510002FF3D3F8744F01253E00A036482169432C
:10B5200070480C18280024F3F5FD00283AD06A482A
:10B53000405D042801D0052853D124F347FD00289D
:10B5400022D164493B39C879C0071DD00120A840E9
:10B5500006908A7810438870F07829003FF366FAE5
:10B56000002805D1F07806990843F070B869E061C9
:10B57000680040196A46115C2034801820983F31D9
:10B5800001000000A0AE00A0000200001D39B07450
:10B590006174417821748078A0742CE0F0782900DF
:10B5A0003FF34EFA002826D00120F178A8408143CD
:10B5B000F170B869E0611EE0280024F3C7FD00289F
:10B5C00004D12800FFF782FF002814D01C20684314
:10B5D00047494018007900280DD14420005D042817
:10B5E00006D0208A3F49C0004039085C012802D1BA
:10B5F0000120207660766D1C2D042D0C072D97D927
:10B60000FEF796FD0FE43849F1B500253B390126D8
:10B610004D71354F31003B3FB8783FF311FA0028A8
:10B620003CD0482070433449441820002EF3FEFAE1
:10B6300038008079012831D030483100A030407A7C
:10B640003FF3FEF9218A294A515C052917D0333787
:10B65000002800D1083F19F345FE28217143401806
:10B66000407821002031385C0A000875A17E00294D
:10B670000BD00A210A2800D90100117505E03C21F0
:10B68000002800D12D21342001553420015D1648B9
:10B690003B384279891841714078A085761C360480
:10B6A000360C072EB5D9104F3B3FB879012806D08C
:10B6B00078793900401E0006000E787120D1387864
:10B6C000801C06060098360E8019B8610220B871F9
:10B6D00019E0000074EA0004CEE800047AEC0004EB
:10B6E00048D600043CEE00B0F75C00B024EB000448
:10B6F000B4B4000490EA000470CA0004B0D100049D
:10B700000026012088710124B87821003FF398F9C0
:10B7100000281BD048216143FF4808180021C1764A
:10B72000BA79012A07D1002D00D10500FB4A121970
:10B73000203AD17703E00121342211548185A842B7
:10B7400004D00099052289192EF3FFFA641C240401
:10B75000240C072CD8D9002D04D0009905222800EC
:10B760002EF3F3FA6DE4F0B518231C26EC4A0025FD
:10B7700052785A43E84BD2180B23DB01D218146AD3
:10B78000028AE84B5643F3189E789C46A8AF58535C
:10B79000010000009CB000A000020000632217C45A
:10B7A0000C237343E54E36689B199B88E44E7688DC
:10B7B000B34204D9836BCB1AB34200D90125002CC4
:10B7C0000BD0E38E934204D1C2698A1AB24200DBE5
:10B7D0000125628A012A00D1002562461279002AD9
:10B7E0000BD09122002C03D0638A032B00D828228F
:10B7F000FFF7B4FD002800D001252800F0BDF7B503
:10B8000082B004000020019019F376FD218A2823DC
:10B8100059434018CB4940780978884208D30399A6
:10B8200019222000FFF79AFD002801D0012000E036
:10B8300000200090BE48218A243880783FF30AF91E
:10B84000002804D103992000FFF797FF0190BC4D19
:10B85000218A2035A8783FF3FDF80700218AE8788F
:10B860003FF3F8F8250006004035002809D0208A6B
:10B87000B549085C012811D0032802D1287909288C
:10B880000CD0AB48218A243880783FF3E3F80128B4
:10B8900004D0002F04D02879092801D1012000E02C
:10B8A000002001990027002923D0002E04D0218AEE
:10B8B000A54A515C01291CD020002EF3C1F9E7767E
:10B8C000A07E00280FD1A148417800290BD18078B3
:10B8D000002808D1208A18F378FE002803D1618A55
:10B8E00003980818039035202979015503990622F9
:10B8F00052E0E17E019A009B0A4303431A433AD087
:10B90000A28DE069039B82189A1A50D420002EF36E
:10B9100097F9002E31D08648218A243880783FF369
:10B9200099F8012803D10398FFF777FE06E0884BCA
:10B93000E7761B68049A0399200098472879052820
:10B9400019D1208A8049085C032814D1794818232A
:10B950004079764958437F4E40180B21C901401861
:10B96000056A06E0A54203D032682900200090470E
:10B970002D68002DF6D105B0F0BD7748016800298B
:10B980000ED0208A884700280AD0E7760399200045
:10B990002EF35BFA049A010020002EF3BC2A35C571
:10B9A0000100000098B200A00002000097CAA97927
:10B9B000E0F9EAE76E4B049A1B6803992000984768
:10B9C000E3E70029E1D0A17E002918D1002E16D08E
:10B9D000218A624A515C012911D1060020002EF310
:10B9E00039F9E7762879052802D1E169049ADDE77B
:10B9F000049A039920002EF3BCF9E661C5E7514D86
:10BA0000243DA8790128C0D1218AA8783FF32CF8D9
:10BA10000128BAD120002EF31DF96879002803D13E
:10BA20000398FFF704FEB0E7E776E1690522BDE77A
:10BA3000F3B581B006000768027A02993800FFF773
:10BA4000E8FE0124482161433D480D184420405D33
:10BA5000317A884214D1AF4212D0298A3F48405CE3
:10BA600004280DD005280BD03A482030C0783EF38A
:10BA7000FBFF002804D0327A0299280030F32CFB17
:10BA8000641C2404240C082CDCD3FEBD70B50025F6
:10BA9000384C25602EF3F4F92A49243948790028D6
:10BAA00003D1488A4004400C48822A481723803832
:10BAB000C069498A8288DB029A4319400A4382801E
:10BAC0002D482060012070BD70B504002348055D3D
:10BAD000200032F364FA29002000FEF7F5F970BD6A
:10BAE00070B50400254D00202860200032F370FB63
:10BAF000234828601948015D2000FEF7E5F9012080
:10BB000070BD012181400F4824388078014201D066
:10BB1000012070470020704770B50D0019490600DC
:10BB200040000C5A2900300018F338FE002E35D0A2
:10BB3000154968062BD50C2060430A5C521C25E091
:10BB400070CA0004E05C00B02CEB0004B4B4000444
:10BB500098EA000430D20004A2E5000424EB0004BB
:10BB600078D5000418F7000478F7000490E6000484
:10BB70000CF800044CF8000475B3000080F70004D2
:10BB8000C9B30000E8B500043CEE00B00A54280632
:10BB900004D50C2060430A5C521C0A5470BDF8B5F1
:10BBA0002EF339F9FD4905000A6A904296B714FD53
:10BBB0000100000094B400A0000200008E3277095A
:10BBC0003ED0FC4F01240D62200017F341FF0078A6
:10BBD000002830D01C206043F749F84A401880788C
:10BBE000126801018918F64AC00012688018C088DE
:10BBF000002801D1012000E00020C0000818C688FC
:10BC0000200018F3F6FC00280CD00C216143C81961
:10BC10004278795C8A4205D14188B14202D14168BB
:10BC2000691A07E00C206043395CC0194170456017
:10BC3000002146800181641C2404240C072CC3D9F4
:10BC4000AEE5F7B588B00400C669008ADD4A049005
:10BC5000126809999047DC4A039012680999049880
:10BC600090470290049844235843D84940180190C3
:10BC7000D748049980783EF301FF0790049818F3A1
:10BC8000B8FCD44D002803D128790299884201D903
:10BC9000012000E000202A79039B01219A4200D86C
:10BCA00000210843059101D0012700E000270498F6
:10BCB00018F39FFC002809D0019940318878097851
:10BCC000884200D308000299884208D305980028CA
:10BCD00007D00198403041780398814201D2012079
:10BCE00000E000200690A07E00286ED1E27E002AAF
:10BCF00003D1E18A0998461AE661079800282BD0FB
:10BD0000617E237E0320C91849084B1C032B01D3F5
:10BD10000800401C002F009007D0012A05D1AE4B2F
:10BD2000029A1B680399200098470020002FE076B4
:10BD300021D00199403108784978884200D3080021
:10BD4000079AE979002A00D1A979009A51438142E2
:10BD500006D9099E00251AE0607E217E4018D8E7AA
:10BD60003421095D002901D00091F2E7618A814206
:10BD70000CD808000AE00820FEF76EF98107608AF7
:10BD8000890F411A0D042D0CA84200D20500069916
:10BD900001200F4300D00098E08207990520092771
:10BDA000002900D00700092F27D18C48218A00786C
:10BDB0003EF364FE002806D18948218AE0DC80F544
:10BDC0000100000090B600A0000200007ADAC9B4B9
:10BDD00000783EF35DFE002819D0052717E0002FFC
:10BDE00005D0824B029A1B680399200098470020D7
:10BDF0000500E0760798099E002805D006980028DF
:10BE000002D00A20A082E8E714200927A082711935
:10BE10003A0020002DF3C1FF0BB0F0BD694910B509
:10BE2000087331F32DFA10BD10B52EF30BFA6D48DF
:10BE3000644980388079097B084301D1FFF7C3FE4C
:10BE400010BD70B51C00CB7E002B18D18B7E002B53
:10BE500015D0694B5D7818236B43684D5B190B2532
:10BE6000ED015B191B6A0125CA61002BCD7604D058
:10BE70005B8A032B01D8072300E015238B85230061
:10BE80002FF318FF70BD70B50D000468E07E002828
:10BE900016D029002000FFF78EFC002804D0A18DC9
:10BEA000E0694018281A0BD420002DF3E7FE00208B
:10BEB000E076608A41193520025D20002DF36DFF88
:10BEC00070BD49494978084070470300454800B5AE
:10BED000407AFFF7F6FF002806D0998A0720072945
:10BEE00000D20800988200BD45480088FAE735482E
:10BEF000407B002800D001207047F7B504001600F1
:10BF0000807E002500285AD13E480078012856D965
:10BF10004020005D002852D1208A18F374FB0028CD
:10BF200015D1314F208A01227978824011420ED1F9
:10BF3000294A0199126890473979884207D3618A62
:10BF400001E005042D0C4819B042FAD337E0608AAD
:10BF50004100B14233D82C492C4A09781278114358
:10BF60002CD1207E617E00264018E18A40080029FD
:10BF700001D1A18D00E0A18A401E081803041B0C0A
:10BF8000FFF7B5FF002802D05B1C1B041B0C608A66
:10BF9000984200D203000B48407BFFF792FF002835
:10BFA00001D00A2606E00F488078FFF78AFF0028B4
:10BFB00000D00826608A9919814200D9050028001E
:10BFC000FEBD0000BC5C00B03CEE00B0C2779098B3
:10BFD000010000008CB800A000020000BDC3CBE946
:10BFE000B4B4000450EA000440EA00041CF7000462
:10BFF00020F7000458D3000450D2000478D5000480
:10C0000010F80004DAEA0004DBEA00042CEB000478
:10C0100070CA000472EC0004D0EA0004D8EA0004FC
:10C02000D7EA0004FFB583B00C0005001F00888923
:10C0300080088000FF49C97A0843A08120002EF3C0
:10C04000D8FCA28D082100913B0021002800FA4D68
:10C0500001922D68059AA8470290E07E00286BD1D6
:10C06000208AE1698200F5488150208A18F3D5FAC8
:10C07000F34A012600280AD01178208A0B00C34019
:10C08000DB0704D1330083400B43137005E0218AA2
:10C09000300088401178814311702000FFF71FFFA6
:10C0A0002268059920002EF3B7FEE6481823407950
:10C0B000E549584340180B21C9014018026A059907
:10C0C00020002EF3A9FEA18A3000012900D9080022
:10C0D000DE49A0820978012907D9618A062904D896
:10C0E000A18D884200D30800A08225004035287920
:10C0F000042804D123F3A6FF002800D0A682687884
:10C10000012809D1E08A002804D0A08AA18D8842A4
:10C1100000D9AE7000206870A878012805D1207E73
:10C12000617E40184008B84202D32878002802D027
:10C130000320E07600E0E676029807B0F0BDF7B5A0
:10C1400082B00D00272204992800FFF7E0FE049931
:10C15000BF4B41181B68002228009847E861012660
:10C1600028004030019048207043B7494418270008
:10C1700040373879042801D0022864D1A54262D022
:10C180000199097981425ED1B24A210012682800E2
:10C190009047002857D0298A228AA84B8E46944679
:10C1A0008900920059589A580120891A002900DC08
:10C1B0000020A97E00231A00002903D0A98F01299D
:10C1C00000D10122A37E0021002B03D0A38F012BDD
:10C1D00000D10121002907D0994B61461B3566C06B
:10C1E0000100000088BA00A000020000492B75542D
:10C1F0001B78CB40D90701D000280BD0002A01D1F1
:10C20000002807D1934A71461278CA40D1070AD153
:10C21000002808D0E969934B491C1B6800222800BC
:10C220009847E8611EE020002DF33CFD0020E076F9
:10C23000A18FA1858D498B4B0988A182B8700120FF
:10C240007870E1691B68491C002220009847E06172
:10C2500001003A7920002DF3B4FD761C3604360C2B
:10C26000082E8AD30020E876A98F804AA9851288F3
:10C27000AA82019A01249070019844707C486A8ACD
:10C2800040889200904200D31000AA7E0004000C67
:10C29000002A09D1298A8A006D498958049A511ABD
:10C2A00081421DD800241BE02A8A1C235A43714B6B
:10C2B000D21892780C235A436F4B1B68D21892887D
:10C2C000824201D9012400E00024012908D1FF2283
:10C2D000049991322800FFF773F8002800D0012458
:10C2E0000422002C00D10222E96928002DF369FD07
:10C2F00005B0F0BDF8B515001E0048234343574C68
:10C30000069A1C19009233002A0031F3B9FE2089E5
:10C31000802108432081B1E4FEB50D001F004823B1
:10C3200043434E4C1600099A08991C19019200913A
:10C330003B003200290031F319FF20898021084396
:10C34000208151E6FEB50D001F0048234343434CB6
:10C350001600099A08991C19019200913B003200BD
:10C36000290032F38FF920898021084320813BE6A0
:10C37000F8B515001E0048234343384C069A1C1993
:10C38000009233002A0032F3AFF92089802108435C
:10C39000208173E4FFB500209FB000210A000C90BB
:10C3A0000B900A90099007A806C023F3F1FE0490B1
:10C3B00020981C230068109022982E4980881C9099
:10C3C0002298FF22408945082298807912901C9873
:10C3D0005843401800791390082105A83DF35EEDFD
:10C3E00000210A000B000C0015A81EC0C374487B76
:10C3F0000100000084BC00A00002000050D3AB2468
:10C40000012064214143049A89180A7B012A13D12F
:10C410004A7B012A10D11C9A904202D12299098AA2
:10C4200007E03422525C002A06D0042A04D04031AE
:10C43000C989420015AB9952401C0006000E08281D
:10C44000DFD31348007D01284AD1114E1C23F08A06
:10C450000D49584340180079317E1BE0C0BD0004EF
:10C46000F8F7000438D30004C6EA00042CEB0004FB
:10C4700070CA0004D0EA000458F800045CF8000414
:10C4800072EC000430D20004B4B4000498EA000452
:10C49000A0BD00044C08717E490800280B9104D10E
:10C4A0002DF36DFB11900A9003E00AAA11A92DF358
:10C4B00093FBB07E21F3A4FA012802D10B990A98CC
:10C4C00004E00A980121490648400B993DF322EE09
:10C4D000601AA14201DD0B994018119908180990C2
:10C4E00010980F900D9001201B902806000E1E90B2
:10C4F0000F9A0E92501B0F9007A81092FF4B1E9997
:10C500001B689847002401260E991098884205D090
:10C510000F9B421AC31A9A4200DA0F91641C24043A
:10C52000240C0B2C0E900FD1F5488078002808D0F1
:10C53000F44A0021126807A89047002801D0012082
:10C5400000E000201B9013E1012C11D1EE4B187D6F
:10C5500001280DD19A8B09990B986F4607C70EA930
:10C56000EA4FD88A3F68139A2B00B84701282BD08E
:10C57000E74920000968884700283DD01398002823
:10C580000AD01C206043E34940180079139988427F
:10C5900002D11298F8282FD1DF4920000968884776
:10C5A00064216143049A6F468B18010098699A8B45
:10C5B0000006000E07C72B00D44F139A3F682000D7
:10C5C0000EA9B847012817D1CD486B468678187F49
:10C5D000401C1877D1480168002908D101E00120EA
:10C5E00000E000206B46997F40189877BBE01C98CC
:10C5F00088470028F5D0F2E7229880885CCD224D4C
:10C600000100000080BE00A000020000A43B1599BC
:10C61000A042F5D064206043049947183420C05DDF
:10C620000028EDD00428EBD01C98642358430499CB
:10C630004018BC491D900968008C88470028139851
:10C6400005D0002805D01298F828D9D11DE000287F
:10C650001BD11C206043B44940180079002814D134
:10C660001D981D99007B497B7A7B401822994008D0
:10C670008989401E4018397B000489184A084A21DC
:10C68000C95B000C521E511817E01D981D99007BC4
:10C69000497B7A7B4018397B40088918139A4908EE
:10C6A000002A02D0801C0004000C1C2262439E4B16
:10C6B000D2181279002A02D0891C0904090C1C9A8C
:10C6C00015AB52009A5A10180004000C1A90600022
:10C6D000185A401800049549000C19900968200068
:10C6E00088474037BA88AA4221D3219A1099891ADB
:10C6F00000E049198142FCDB00E0491B8142FCDC7F
:10C700001A9A8A18531E834203DB8249101A8E78C4
:10C710002AE0199A49198218521E8A422DDB091AF9
:10C720007C4A1A98967808181EE0801A02E0109B3E
:10C730002199591A8142F8DB00E010188142FCDC93
:10C740001A9BCB185F1E874203DB7249181A8E783A
:10C750000AE0801A199A8218521E8A420DDB6D4A2D
:10C76000081A1A99967840180E996B46081A800193
:10C7700080090E90187F401C1877012E00D1CDE65D
:10C780000B2C3BD11398002838D16B46987F00289A
:10C7900034D11C992298490015AA515A80896423E2
:10C7A00041181C98049A58436B468018027B407BC2
:10C7B000101840081A8E401E5E4B081800041E68B0
:10C7C000000C29000EABB047002817D001216B46A2
:10C7D0001B91197F491C19779A7F0121022800D0EB
:10C7E000002150186B4698770E991098884205D012
:10C7F0000F9B421AC01A824200DA0F914E4A05A9D5
:10C80000126807A890471B98012811D106EB5150D8
:10C81000010000007CC000A000020000416C489EA6
:10C820000D98401B06D40F99884200DA74E6002068
:10C830001B900AE00D9A0F999142F7DD01218906BC
:10C840004018F0E71B98002817D10B2C18D00023B4
:10C85000012015AE4100725A002A02D0521E012357
:10C860007252401C0006000E0828F3D3002B04D09F
:10C8700001201B900D980F904EE61B980128D5D0F3
:10C8800029488078002813D0284D00212A6807A85D
:10C890009047002815D02A6814A905A890470028B9
:10C8A0000FD010AB187C00280BD10698109007E031
:10C8B000274B02201B6810AA0CA99847012800D119
:10C8C0000B241F98048020981099016023B0F0BDBC
:10C8D00070B50400080016002DF3C9FA05003000F9
:10C8E0002DF3C5FA1B4E2D1A012248205043801902
:10C8F0004168002936D02E21095C002932D0817E82
:10C90000A1422FD1016A691A090609162AD00562C7
:10C91000C3695B18C36144231B5C022B01D0042B49
:10C9200020D119E034FC000420E9000438FC0004A4
:10C93000A0BD000458FC000468FC0004B4B400046A
:10C9400048F7000490E600049CF3000430FC000467
:10C95000ACF3000470CA0004036B5B180363436B01
:10C9600059184163521C1206120E0B2ABDD370BD1A
:10C9700010B530F35CFBFF490B68198800290BD117
:10C98000CA00D21894886404640C9480491C090677
:10C99000090E0E29F4D310BDF749497DC900C91805
:10C9A0008A885204520C8A8010BDF8B50C00C97EEA
:10C9B00000291CD1250040352979072917D1EF4ED0
:10C9C000B178002913D0B169891A10D40127BF02A8
:10C9D000B9420CDA20002DF383F9B1692A79C91C18
:10C9E00020002DF30CFA0120E0760020B1E42100B4
:10C9F0002EF3DCFFADE4F8B58446E14DDE4CCF7E8E
:10CA00002E782034002F06D1607A002801D008202B
:10CA100000E010208885DB4F387801287C6E81DFAC
:10CA20000100000078C200A000020000B584F623D7
:10CA300004D1A078002801D00120287060462EF390
:10CA400095FE3978012903D1A178002900D02E70F4
:10CA500089E470B50400CE4D10000026233500296E
:10CA600009D0FCF7CAFE002801D1012607E0218A7F
:10CA70000020485503E0208A415D491C41552000B3
:10CA8000FCF7B4FEC249002804D0207E627EC9783B
:10CA9000801811E0208A1C235843C04A0C238018B8
:10CAA0008078BF4A5843126880188088142807D2BB
:10CAB000207E627E097980184843C005000E00E0A0
:10CAC0002D20218A495D814200D90126300070BDA8
:10CAD000F8B50600B34800250068408FAC4C00064E
:10CAE000070F318AA0783EF30FF800280CD0308A67
:10CAF000AD49085C052807D1A4483A006038C17DDB
:10CB00003000FFF7A6FF05000021002D00D161795C
:10CB10002800617127E470B505009C4C4823603CF7
:10CB2000A08AA2495843461829003000FFF7D0FFD9
:10CB3000002803D00020E0750120B085280030F3E4
:10CB400061FE70BD10B530F361F9904860388079AE
:10CB5000022812D18E4A907800280ED08A480068A8
:10CB600083881721548AC9028B430C402343838056
:10CB70005079002801D0401E507110BDF8B50E004C
:10CB80000468E17E00293ED0A78DE56931002EF3CF
:10CB9000A3FE81480078012803D085480078012849
:10CBA00031D1E819301A2ED420002DF3A3F8814892
:10CBB0001823407A7D49584340180B21C901401879
:10CBC000056A7948298A405C012806D16F482030DF
:10CBD000C0783DF399FF00280ED1002D0CD0287E9F
:10CBE000697E4018A97E4008002901D1361803E06B
:10CBF000430018188619761C4420A785025D310071
:10CC000020002DF306F9FBE670B55F4D2A68148805
:10CC1000C27E032A0BD1827E002A08D1664A12788E
:10CC2000002A04D162040123520CDB036965E294FB
:10CC30000100000074C400A000020000AC7C285376
:10CC4000D41830F31FFD2868048070BDF8B50400C7
:10CC50001C238088564958434018457900202CF3FE
:10CC60002AFE28216943405C01281FD1E088A6687C
:10CC7000574930188778096868014018C18A008BC5
:10CC8000081A544940183DF36EEA2D200001401A5D
:10CC90000004000CB84209D24F48C069002805D0F2
:10CCA0004E4A3100126828009047B3E620002CF36A
:10CCB000D7FBAFE631B582B0029800240168FF3996
:10CCC000F7391CD0464A89181FD18588280016F3E9
:10CCD0000FFF0078C00718D042492800096888472C
:10CCE000002812D00820FAF2F1FA3F4901900160C1
:10CCF00085803E48016801A8FAF2F7FA05E0FFF7DF
:10CD0000A5FF012402A8FAF2E4FA20003EBD70B5A6
:10CD100005000C0004D13448290009302BF341FCF4
:10CD20002100280028F332F91E4A0121107AA94077
:10CD30008843107270BD3EB504000D0008F319FD64
:10CD4000882161436B460818017D29A023C3002276
:10CD5000284B110020001EF357FC3EBD38B50400DF
:10CD60001020FAF2B3FAFF21433100900160011D57
:10CD7000200023F38AFE19F362FB1F493DF3C6EA44
:10CD80000A00E1001D480919490108180400FF3094
:10CD9000401C426120000099653031E028EA00041F
:10CDA00030D20004BC5C00B0D5EA0004D7EA00042D
:10CDB000B4B4000498EA000484EA000424EB0004FC
:10CDC00070CA0004D8EA00042CEB0004C5EA000491
:10CDD0006CEA0004D202000008D7000408F700043F
:10CDE00064F5FFFF14F60004BB0C000000AA340039
:10CDF000696200007F1F000040420F00E0BD000498
:10CE0000CA6004220C313DF384E8009920005530BB
:10CE100004220C313DF37CE8FF4801686846FAF2D1
:10CE200064FA38BD10B52FF366FFFC48007801287E
:10CE300012D1FB480068018809090901F3BF6F0698
:10CE40000100000070C600A000020000589496EE99
:10CE5000491C0180F84B9978002907D08188172256
:10CE60005B8AD2029143134019438180F3493220F7
:10CE7000087210BDF14910B58979022902D1EF4934
:10CE80002039886130F3A3FB10BDF8B506000F0010
:10CE900008F379FC05003900300005F375F904004A
:10CEA00001281AD13068572817D1E54A390012688D
:10CEB00030009047012810D1388888235843401902
:10CEC000C08D002800D10B200EF349F9002804D0B2
:10CED000DC4930000968884700242000A4E5F1B54A
:10CEE00084B00326049805680AF30EFC070008F3D3
:10CEF0004AFCE979020001204B082B2B00D10020CD
:10CF00000190C807C00F0290A88888230390584357
:10CF10008418E08D002802D008380604360C5D2005
:10CF2000C05D012805D01E207043C019C0780128BB
:10CF30004FD1217D029881424BD0A87D002803D09B
:10CF4000C14803992BF337FB01982B22002801D00D
:10CF5000BD4A6732A1780D2001290DD10199002920
:10CF600001D1297A00E0697A1E237343DB199B798A
:10CF70008B4208D00A2006E0217D00290BD1617880
:10CF8000012900D123200306029903981B161EF3E2
:10CF90001DFA05B0F0BD0121742001550498006808
:10CFA000206704990020086060780128F1D11E21D3
:10CFB00071433720C9198978012904D10199362094
:10CFC000002900D03920A14B0399002211F3E8FF7A
:10CFD000DFE704980DF368FDDBE710B504F31CFAF6
:10CFE00095490020887310BD10B5040018F3F4F9BA
:10CFF000200027F3B1FB10BD70B50B1D4A88D20489
:10D00000920D9A189278D20725D0914B1222424362
:10D010001C68A35A5B071ED58E4D142343432D680D
:10D020005B19DD88002D16D11D89002D13D15D8976
:10D03000002D10D1A55AAE077F4D07D4A35A022662
:10D040003343A352AA8A521CAA8204E097EEBD364B
:10D05000010000006CC800A0000200009F8D94B386
:10D060000122DA80EA8A521CEA8217F38EFE70BD32
:10D0700038B500247D4A0168891808D180880828BD
:10D0800005D200221100130000921BF339FC20008E
:10D0900038BDF8B504000D001600002016F33CFD65
:10D0A000070032002900200027F32EFE032D15D1A2
:10D0B0002000FDF7F1FF002810D038206043C01990
:10D0C000006A00280AD01C216143694A012089189E
:10D0D0008978654A1423594312685052AEE4F7B573
:10D0E00098B00500002016F317FD1C216943049039
:10D0F0005F48081817900679E8005E49401940011A
:10D10000441827008037F87C002806D11A9A19990C
:10D11000280024F3F2FE1BB0F0BD002E06D1002043
:10D1200014900EA819F3FAFB0CA905E00120149045
:10D130000CA819F3F3FB0EA9280023F3BAFC002076
:10D140006B461875B87B002800D001206B46220082
:10D1500058757D32484F2300169200923F682D3358
:10D1600020000CAA0EA9B847200060301590408B13
:10D170001021081A07063F0E04D005A83900801CAC
:10D180003CF3A0EF15981A22825E780005A940189A
:10D190001699801C3CF3D0EE210009A89831082292
:10D1A000801C3CF3CAEE35486B46007818752800A1
:10D1B00023F3F5FC05AA0092149A0021280001230C
:10D1C0001BF39EFB002E0DD11998102210A901AB64
:10D1D00007C32BA2009201220021280011231EF375
:10D1E00027FA98E72800FDF757FF00280ED03821CE
:10D1F000694304980818006A002807D017991A4A4A
:10D200008978012014235943126850521998112229
:10D210000106091628001EF3D8F87CE77CB50C003F
:10D220001500A67E079A0699002E2DD14426365D5C
:10D23000092E03D0062E01D0052E25D1012921E08B
:10D24000F4E70004CBEA000428EA0004BC5C00B068
:10D25000D0D10004A0F90004CCF90004501050F023
:10D260000100000068CA00A0000200006B652A0EE1
:10D27000180C0000317F31005CEA000460EA000411
:10D2800007F4FFFFB4B40004E0BD000450FD000447
:10D2900054E90004696D000000D10221019200915F
:10D2A0002A0021002DF340FC7CBD38B5040029F391
:10D2B000FBFFA188012088406649097A08420DD009
:10D2C0000820FAF221F8FF21883100900160A1883E
:10D2D0008180614801686846FAF225F838BD70B56A
:10D2E000040000685D4A01680025891808D1FFF72D
:10D2F000DCFF20680125002802D02000FAF207F8A0
:10D30000280070BD10B526F307FE52490020C872F0
:10D3100010BD0821203041737047514938B50500D0
:10D320000968884700282DD04A4CE07A002829D186
:10D33000E8004C49401940014018807C0025002835
:10D3400003D1607A401C60720AE0A07A401C00069B
:10D35000000E0328A07203D1607A401C6072A5728F
:10D36000607A03280ED10420F9F2CEFF3E490090E6
:10D37000016065720120A572E0723C480168684650
:10D38000F9F2D1FF38BD10B5040024F321FA2000D2
:10D39000FFF7C3FF10BD10B5040024F371FA20009D
:10D3A000FFF7BBFF10BD10B52A4904000120097A20
:10D3B000A040084288B01FD004A823F3CEFB200071
:10D3C00008F314FCE000274B00194001C01840305E
:10D3D0008078102204A901AB07C325A20092012284
:10D3E0000021200041231EF32DF9224A0721126853
:10D3F0002000904708B010BD200028F35BF8F9E743
:10D40000FFB581B01E00070002980A280CD1114D0B
:10D410000124287ABC40044206D0039810213CF332
:10D420005CEE287AA0432872039A029933003800F0
:10D4300028F3DFFBC1E510B5FCF279FA00221100F8
:10D4400011201DF357FC0022012111201DF352FC75
:10D4500010BD0000BC5C00B0F4E700045DF0FFFF0D
:10D4600094F60004E0BD0004A90F00005D0229A5A8
:10D470000100000064CC00A000020000729DF47E58
:10D48000D0A63400696D000090F60004012B10B5A1
:10D490000BD0042B07D127483DF323F8002220218D
:10D4A0002548F6F28DFA002010BD24483DF319F806
:10D4B00000220121F4E74B2910B504D11E480022B7
:10D4C0004021F6F27DFA002010BD70B51C4D6C684D
:10D4D000A00706D5184800220421F6F271FA0220AE
:10D4E0006860E00706D0144800220221F6F268FACC
:10D4F00001206860286B0121090608432863002089
:10D5000070BD10B50F4C1048216881600021016189
:10D5100041618161C1610D4901620D4941620D495D
:10D520008162F9F2E1FD00210BA0F9F228FE6060B2
:10D5300010BD0000642101B0782101B0502101B07C
:10D5400000F003A9805D00B0B4EF00B071CC000022
:10D550009BCC0000AFCC0000626C656D627800006F
:10D5600013B50C00FF490098CA7E032A02D0897EB9
:10D57000012904D11C3800903CF3FEFE1CBDFA4A80
:10D580000168914210D1407913280DD1F54A3F230B
:10D59000203A108F1B0201008004800E401E80067E
:10D5A0009943800C01431187F5F736FB210068464B
:10D5B000F9F2C3FE1CBD10B504000022EB480A219D
:10D5C000D2433CF303FF002816D00189002208183B
:10D5D00082710E21C271042301724372012383728E
:10D5E000230AC4720373E04B4273036041710271FA
:10D5F0000A22C280FFF7B4FF10BDDD4800220821D7
:10D6000010B5F6F2DDF910BDDA487047142170B597
:10D610004143D44D1423203D4919096958430A89CF
:10D620001F23521814682A00801800691B030289FE
:10D63000298F1218D0880F260005000D98435379C2
:10D64000FF3CDB06DB0B18431F235B049843137975
:10D650007606DB069B0A184307239B059843CB07F6
:10D66000DB091843C0000123C0085B07C018653CF4
:10D67000B0430832002C05D0BF4BE318EC59812091
:10D680000100000060CE00A00002000086754AC3C1
:10D6900005D101239B0601E001235B06C0188B081E
:10D6A0009B008907A86000D15B1CB9492B870A62DF
:10D6B000086100F0A1FA70BDAF49002230B410003B
:10D6C000F02520390C8F142343435B189B69002BF2
:10D6D00005D0401C000400140228F4DB04E00228FA
:10D6E00002DAAC430C870EE00820C4414006201843
:10D6F0001824E04104060B00240F072C088702D9E8
:10D70000A843012218870120801A0C8F00040014FE
:10D71000A204920E22E0142343435B189B69002B62
:10D7200019D0002809D1102A15D20E22D441012285
:10D730009206A2181223DA410A870A8F0C239A4311
:10D7400083071B0F1A430A878B4905220004CA76F8
:10D7500030BC000C64E7401E000400140028DADA34
:10D7600030BC7047030570B50120834C1B0D0006CB
:10D770008343203C208F0907C507ED092B43DB00BD
:10D780000325DB086D075B190F256D06AB43C90840
:10D790000B43810889008007A36000D1491C7C48A5
:10D7A00021870262036100F027FA70BDF8B5724C60
:10D7B000A07E2500203D002810D0E07E03280CD05C
:10D7C0000320E0760220A076288F72490022884349
:10D7D000288703211000FFF7C5FFF8BD28686E4FAA
:10D7E0000126002819D140216548002200913CF310
:10D7F000F7FD00280FD0417B3143417387610189D8
:10D800000A18101D28600620E0760098121D0121DC
:10D81000FFF7A8FF01200028DFD1686800281AD18F
:10D8200000225E4811003CF3DBFD002811D01421DA
:10D83000C180417B314341732421876101812430C0
:10D8400006216860E17602000221C801FFF78AFF25
:10D8500001200028C1D1E07E0428BED1A86800289C
:10D86000BBD1FFF729FFF8BDF8B50024484FBD69CB
:10D8700041482038C5607E6A0100098F01239B035F
:10D880008C466A0F9943022A13D0032A333BE1C026
:10D89000010000005CD000A000020000F86EED73F3
:10D8A00007D162461A43EB001B0F082B00D00A0079
:10D8B00002877D6100F0AAF93448C07E042801D1B6
:10D8C000FFF77EFFF8BDEA00130F3CF34CED0504B3
:10D8D000040A0A0410000268B24208D10022026061
:10D8E00004E04268B24202D1002242600124018772
:10D8F0007D6100F08BF9002CDED0300000F0A1F942
:10D900000028D9D0A902C90EFFF73EFED4E7410F87
:10D9100070B5032919D11D49C400CA7E230F012AFD
:10D9200014D00425022A1DD0032A0ED10A00927EAB
:10D930000024032B1AD0042B07D1032A05D18C769F
:10D94000CD7600F04FF9FFF73BFF70BD052BFCD102
:10D950000220C876F8F7F8FA16494000085A002263
:10D96000062112E0200FF0D1CD76ECE7074B203BEB
:10D970009D688542E9D1022AE7D1032088769C6020
:10D9800000F099F900220421100015E004F000B025
:10D990000C14000068C800B0782101B0DFCD000091
:10D9A00059EDFFFF00F003A9F03F0000EDCD0000AE
:10D9B00080C800B000000004FFF7DEFE70BD70B547
:10D9C000060014204843D34A8518103524E0D14975
:10D9D0002031CB7E3CF3C6EC08050808050D08088D
:10D9E00014053CF3DDFC17E0010028003CF38DFD3D
:10D9F00012E0010028003CF388FDFFF7E1FE0BE098
:10DA00000189091808314A79097914020C433CF359
:10DA1000C7FC2000FFF7E3FD30003CF34DFD00287C
:10DA2000D5D170BDBB4810B52030C07E042801D1CF
:10DA3000FFF7C6FE012010BDB64A10B52032D37ED6
:10DA4000002B07D0937E002B06D101239376FFF79E
:10DA5000E9FF01E000F0C6F8012010BDAD4810B5A7
:10DA60002030C07E002803D0072801D0FFF706FF32
:10DA7000012010BD70B50120A64CA74D2034E37ED7
:10DA8000A44E3CF370EC071E0505051E09121E008E
:10DA9000E869FFF73CFF14E0E969B2680FFCD1BB0D
:10DAA0000100000058D200A0000200000C8653CEF6
:10DAB0008A4204D1308F0007800F00F0BAF8E9697C
:10DAC000002808D0B068884205D10420E076002004
:10DAD000B060FFF77FFE012070BD9548012110B5B1
:10DAE000FFF777FF012010BD9248002110B5FFF726
:10DAF00070FF012010BDFEB50020471E8E4E019024
:10DB00008E4801227F2101AB0097F5F2E7FE002449
:10DB10000EE0E100725889194D68284204D0002AAD
:10DB200002D00021080090470198A843641C01908E
:10DB300001980028EDD1E3E77B4870B52030C07E26
:10DB400001242200042800D10022774D002120006A
:10DB5000002A06D114224A4352199269002A00D1A0
:10DB60000020491C09060200090E0229EFD3002AF1
:10DB700016D1714E083E317800290AD07068F4F74A
:10DB800048FD7D21C900884201D2012000E000202B
:10DB90003070002802D1288F400403D5002C01D01A
:10DBA000012100E000212000002900D0002070BDEC
:10DBB00070B500255C4C2034E576F4F7C1FA5B487B
:10DBC0000123E376016B03221202914301635C4956
:10DBD0008A680824A2438A60426B1A4342638A68B7
:10DBE00022438A60574981635048403041689A0413
:10DBF00011434160856070BD534810B50468002230
:10DC00005248D24310213CF3FFFB002807D0018982
:10DC10000818FF21633101602100FFF7BFFC10BD30
:10DC200010B5F4F7F2FC4449083948600120087047
:10DC300010BD142358433C4910B54018103000243F
:10DC4000002806D03CF342FC002802D03CF3B2FB93
:10DC50000124200010BD344910B5CA683C4CD100E5
:10DC60000B0F010008393CF388EB05090414220965
:10DC70002E00001FFF216431016010BD0179001FDB
:10DC8000046041711102890F01711105090DC180F4
:10DC900010BD437802781B021A438378C0780002D3
:10DCA00003432B48401C08608A80CB8002B4E3CF3A
:10DCB0000100000054D400A000020000157E8DBEBB
:10DCC00009E0037810020C60800F4B710871100599
:10DCD000000D001DC880080010BD002010BD70B5EB
:10DCE0000025164C2068002803D020383CF36CFB3C
:10DCF00025606068002803D024383CF365FB65602C
:10DD000000242006000EFFF79EFF0028F9D1641CB6
:10DD10002404240C022CF4D301E03CF355FB094805
:10DD20003CF3DEFB0028F8D101E03CF34DFB064854
:10DD30003CF3D6FB0028F8D170BD0000E4EF00B042
:10DD400000F003A9502101B0642101B0905D00B042
:10DD5000782101B0802100801E1E0000E4A634005E
:10DD600068C800B00C140000F8B50500FF4C607ADC
:10DD70001AF319FD06001420F9F2F8FAFC49009094
:10DD80000160FC49098981808572217A817306824C
:10DD900061894182F84801686846F9F2F6FAF8BDEF
:10DDA000F8B5C021F54C2068020060325181EF4E79
:10DDB0000123317BDB020029818B01D0994300E0F4
:10DDC00019438183EE4933780968DD0900D1CB819D
:10DDD000B378DD0900D14B82EA497379FF27E54D1D
:10DDE00009787F1C002B0FD1838B3B438383B07951
:10DDF000F379401800025918084310816020A87177
:10DE0000216800208884F8BD828BBA438283C18355
:10DE1000D649DD480A22006815313CF3CAE8502093
:10DE2000EDE7DA49D34810B50968083086B088476D
:10DE3000D04C1C2120894143D54808188178617154
:10DE40004178E170007920710001C121C9010843C6
:10DE5000D0490968088001202AF3F8FB01A818F3CB
:10DE600099FD01A903A818F316FD2079CA490C23CE
:10DE7000584309680C2240184C3003A918F366FB7C
:10DE8000C64A207913680021400119521368C3184B
:10DE900059801268801881810A21818006B010BDE6
:10DEA00070B5F8F78EFEB54C2068418CCD2211403C
:10DEB0004184F9F23FFBBA480068818C57CB91311D
:10DEC0000100000050D600A000020000E1963303DC
:10DED000090B09038184F9F243FB20680021FF301C
:10DEE000E1304181FFF7A7FFFFF764FF00F0ADF9D4
:10DEF000A3480079FFF742FFA34D01246C7000F0A6
:10DF000082F900F025F92C7070BD1CB59E4AD268CC
:10DF1000019200900021FF201923A7A2FBF267FCC9
:10DF20001CBD70B52BF396FEA44800220068427118
:10DF30000123C370A24C10002568C1006B522568F4
:10DF400049194A80401C0E28F6DB2BF38BFE70BD6E
:10DF500070B58D4C6078002500281FD06570FFF7E4
:10DF6000E0FFF9F2F1FA934E3068418FFF229132CF
:10DF700091434187F9F2E8FA6079316840000A5A22
:10DF8000C0239A430A52F9F2EBFAF9F2E9FA00F0E7
:10DF90008DF9FF20FFF7F2FEF8F71FFE257070BD28
:10DFA000F3B50C0081B0784F7878002804D0207940
:10DFB000FF2801D0FFF7CCFF21797148FF290171BB
:10DFC00009D17878002804D0FFF7C2FF0120FFF7BD
:10DFD0009CFF0020FEBD2178017061784170A1781E
:10DFE0008170E178C1702179017161794171A17904
:10DFF0008171E179C171217A01720091657A45726E
:10E00000E17AA67A09020E434681217B01730199C8
:10E0100012290CD3A27B617B12021143E27B237C89
:10E0200012041B061A4311430161617C02E00021C6
:10E030000161042101755248019915301C2905D34D
:10E0400021000A2212313BF3BEEF03E0FF220A2136
:10E050003BF3B0EF002E07D05A496800085A8642B9
:10E0600002D800980E2801D91220FEBDE806C00F84
:10E07000B870FFF71FFFACE7F8B5534D2868C48FA1
:10E08000008C002801D01CF3B1FF3F4FE00629D5DA
:10E090002868468FF0050BD5F868401CF8603848B2
:10E0A0000069002804D0F968884201D8022038703D
:10E0B00030060DD5387802280AD1FFF732FF3D48E7
:10E0C0000068418FFF228132914341871278177196
:10E0D000010000004CD800A000020000268F315E35
:10E0E00003203870F00607D53878032804D1FFF7ED
:10E0F00039FF0020FFF713FFA00611D52968402043
:10E10000405A80050CD078794200895A002907D0FE
:10E110000A06920F04D0324A09061268091690477F
:10E12000600601D52868C08CE00508D52968002064
:10E1300042005218528E401C0328F9DB088F20063B
:10E1400007D52968002042005218128D401C05286E
:10E15000F9DBA00501D52868C08B600501D52868CA
:10E16000408CF8BDF8B52BF37FFD194800210068FD
:10E170004171084B197AC1700849FF278A7900203C
:10E1800015022E000A79133611353F1D114C4979BD
:10E19000920327E020F000B0940C0000C85D00B0AE
:10E1A000FCA9340084EA00048CEA00041FE900049E
:10E1B000A8EA0004E8FB0004B4B4000480EA000408
:10E1C00088EA000478EA000434EA00046262770016
:10E1D00020EA000428EA000480A9340038EA000498
:10E1E000ECF400040A431204120C0FE0002802D1E0
:10E1F00021680E8002E02368C1005D522368C100DF
:10E20000CB185A802368C9188F80401C4049097A6E
:10E210008142EBDC2BF330FDF8BD10B53D4C012005
:10E22000617988403C4909686031C883F9F296F900
:10E230000020E060F9F292F96079384C40002168E2
:10E240000A5AC0231A430A52F9F294F92068418FFE
:10E25000FF22913211434187F9F28CF910BD304809
:10E2600010B5026813882B4C0121607981400B4363
:10E270001380A2782B4B002A1A68148801D18C4392
:10E2800000E00C43148019680A8823490968FF31AB
:10E2900081310A821E4A142151560C220C2900DABF
:10E2A0000A001321C9438A4200DD110049002931C7
:10E2B0000906090E442900D3432113F072ED10BD65
:10E2C00010B5144C1848E17818F33BF861791748F9
:10E2D00018F337F8208901061548090E4CA05D6037
:10E2E0000100000048DA00A000020000D2678FE3BE
:10E2F00018F331F8218900201C235943124A505445
:10E300000C48006802886379012199408A430280A1
:10E310000948006802888A43028002888A43028092
:10E3200010BD000020F000B0C85D00B084EA000419
:10E3300034EA000430EA00041CEA000488E800041F
:10E3400084E8000480E80004B4B40004020010B5BE
:10E35000937811203CF338E8081B05080E0B1114C4
:10E36000171B10001C4A10E010001C4A0DE01000A2
:10E370001B4A0AE010001B4A07E010001A4A04E09A
:10E3800010001A4A01E01000194A1268904710BDA7
:10E3900070B5060010781400E02886B004D1200083
:10E3A000FFF7D4FF050000E011250021481EFBF215
:10E3B00049FB2279E178A07803AB07C33300627888
:10E3C00021780191FF21029221310E2009A20095AE
:10E3D000FBF221FA06B070BD0CF9000410F900043C
:10E3E000FCF8000408F9000400F90004F8F800043F
:10E3F00004F9000452686262626262620000000016
:10E40000F8B50D0000210091382116004143FA4A69
:10E410008C180021F9F74DFE00282AD0607DC11C20
:10E420008A07411C8000001983698907920F890FB0
:10E43000002B0AD1876A002F07D192001219976921
:10E44000002F02D1926A002A01D001220092002DF1
:10E4500008D0002E06D02A68D2182A603268806A56
:10E460001018306000228800001982618262A27553
:10E4700061750098F8BDF8B538235843DE4B8E7AA5
:10E48000C418C87A4B7A00020643087A1B02184364
:10E490008446E07C257C042801D3002D75D10879C1
:10E4A0005700022805D0032831D006287BD1002050
:10E4B00055E0002102206174009008256046112873
:10E4C00006D0132804D019286FD101250095A17416
:10E4D000207C002804D1382120003BF324EE0FE0FB
:10E4E00000208100625A002A05D1091936CA23F694
:10E4F0000100000044DC00A000020000CB9F51930B
:10E500004988002901D1207504E0401C0006000E56
:10E510000428F0D3207D81000819C6532574009883
:10E520004AE0207D800003190120002A00D000204D
:10E530004000185AB04240D10222012D05D1227468
:10E54000012262740022A27404E0082D02D1092085
:10E5500020746274087B002805D1487B002802D112
:10E56000E07C401CE074217D60468A001119C8538C
:10E5700023E081000B19D95BB14211D10121002A9E
:10E5800000D000214900595A614509D18200111972
:10E5900000220A804A80E17C491EE17405E016E011
:10E5A000401C0006000E0428E3D3002805D1082DE6
:10E5B00005D0092D03D020746074002D08D0207C74
:10E5C000002805D1F5F75AFE0020F5F74EFEF8BDFC
:10E5D000607C0128FBD1F5F751FEF8BDF8B50024A9
:10E5E00006008A4F250000212800F9F76CFD00285D
:10E5F0001AD0002E03D1641C2406240E14E0012E30
:10E6000008D138206843C019007C0128F3D00228C3
:10E61000F1D009E0022E07D138206843C019007CF0
:10E620000828E8D00928E6D06D1C2D042D0C082DF3
:10E63000D9D32000F8BD0020D0E71CB500207449D4
:10E64000019000900400087020006A4601A9FFF7BD
:10E65000E1FE002801D000F003F9641C2404240C1E
:10E66000082CF1D300990198F5F71AFE1CBDFFB5EF
:10E6700083B0050008285CD238236B4363489207B7
:10E680001C18677CA07C029048780E780002CB783A
:10E69000064388781B021843920F012A49D0069A34
:10E6A000012803D0280000F0E9F802E02800FFF775
:10E6B000ECFE607C2A003100FAF7F4FF069800288F
:10E6C000607D05D080000019816A8919816204E0AB
:10E6D0008000001981698919816100F0C1F8607CAE
:10E6E000B84208D1002824D0012822D16B46A17C51
:10E6F0001A7A91421DD0012801D101265B929344E0
:10E700000100000040DE00A0000200003F77EF2E75
:10E7100000E000260127022800D000270C20F8F294
:10E7200057FE41490190016085808671A17C01728C
:10E73000C7713E48016801A8F8F259FEA17C607CCF
:10E740002A00FBF726F807B0F0BD70B504000828D2
:10E750001CD2002211002000FFF766FEFFF775FFB4
:10E7600000280CD12F4D2878002808D030480021EF
:10E7700029F3D5FF002001002870F5F79BFD382014
:10E7800060432749401838213BF3E0EC70BDF0B5F9
:10E7900000263821414387B0214A05968A18162160
:10E7A00004960296019600925156350037000029D2
:10E7B00001D00E0051E00021F9F78FFC00284CD069
:10E7C0000024009AA00082189069012319000028F3
:10E7D00000D00021C9190F06916A3F0E0029069149
:10E7E00000D000230199049A59180906090E8018CF
:10E7F0000191059B002159410490029A06980591C8
:10E80000801800214D41641C2406240E042C029023
:10E81000D7D3022F0ED3019802280BD300261AE07B
:10E8200040F000B0D85D00B0120D000000AA340026
:10E83000F3130000029A049805992B00121A8B41D9
:10E8400001D2012607E0029A04980599801AA9418D
:10E8500001D20026F64300988675300073E7010068
:10E86000382359432C4A01208918497C022900D0B9
:10E8700000207047294810B50178002907D10121EF
:10E8800001707D2026490022C00029F335FF10BD0C
:10E89000F7B53823009858431F4BC518C8788B78B4
:10E8A00000020343287C012807D0022805D008284D
:10E8B00001D0092803D1022402E0012400E0002451
:10E8C0000120002A00D000204600A85B984206D113
:10E8D000012C6C7402D10120F5F7DAFCFEBD012099
:10E8E00081004919895B99420FD1012C6C74F5D1D3
:10E8F0000220002A00D10120A874FAF765FFA97C44
:10E90000009A2000FAF745FFFEBD401C78ED5E0836
:10E91000010000003CE000A00002000037A81EF348
:10E920000006000E0428E5D3FEBD000040F000B054
:10E93000D85D00B0F31300002E4810B50068002227
:10E940004B21F8F2CCFC10BDFFB581B006000D00E4
:10E950003C292CD82F0009373806000E30F3FEFB77
:10E96000040024D02089244900190160002101718C
:10E9700022492A00096841711F49C7800830783947
:10E980000160868085710399C01D3BF34EEB1948E9
:10E9900000220068210001233BF3CAFD04980028EF
:10E9A00003D100210120FEF2D2F805B0F0BDB3057D
:10E9B00012219B0DB20A0420FAF2F2FFF5E7FFB52F
:10E9C00081B0050016001F0030F3C8FB0400ECD036
:10E9D0002089FF2100196531016007714671C580EA
:10E9E00002992A0008303BF320EB200030F3BCFBF7
:10E9F000DBE70000845D00B00A140000E4A63400E8
:10EA0000F8B5002406008038864B87490004000CC6
:10EA10001A5C0D88854F52190A801C5411E0A00021
:10EA20003D58A8880005000DB04207D11C3D2000CC
:10EA3000FAF2E3FB28003BF303FD02E0641C24062A
:10EA4000240E7B4800788442E9D3F8BD10B5C17824
:10EA5000827809020A4324381C2143180181754930
:10EA6000C16103211971744909685971111D4184EB
:10EA700001007248042300683BF35AFD10BD70B5D5
:10EA800004000D000020F8F705FB052D19D1E188E1
:10EA9000A088091D0A046A4900050978000D120CB6
:10EAA000002912D0010080393F290ED85E4B198809
:10EAB000491E19805B49081880380178491C01708B
:10EAC00003E0E088001F0204120C5E482100006889
:10EAD0001C392B003BF32CFD70BD594930B409782B
:10EAE000002903D050490988002903D056490968F4
:10EAF00030BC08474E4A4D4C11788B00491CE05001
:10EB0000117030BC704770B5474C2588FFF778FF0F
:10EB10004E4A20881388411BC918401A903BEEB614
:10EB20000100000038E200A000020000C340A04E37
:10EB30001180208070BD10B580242000641C240446
:10EB4000240CFFF767FFBF2CF7D910BD1CB5454A51
:10EB50001178002912D09178D2786B461A705870CB
:10EB60000A0A9970DA700A0C1A71090E59713E4C32
:10EB70000300062120006A46FFF7F0FE1CBD0006D8
:10EB8000001610B513F042E90020FFF7DFFF10BDBB
:10EB9000020035480A21801C012310B5FFF7DEFE74
:10EBA00010BD10B52F4C6070A170E2700120636041
:10EBB000207010BD00B589B000906B462B481971CC
:10EBC000006800230206120E24206946FFF701FFA9
:10EBD00009B000BDF0B50400241D61792579090252
:10EBE0000D432349234B0E782168002002229942CD
:10EBF00021D130207043204B0021C6180F0048005F
:10EC00004018A31830181B79521C12048370120C80
:10EC100001238B402B4205D005230370114BDB7879
:10EC2000437002E0077047708770491C0906090E9F
:10EC30001029E4D30120F0BDA09D0004A8E5000444
:10EC4000E09D00049CE500040B140000E0A63400E5
:10EC5000845D00B09BE50004880E0004B0E500046C
:10EC6000AAE50004DC5D00B087FC0000E4A63400E7
:10EC7000CD5B00B05321000000F200B00100002283
:10EC80000C48D243083110B53BF30EFC10BD10B553
:10EC9000040000681C383BF3DDFB0020206010BD41
:10ECA0000100054810B50068002201233BF34AFC2F
:10ECB00010BD000068C800B0845D00B010B52A4CDB
:10ECC0002848208004F096FF60602648401C208180
:10ECD00005F015F82100C86010BD31B50098002876
:10ECE00019D0214D00240098E1006A5A83889A4285
:10ECF0000ED149194B68002B0AD081790022C01D22
:10ED00009847002804D06846F8F279FB012038BD06
:10ED1000641C022CE7D3002038BDFFB581B00C0085
:10ED200007000498114D461830000F30AD861703C8
:10ED30000100000034E400A000020000DAB87E3ECA
:10ED4000F8F264FB0028009014D005600772467248
:10ED5000039922000A303BF37CE90098049A0019D9
:10ED60000A990A303BF374E9064801686846F8F2EC
:10ED70005CFB012005B0F0BD80FE000060F200B039
:10ED80009C130000E0A6340030492F480860314849
:10ED90002F494160314930480860324930480860A5
:10EDA00032493148086033493148086033493248B4
:10EDB00008603449324808603449334808603549AE
:10EDC000334808603548344901603549364A416066
:10EDD00034491160364A354911603649C1603649B7
:10EDE00001613649374A416135491160374A364930
:10EDF0001160384A36491160384A37491160394A3A
:10EE000037491160394A384911603A4A3849116026
:10EE1000394981603A49394808603A483A490860B6
:10EE20003B493A4808603C493A4808603C493B48FD
:10EE300008603D493B4808603D493C4808603E4900
:10EE40003C480860704700009C5E00B078ED00040C
:10EE500050F500B070DC00044934010000EF0004FC
:10EE60004134010004EF0004A93D010008EF000453
:10EE7000373E01000CEF0004A13F010010EF000439
:10EE8000B33F010034EF00045940010030EF0004AB
:10EE9000F73F010014EF00044B3A0100E45D00B0BD
:10EEA000733A0100633B0100F4EF0004A13A010052
:10EEB000BCEF000489380100C5380100633D010042
:10EEC00003390100DCEF0004D9360100A0EF000493
:10EED000314101008C5E00B09F410100985E00B09E
:10EEE000905E00B068ED0004D541010074EF0004AD
:10EEF0004D44010070EF00046B430100785E00B0E8
:10EF00006CED00047C5E00B070ED0004A9440100CB
:10EF100020F00004AD44010058F00004CB4401008F
:10EF20005CF000041746010060F000042941010074
:10EF30002CF000048547010050F00004BB9FD7442B
:10EF40000100000030E600A0000200002E50C08347
:10EF500037493648086038493648086038493748E4
:10EF600008603949374808603949384808603A49E3
:10EF7000384808603A49394808603B4939480860D0
:10EF80003B493A4808603C493A4808603C493B489C
:10EF900008603D493B4808603D493C4808603E499F
:10EFA0003C4808603E493D4808603F493D4808608C
:10EFB0003F493E48086040493E48086040493F4854
:10EFC000086041493F48086041494048086042495B
:10EFD0004048086042494148086043494148086048
:10EFE000434942480860444942480860444943480C
:10EFF0000860454943480860454944480860464917
:10F000004448086046494548086047494548086003
:10F0100047494648086048494648086048494748C3
:10F02000086049494748086070470000B0F900B0DF
:10F0300008F20004885F00B00CF20004940600049B
:10F0400010F20004B006000414F20004D3700100B2
:10F050009CF10004A3480100B0F100040F49010035
:10F06000B4F10004FFBA01001CF20004D9BB010096
:10F0700020F20004DDBA010018F20004E3B9010037
:10F0800054F10004D3B8010050F200042DB3010084
:10F090006CF2000421BD01002CF2000409BE010045
:10F0A00094F200043DBE010098F20004CDBD0100C1
:10F0B0009CF2000445B7010064F200048D5B01007E
:10F0C000F0F20004D35B0100F4F20004636301007A
:10F0D00014F300048F6301001CF300049D6501001C
:10F0E0002CF30004FF650100F8F2000497660100AC
:10F0F00024F30004B9A001004CF3000463A1010053
:10F1000068F30004B9A101006CF30004D7A1010069
:10F1100074F30004EBA1010060F30004934600B017
:10F1200084F000049DAD010088F00004EDAC010006
:10F130008CF00004DDC7010078F300043FC001003B
:10F140007CF300045DB0010080F3000423B98A8DD4
:10F15000010000002CE800A000020000E949C2DE26
:10F1600010B50FF080F9012000F0F5F810BD7F4ACE
:10F1700010B551880B00034209D081437C4851806F
:10F18000014202D14808400050800BF078FE10BDCB
:10F190000120ECE7022010B500F0DDF810BD0220E0
:10F1A000E5E7042010B500F0D6F810BD0420DEE736
:10F1B00001204002DBE7082010B500F0CCF810BDBC
:10F1C0000820D4E7102010B500F0C5F810BD1020BD
:10F1D000CDE7202010B500F0BEF810BD402010B5DE
:10F1E00000F0B9F810BD6020C1E7802010B500F034
:10F1F000B2F810BD8020BAE70120800210B500F0FF
:10F20000AAF810BD01208002B1E7FFB581B0160059
:10F21000994200D919000D0054480021554F0C00A7
:10F22000818013E0305D00280DD0019821000BF0A3
:10F23000F3F881007A5C824205D14C4AC919908862
:10F24000498808439080641C2406240EAC42E9D30C
:10F250000BF015FE05B0F0BD4449087070474348F7
:10F2600000787047414A00B55288002103003BF303
:10F27000F2E80A06080A0D0F060D111321140221E7
:10F280000BE0042109E00121490206E0082104E025
:10F29000102102E0202100E040211000084000D0B1
:10F2A0000120114000D00121002803D0002901D005
:10F2B000012000BD002000BD2C4841880020CA0765
:10F2C00005D02B4A114202D0002900D001207047FE
:10F2D00070B50025FFF7F0FF002812D000240121AF
:10F2E00020000BF020F9092805D0FFF7BBFF00280C
:10F2F00001D0012504E0641C2406240E0A2CEED360
:10F30000280070BD19480B214088C901084000D071
:10F310000120704715484088C005C00F704713484A
:10F3200040884005C00F70471349012010B588710F
:10F330001248007806280DD10C484188090609D5E5
:10F340000078012806D10E49096888470D498020B8
:10F350000968884710BD054A10B55188A8C216C46F
:10F360000100000028EA00A0000200001DA17C634B
:10F3700003008B4303D0014351800BF08AFD10BD85
:10F38000FC5D00B07E02000004030004455F00B095
:10F39000365F00B0D4F20004D8F20004FF48002128
:10F3A000FF22017042708170C1700171417141731F
:10F3B000012181737047FA4810B500680024804726
:10F3C000F6498878002808D0072809D14879042808
:10F3D00006D10EF08CF9002802D001240EF020FA9C
:10F3E000F04800688047200010BDED4870B5006807
:10F3F000804702200CF0CDFAEB48EA4D0078062851
:10F4000006D1EA480078002802D02868804770BDFD
:10F410000BF0E0FAE14C002805D10EF041FA00288B
:10F4200001D1042000E003206071286880476079E2
:10F430000428ECD10BF0C4FA002802D0DC480068A4
:10F44000804706F009FB002801D006F0CBF9D94926
:10F450006078096888470EF0C1F90720A07007F0AE
:10F46000E9FF70BD10B50BF0ABFA002802D0D04810
:10F470000068804706F0F0FA002801D006F0B2F9E3
:10F48000CC49C64C096860788847042060710EF04A
:10F49000A5F90720A07010BD70B5C04DA878002850
:10F4A00028D000242C706878FF2808D0C249096849
:10F4B0008847002803D0BF496878096888470BF05F
:10F4C0007FFABE4E002805D00BF072FAB168012019
:10F4D000887401E0B068847406F0BEFA002801D098
:10F4E00006F080F9A878092805D100200EF046F929
:10F4F000AC706C7170BD0120F8E770B5002806D0C3
:10F50000002901D0AE4C04E0AD4CA41E01E0AC4C8F
:10F51000A41C022501200EF08CF9002809D0A94B6B
:10F520002A001B6801002000984701200EF0EDF929
:10F530000120002806D1FFF7AFFF022101200CF0C7
:10F5400051F970BDA14B954805211C68C90140784F
:10F550009D4A0023A04770BD70B500288F4C42D152
:10F56000A0789A4D012810D10EF0CAF87559249050
:10F570000100000024EC00A0000200000459A213C6
:10F5800002210028A17006D060782C682021934ABF
:10F590000023A04770BDFFF789FF022125E0022864
:10F5A0000ED10320A07001206071607805212C68C5
:10F5B000C9018A4A0023A04701200EF0C2F870BD9D
:10F5C000032803D0042801D0072812D12078401C3A
:10F5D0000006000E032820700BD8E078012800D028
:10F5E00000200121FFF793FF70BD01200CF004F90A
:10F5F00070BDFFF75BFF0321F7E70128F8D16F48E3
:10F6000001786F48062902D101780029F0D1007AEB
:10F61000FF2804D06D49096888470028E8D1A07800
:10F620000528E5D102200CF0BEF904206071072006
:10F63000A0700EF0DDF80BF0CDF9002802D0614883
:10F640000068804706F012FA002801D006F0D4F8CE
:10F6500007F0FAFE70BD10B50EF0DEF85448002138
:10F660000170012141715E4B05211C68C901407880
:10F670005A4A0023A04710BD70B505004C4C607875
:10F68000FF2804D157490020096888476070280086
:10F690000DF0F8FF002801D00EF001F870BD10B594
:10F6A000434CA078082810D10920A0700EF032F841
:10F6B00000280CD04A4B60781C6820214A4A00235D
:10F6C000A04701200EF03DF810BD092801D1FFF739
:10F6D000EDFEA1680120884710BD70B50600344CCE
:10F6E0000D00A078002803D00120A847002070BD9D
:10F6F0003848001D805DFFF7BFFF002802D10EF0E3
:10F7000047F8F1E70820A07000202070A560344B76
:10F71000267360781C682021334A0023A04701200B
:10F7200070BD10B5224C0022227062732271E1700C
:10F730000121A173A1702749091D085CFFF79CFFF7
:10F74000002804D101200EF023F8002010BD244B26
:10F7500060781C682021214A0023A047012010BDA9
:10F76000F8B50125124EB078072803D000210120FA
:10F770000CF042F80520B07030790028FAA72DEF80
:10F780000100000020EE00A000020000F0B11CAE5D
:10F790003BD001F090FD040037D0E088022834D936
:10F7A000A188891EA1801649801EE080096820007A
:10F7B000884707000CF0E9FD002826D0210038001A
:10F7C00020E000007CF200B0CCF20004D0F2000493
:10F7D000365F00B0455F00B064F3000438F3000406
:10F7E0003CF3000440F600B02E030004D0F1000406
:10F7F00011EC000030F3000434F3000443ED00008A
:10F80000C4F1000406F018F809E00BF0BEF8002877
:10F8100004D0002030700220707100E00025280024
:10F82000F8BDF1B582B001260298C588002D01D13E
:10F830000020FEBDA5490298096888470400A44835
:10F840000178032906D9FFF73BFE032101200BF0C5
:10F85000DDFFEDE783789F499F4FDB1E3AF318EEFB
:10F8600007054A61F8A8F8E5F80099480968407862
:10F870008847032D01D0042D2FD1600903282CD1F6
:10F88000E7200440612C28D1904C029821688847D9
:10F89000924D297A884205D1216802988847697A71
:10F8A000884205D08A48002101710120387402E0A5
:10F8B000874901200871864CE078012807D1002192
:10F8C000FFF72FFE002020700420A0700DE000281C
:10F8D0000BD1FFF74FFF060007E07D48C0780128F5
:10F8E00000D000200121FFF71CFE79480178491C57
:10F8F000017084E00968070040788847012D01D035
:10F90000022D06D16009032803D1E7200440602CB2
:10F9100072D038780121401C38700800FFF701FED2
:10F9200075E00968050040788847A87B002806D064
:10F930000020A873387C002801D10CF049FD600933
:10F94000022805D10298210006F007F8060026E0FB
:10F95000E00924D062480190077C06F091F8002865
:10F9600001D005F053FF06205E4AA8701268029885
:10F9700021009047002801D100260EE0002F0CD076
:10F9800001980078002808D0574800684EA697EFE5
:10F99000010000001CF000A0000200008EAABB1EA7
:10F9A0008047002803D1564902200968884705206E
:10F9B000A870554B7D211C6889026878514A012343
:10F9C000A04726E04748096840788847032D2AD198
:10F9D0006009032827D1E7200440612C23D1404C43
:10F9E000029821688847424D297A884205D12168CA
:10F9F00002988847697A884205D03A480021017107
:10FA00000120387402E0374901200871FFF7BCFE7D
:10FA10000600002E05D1FFF75DFD022101200BF04D
:10FA2000FFFE3000FEBD2F4CE078012800D0002002
:10FA30000121FFF780FD2078401C2070F1E7096864
:10FA4000070040788847032D01D0042D0BD16009B1
:10FA5000032808D1E7200440612C04D100240A20A7
:10FA6000B87001E006E00124FFF734FDB96820001A
:10FA70008847D6E70026CEE770B50500194CA07878
:10FA800005282CD11849607809688847002D03D0D3
:10FA90001E480068804717E06079032814D10420CD
:10FAA00060710720A0700DF0B7FE0AF0A7FF0028D4
:10FAB00002D017480068804705F0ECFF002801D00D
:10FAC00005F0AEFE07F0D4FCA078052807D10E4B58
:10FAD00060787D211C6889020A4A0123A04770BD15
:10FAE000C4F100047CF200B038F3000470E00004BC
:10FAF00090ED0004CCDF000454F3000448F300044C
:10FB000044F2000411EC000030F3000470F3000430
:10FB100064F3000470B50D004178040000782A00F9
:10FB20000BF022FD002803D0FF4920784855012022
:10FB300070BDFD4A10B5115C052908D0FB4C890049
:10FB4000091949680023DB434B600521115410BD9E
:10FB50000522F548110010B53AF3AEEAF24900204B
:10FB60008860C8748873487410BDF8B50400150027
:10FB70000220F8F723FDEC48005D052815D0810030
:10FB8000EA48081840684168A1420ED14078E84E22
:10FB9000E84F01280AD1E8492800096817D4443100
:10FBA0000100000018F200A0000200007A4205A344
:10FBB0008847002804D03A68012120009047F8BD0A
:10FBC000316828008847F6E710B50DF0BCFB002827
:10FBD00009D00022C2706122012102700A22427003
:10FBE0008170D649886010BD70B5D44CA0680028DB
:10FBF00009D081780025012902D80DF0A0FB01E091
:10FC00000DF0ABFBA56070BD00280BD0022809D019
:10FC1000052807D0CA4A810089184968497802290D
:10FC200000D101207047FFB581B006000D0000280B
:10FC30003BD0052E39D03000FFF7E6FF0400052841
:10FC400033D0039930000BF080FC00282DD0BB4E40
:10FC5000B268002A29D09078401DF62806D3FFF715
:10FC6000C3FFFFF7B1FFB268002A1ED0D31C111DDD
:10FC7000D678002005E04F78891C7918401C0006D2
:10FC8000000E8642F7D8761C0120002D1E7000D091
:10FC90000020087003204870891C0C70039848707D
:10FCA000049888709078401D907005B0F0BDFFB545
:10FCB00081B00D00070016000028F6D0052FF4D003
:10FCC0003800FFF7A1FF04000528EED0310038000E
:10FCD0000BF03BFC0028E8D006200DF036FB002896
:10FCE000E3D00122C11C002DC27000D000224A7056
:10FCF00003228A70C91C0C704E70049A8A706121AC
:10FD000001700A214170062181700DF026FBCCE7BD
:10FD1000FEB5052500280CD0894901280CD0022801
:10FD200007D0052805D0820051184968497A002972
:10FD300000D105002800FEBD814800248068C66807
:10FD4000307A0028F6D0012801D1346817E0804BC2
:10FD500000211F68BA206A4601ABB847307A009A82
:10FD600000210AE08B00F3581778DB681B78BB4250
:10FD700002D18800345802E0491C8842F2D8002C95
:10FD8000D8D060780228D5D16D480321027808E0E8
:10FD90008B001B185B68A34202D10D062D0EC9E72C
:10FDA000491C8A42F4D8C5E7052810B59652C37F8E
:10FDB0000100000014F400A00002000063BADBD3CD
:10FDC00008D0002806D0634B8200D2185268527ABD
:10FDD000002A01D0002010BD0BF092FA10BD5C4843
:10FDE000052210B50021C27301740273417312F031
:10FDF0006CE810BDF7B50E00FFF794FF050005286D
:10FE000001D10920FEBD0124F00709D0029A00218A
:10FE1000280012F05EE80400FFF7C2FA002C40D080
:10FE20004B4FB0071DD5387B052801D0A84202D121
:10FE3000F87C002801D0002433E03D7302980BF0D9
:10FE4000D2FE797B08437873029A0121280012F0D0
:10FE500040E8B97B0400014301D0012000E000200C
:10FE6000B873002C1DD070071BD5F87B052801D076
:10FE7000A842E0D1F87C0028DDD1FD7302980BF098
:10FE8000B2FE397C08433874029A0221280012F02D
:10FE900020E8797C0400014301D0012000E000202B
:10FEA00078740020002CADD10320FEBDF7B50E0004
:10FEB000FFF738FF0500052801D10920FEBD012408
:10FEC000F00709D0029A0021280012F006E8040089
:10FED000FFF766FA002C4DD01D4FB0071DD5387BBB
:10FEE000052801D0A84202D1F87C002801D00024C6
:10FEF00040E03D7302980BF088FE797B08437873ED
:10FF0000029A0121280011F0E8EFB97B04000143B7
:10FF100001D0012000E00020B873002C2AD0700727
:10FF200028D5F87B052801D0A842E0D1F87C00282C
:10FF3000DDD1FD7302980BF068FE397C08433874FC
:10FF4000029A0221280011F0C8EF797C04000BE02E
:10FF50008CF200B040F600B0BCF100047CF3000469
:10FF600068F20004ECF10004014301D0012000E03C
:10FF7000002078740020002CA0D10320FEBDFFB526
:10FF800081B00E001D00FFF7CDFE0700052801D14E
:10FF9000092094E60124F0070AD0039A2B000021DF
:10FFA000380011F09EEF0400FFF7FAF9002C13D08F
:10FFB000B00706D5039A2B0001213800BDCD446956
:10FFC0000100000010F600A0000200009752656ECC
:10FFD00011F090EF0400002C08D0700706D5039AAA
:10FFE0002B000221380011F086EF04000020002CC5
:10FFF000D9D103206DE6FFB581B01E00FF494978D5
:020000021000EC
:10000000002921D000281FD005281DD0FFF710FEA1
:100010000500052818D0F01C07063F0E38000DF02B
:10002000A8F9040010D0E570029921716671039956
:100030003200A01D3AF366E861202070092060704C
:100040002000A7700DF09DF943E6FFB585B00400D0
:100050000E00002702970F70089811F050EF05006E
:1000600075D00798002808D001283BD002286ED10F
:10007000E87C002835D0002099E028780028F9D0C5
:100080000020019029E001982818417805291DD009
:1000900000212170032161704078FFF7C9FDA07035
:1000A00008980BF08AFDE0700198207102987F1C7F
:1000B000401C0006000E0290307861783F06401820
:1000C000801C307060783F0EA41C04190198401CFD
:1000D0000006000E042801906DD229780298814212
:1000E000D1D868E06879002865D00020019029E027
:1000F00001982818817905291DD00121217003213B
:1001000061708079FFF794FDA07008980BF055FDA1
:10011000E0700198207102987F1C401C0006000EC0
:100120000290307861783F064018801C307060780B
:100130003F0EA41C04190198401C0006000E09285B
:10014000019038D2687902998842D1D833E035E0FD
:1001500001981223584340190490203003904079AD
:10016000052820D00220207003980079801C607040
:1001700003984079FFF75CFDA07008980BF01DFD17
:10018000E0700398049902791431201D39F3BAEF15
:10019000307861787F1C4018801C307060783F0692
:1001A0003F0EA41C04190198401C0006000E01908B
:1001B000E97C8142CCD8380009B0F0BD0020FBE7D3
:1001C000FEB5050000208E490090096801E59335D1
:1001D000010000000CF800A000020000504B673343
:1001E000F62088472B00002269460190FFF737FF71
:1001F00001266127002802901BD06B461878801CCE
:100200000006000E0DF0BFF80400C01C0670029935
:1002100041706B461A780199801C39F37EEF0221F8
:1002200027706B46617019782000891CA1700DF051
:10023000B2F801982B0001226946FFF710FF002851
:1002400002901BD06B461878801C0006000E0DF043
:100250009AF80400C01C0670029941706B461A7827
:100260000199801C39F358EF022127706B466170A9
:1002700019782000891CA1700DF08DF801982B00D1
:1002800002226946FFF7EBFE05001AD06B4618788C
:10029000801C0006000E0DF076F80400C01C0670ED
:1002A00045706B461A780199801C39F336EF0221AC
:1002B00027706B46617019782000891CA1700DF0C1
:1002C0006AF85549019809688847FEBD002010B5B5
:1002D000FFF780FF0120FFF77DFF0220FFF77AFF85
:1002E00002200DF050F80022C270612102710170ED
:1002F0000221417081700DF04EF810BD022010B542
:100300000DF041F80022C2706121027101700521D7
:100310004170022181700DF03EF810BD022010B531
:100320000DF031F80122027103226121C2700170C7
:1003300006214170022181700DF02DF810BDF3B53A
:1003400081B001250F0028000DF01DF84F2101702C
:100350000021417001210400C61C012F817000D2D0
:10036000002501980078FFF7F1FC2C498000401827
:1003700040684078032800D0002511F0CEED002819
:100380000DD1002D0BD0022011F0CAED002806D0AF
:100390000020307020000CF0FEFF0020FEBD032086
:1003A000F7E7F8B5070002293FD3891E0D06387814
:1003B0002D0EFFF7CBFC022837D1BC1C002651E0E4
:1003C0002078002833D001282FD1A01C0B2D2CD34E
:1003D0000B3D01782D062D0E022926D1ABF2E1B698
:1003E0000100000008FA00A000020000A4A3D98EBA
:1003F0004178042923D18278417912061143C278C9
:10040000037912041B021A431143801D0278032A48
:1004100015D14278012A12D36B1C9A420FD80904D5
:10042000090C07E084E00004D8F10004DCF10004CA
:1004300040F600B0801C04F0EDFE002818D1032027
:10044000F8BD062DFBD360780428F8D1A178607937
:1004500009060843E1782279090412021143AD1F0D
:1004600008432D0600042D0E000C04F0F1FEE4E715
:100470006078A41C0419761C7878B042AAD80020B1
:10048000F8BD10B5FFF797FF04000BD101200CF069
:1004900084FF4F2202700222427001228270C470D7
:1004A0000CF083FF200010BDF3B581B00CF073FF9A
:1004B0000500C41C02980126032703285AD302987A
:1004C000401E0006000E029001980078FFF748FCDD
:1004D00002284FD101984078002823D0012849D123
:1004E00001980299C01C082944D30178022941D1FE
:1004F000417804293ED18178427909060A43C178BE
:1005000000790904000201430A43009204F0ABFEA3
:10051000009AF12182422DD2009A801AF12814D932
:100520000E0014E004F09FFE0299022922D300225B
:1005300004216270A170010EE170010C2171010AA9
:100540006171A0710726227015E00604360C0120A7
:100550006070B01CA070E770267100993200090429
:10056000090C601D04F066FE0020761D3604360C72
:10057000207000E0277024784F2028706F702800CA
:10058000AE700CF012FF2000FEBDF7B5901C1500F8
:100590000606360E30000CF000FF009A040000271B
:1005A000C01C3900002A00D1032101704570019957
:1005B0002A00801C39F3BAED6F202070677020008C
:1005C000A6700CF0F2FEFEBD70B50400FC4D0026D6
:1005D000297B012800D0E97B052914D011F0AEEC6D
:1005E00011F0B0EC200011F0B2EC0028DE7B5531A8
:1005F0000100000004FC00A000020000BD5B07FE3B
:100600000BD0A87C002800D001240120012C00D1AF
:100610000020002111F0A8EC0600300070BDF8B5F4
:1006200000240327EB4D2600287D00280BD001284D
:1006300021D002282BD0032845D1012011F098ECBD
:10064000042028753DE0687C002807D00220FFF7D1
:10065000C5FF00280CD0012028750AE0A87B0028DF
:1006600006D00120FFF7BAFF002801D02F7500E067
:1006700001246E741EE0012011F07AEC01210800C3
:1006800011F072EC002817D002202875F8BD012067
:1006900011F06EECA87B002808D00120FFF79EFF28
:1006A000002801D02F7504E0012402E00420287501
:1006B000EE74AE73002C06D0042028756F756E742E
:1006C000AE73EE7402E0287D0428DFD10021012002
:1006D0000AF061FCF8BD10B5BE4CA07B002807D124
:1006E000607C002804D1002101200AF054FC10BDD8
:1006F000B94800688047E07CB849002804D0086801
:10070000804703206075EEE7627C0120002A00D05C
:10071000A074E0740868804700202075FFF77FFF11
:1007200010BD7CE7AB490120C97C002900D0002026
:100730007047F3B583B005000026049C641C0228B2
:1007400015D100202070A64901206070097BA1709E
:10075000E41C207002206070A2480226017AA17079
:10076000407AE070241D0021282001AA02E0002127
:10077000272001AA9C4B1F686B46B84702202070B7
:100780000820607002000199A01C39F3DAEC60784F
:10079000761CA41C36060419360E022D01AA02D1BD
:1007A00000212D2001E000212B208F4B1F686B467C
:1007B000B84703206B462070187860701A7801994A
:1007C000A01C39F3BEEC6078A41C0419761C30061A
:1007D000000E022D02902AD104202070834E262282
:1007E00062703168A01C39F3ACEC6078029FA41CE5
:1007F000041905214C22217062703168966E2E72A8
:100800000100000000FE00A00002000049B3B9434F
:100810007F1C2631A01C39F39EEC6178A01C0C18BB
:10082000062113222170627031687F1CA431A01C44
:1008300039F390EC6178A01C0C187F1C3806000E70
:1008400002900720207000200600A71C6070062080
:1008500070436C4941188878A84207D16078062215
:10086000C01939F378EC6078801D6070761C36060C
:10087000360E042EEBD314E00621714361480918AB
:10088000487800280AD08878A84207D160780622E4
:10089000C01939F360EC6078801D6070761C3606F4
:1008A000360E2C2EE8D36078049AC1190298401CA9
:1008B00010700498081A0004000C05B0F0BDF7B5DC
:1008C00082B00024170001297ED302780229019208
:1008D00000D3441C491E0806000E039001987AE0DC
:1008E00062780399901C88426FD80398801A801E02
:1008F0000006000E0390237839F31AEE0862050B08
:10090000161C20272C623C48A1780172E1784172C4
:1009100056E013002820022F00D027203A4DA21CB9
:100920002D680021A8474BE013002D20022FF5D0A1
:100930002B20F3E73248A11C006803E03048A11CDB
:100940000068263039F306EC3AE02D48A11C006817
:10095000A430F7E7A61C38000BF08FFF29490025CB
:100960000620684340188278BA4205D172784270F6
:100970006078B61D801F60706D1C2D062D0E042D35
:10098000EED318E0062169431E4808184178002973
:100990000ED13178891CA9420AD1B178B94207D168
:1009A0000622310039F3D6EB6078B61D801F6070E7
:1009B0006D1C2D062D0E2C2D02D260780028E1D161
:1009C0006078A41C041901E007E025E00198401EAE
:1009D0000006000E0190002882D10C4A012F17D189
:1009E0000021252016E000008CF200B0CCF20004BB
:1009F000D0F200047CF200B090ED0004ECF10004B1
:100A000008F20004ECED0004F0F10004B62E497089
:100A100001000000FCFF00A0000200008D66666877
:100A2000F8F1000400212620126890474FE70000EB
:100A3000FF4810B5016B490849000163FC4840308C
:100A40000169490849000161F94880300168490895
:100A500049000160F7480068804755204006026958
:100A600002218A430261C160F3480068804710BDDB
:100A7000EF4A01218032030000B539F364ED090625
:100A80000B0A1115061106110A00E94A106B0843FA
:100A9000106300BDE648403002690A43026100BDB0
:100AA00010680843106000BD90690843906100BD64
:100AB000DF4B002A10B505D1002903D05A681C0667
:100AC00022435A60002902D00121490701E0012197
:100AD000C9070843586010BDF8B5D54B9A6B202460
:100AE000A243C5070124002D01D0224301E0520892
:100AF00052009A63CE4B40331A6A0225AA438607F6
:100B000001D5224301E0520852001A62C84B8033DB
:100B10001A6AAA43FF256D1CAA43050701D5224383
:100B200001E0520852001A629A68450701D5224333
:100B300001E0520852009A605526BE4DBE4F76061F
:100B4000002807D12868804730694008400030619C
:100B5000F4600EE000070ED0002904D0002201212D
:100B60000A20FFF7A5FF28688047F460306920431A
:100B7000306138688047F8BDAD48416802061143CE
:100B800041607047704755225206516B20239943AC
:100B9000400101431820814351637047F8B50600B6
:100BA0000020FFF7F0FFA548C06A0121490508436E
:100BB00049008843A149C862552252061168102095
:100BC000014311609D4A9E49D1639E4AFF2108312D
:100BD00011609B49891F9162954CE36801210B4389
:100BE000E360002E02D1536A03435362904D803577
:100BF0002C6B914F84438F48002E06D100680C4324
:100C000080472C6338688047F8BD0600006880473D
:100C1000286B20210843286338680C43145C0625A0
:100C200001000000F80101A000020000BF0D01D783
:100C30008047306880472C6338688047FFF7A6FFFD
:100C4000F8BD70B506000C00FFF7FCFE7D4D803549
:100C5000002C04D000210800FFF748FF09E07A4883
:100C600000688047286B2021084328637748006884
:100C70008047286B400840002863002C08D0774844
:100C80000078032804D1042002F07AFC01F041FB33
:100C90006C48C16849084900C160002E05D0552143
:100CA0004906086802221043086070BD10B511F0B3
:100CB00082E9002802D0012108000CE011F05EE971
:100CC000032806D101210800FFF7BBFF11F076E9E8
:100CD00010BD01210020FFF7B4FF10BD55204006D4
:100CE0000168022211430160704770B50C000025B5
:100CF000030039F332EC090A1D2521250A0A0606EC
:100D00002500002C1CD1564C1AE0002C18D1554857
:100D1000407803280AD005DC002807D001280FD12D
:100D2000514C0DE0082801D00A2809D14F4C07E0AA
:100D3000002C05D14E4C03E0002C01D109246405A0
:100D40004C488078002801D14B4824184B488442F5
:100D500000D90400002A03D00125280001F073FB0C
:100D600060004008E907084336498860444901208B
:100D7000087070BD3348434941614349C161FF2157
:100D80000A310161816170472F4810B500688047C2
:100D9000552040060168012292029143016081685A
:100DA0000322114381600169FF22521C91430161BA
:100DB0000021816125480068804710BD264870B534
:100DC000403041680126314341604168B143416090
:100DD00055246406206830432060C046C046C046A3
:100DE000C046C046C0462068102108432060FFF777
:100DF000CBFF206808210843206000210800FFF78E
:100E000075FE134D40352869310208432861FFF70C
:100E1000B1FF002020613F20E0610D488030C168B3
:100E2000F82291431831C160184846719FFE47333C
:100E300001000000F40301A0000200009F69625459
:100E4000184800688047E96840208143E9602969C3
:100E500001432961034927E0400000AACCF20004C5
:100E6000D0F20004400100AA03060000000800AA16
:100E70002D5E00B0FF0F000080ED0004103506006D
:100E8000D4090000D008000483ED0004AC08000081
:100E9000FFFFFF0F045E00B0001000AA001200AABE
:100EA000001F00AABCF000044039086A072212069D
:100EB0009043AA0480180862D0132860FF48016B91
:100EC0003F2252069143EA048918016370BD70B550
:100ED0000500FA4CE06805D1F9480078032801D1F3
:100EE00001F021FA55204006016808229143016073
:100EF000416B202291434163F348F249D2000160E3
:100F0000F24B2B214905D963F1498162EB4840300E
:100F100081681F231B02994305235B02C918816066
:100F2000A06B80218843A063002D05D1A0691043E8
:100F3000A06120691043206170BD0021080010B538
:100F4000FFF7DEFDFFF788FDFFF71EFF5520400687
:100F50000168082211430160D949002048700870D7
:100F600010BD10B50400002155204006C0694200A4
:100F7000D20D8002400F02D0521C1204120C002A23
:100F800006D0D44822600168D34839F302E9012130
:100F9000002902D10020206010BDCF4810BDF7B558
:100FA0000D00C64FB869FF21491C0843B861386974
:100FB00008433861C94800992A0039F3EAE8022059
:100FC00055267606F060C6480068804730690224DE
:100FD00020433061C34800688047C3480678FEF765
:100FE000CAF9002804D1029900223000FFF787FED9
:100FF0003300B24EFF21090228020122803639F364
:10100000B6EA09063463404A064006406300AB4B2B
:101010001E6BB54F00237F78002F04D101231B06E0
:101020001E43102302E001273F06BE438E430643C2
:10103000F0208643AD4816432643864334C94EEF1D
:1010400001000000F00501A000020000521D611A1D
:101050009F4806630099097850290ED020210B4340
:1010600013439B4A80218B43403291681F24240202
:10107000A143052464020919916083632EE0944A18
:10108000403213698B43034323431361106A4008C2
:101090004000106222E03368E027BB43A0338B435B
:1010A000034313432343336018E0B7698F43074377
:1010B00027431743402087439248007801280CD0EB
:1010C000B06940084000B061FFF774FDF06A00228B
:1010D000000100090121FFF709FDB761002000E0D0
:1010E000401CA842FCD3FEBD7948C0684006800F72
:1010F000072800D908207047FFB5022055241D009D
:10110000640681B0E0607B48006880472069022661
:10111000304320617848006880476D4FB869F1011D
:101120000843B861386908433861FEF72EF90400B6
:101130006D4800210838012D02D0022D02D100E0B7
:1011400001210170002C03D06F480078042826D1BB
:10115000002D1FD000210800FFF7DCFC022D19D163
:10116000B86869070843B860002001F080F92020C2
:1011700055214906C8605F480068804755204006F1
:101180000069202188435521490608615A480068B2
:10119000804704E0039902980022FFF7BAFD019806
:1011A0004B49029B0002403139F3EAE909063FB49A
:1011B0005F70065F065FB4003B6B504842780120C9
:1011C0000006002A01D1034300E08343FF20000210
:1011D0008343019821220006000C03434848E03075
:1011E0008343334301201F2603433602002C09D1D9
:1011F000FFF77AFF002805D18868A122B0430126B5
:10120000360303E08868B0430526760280198860BB
:101210003A484078002801D110200243BA633B636A
:10122000086940084000086118E02949403109690F
:101230000122FF2311431B02994301433143012C37
:1012400005D1234B4033186A1043304353A79A63A8
:1012500001000000EC0701A000020000DFA1A55280
:101260001862204840300161386B40084000386304
:101270001C488030016849084900016054E0A02200
:10128000024301200243174832438030026008695C
:10129000400840000861386B40084000386343E074
:1012A000104F8037B969019B4022002B01D11143B7
:1012B00000E09143FF2212029143014303200143C6
:1012C000B8690E0040084000B861FFF77DFCF86A7D
:1012D0000022000100090121FFF712FC012C22D19C
:1012E000386A1DE0400000AA2D5E00B010830000A7
:1012F000000800AA400100AAFD0500000C5E00B035
:10130000A4F200B0001000AACCF20004D0F2000455
:1013100080ED00040C008000365F00B0A4F500B042
:10132000032108433862BE61002D0DD002980428C5
:101330000AD0002C03D0FB480078042804D10022F6
:1013400001210A20FFF7DCFB05B0F0BD7FB50028C6
:10135000F54D2CD001AA02A903A86B4604F00BFDA1
:101360006B46187A002803D0FF21FD31880002E087
:101370000121490288006B461A7B0400002A02D131
:1013800089008000A4004A00852312185B01D2184E
:101390006B461B79022B04D16023594308180019AE
:1013A00082182C68042100200123A0477FBD002261
:1013B000042110002C680223F7E755204006C0697D
:1013C000DA494000C00D8880C88008007047D749BE
:1013D00000201031C88008007047D5488169FF227D
:1013E000521C11438161704755204006C0690006B8
:1013F000C00F704770B50126360303207500000347
:1014000055246406E060CB4800688047206930437B
:1014100028432061C8480068804770BDC54810B5A2
:10142000006880475520400601690322120391435A
:1014300001611100C160C0480068804710BD70B5EF
:101440000500BC4800688047B64C2034A0780128CD
:1014500002D0022806D101E0FFF7B6FBB4BB22E9B7
:1014600001000000E80901A00002000061ECDDFAC3
:1014700000210800FFF70DFCFFF7C6FF0320A07056
:10148000B34900222800FFF758FC202055214906C7
:10149000C8600869202210430861FFF7AFFFA94A1E
:1014A00000280ED00B69012003430B61072D14D0D7
:1014B000082D04D1A34B803399680143996004201F
:1014C000A070906801214907084390609A49002064
:1014D000C8719E480068804770BD916B014391635D
:1014E000EDE7984800B5016B490849000163016BBD
:1014F0000122114301631B2000220121C001FFF7DB
:1015000009FB00BD00B5FFF705FB00BD002211007F
:1015100000B5FFF7FFFA00BD8A4810B580680401E6
:10152000240905F028F8002801D08A48807A00288C
:101530000AD001280ED0022818D0032810D101208B
:101540000004854900190AE001208349C0040019FC
:10155000383104E001208049800400191831441812
:10156000002211002000FFF7D5FA10BD01207A49B2
:10157000400400190831F2E710B5724A040008006F
:10158000116B4908490011636E4A403211694908DC
:10159000490011616B4A80321168490849001160A5
:1015A0009169490849009161FFF794FAFFF716FB2A
:1015B000002201212000FFF7ADFA10BD70B50D002B
:1015C00060490400C031886A644AC008C000C01C79
:1015D0001040FF22D20080180322120490430A0216
:1015E000801888620020FFF70BFB002D04D001F06B
:1015F00036F88007400D0419102055256D06E86067
:101600005148006880472869102108432861012259
:1016100011002000FFF77EFA02F096F8514BE10925
:101620001C681F314E4A0023A0474F490120087013
:1016300046480068804770BD002810B505D1414874
:101640008169FF22521C114381613F480068804735
:101650005524640620691021884320613B480068B6
:101660008047E0694009C00704D0E069BA6FEE2DF9
:1016700001000000E40B01A0000200004188BE79D7
:1016800020210843E061012010BDF7B584B000249B
:1016900007001B20019006982500260004280394CB
:1016A000029403D00599380000F0D8FD2A4903229E
:1016B000069BFC201203803138F380EF090680CFAF
:1016C000DCFA06DC06DC4700002F61D0012F63D076
:1016D000022F66D0032F02D1294C2A4D2A4E1E4AD2
:1016E0004032D3681B0F1B072343D3601A4BDD63C3
:1016F00016605568AD0AAD02FF3531355560059A63
:10170000002A53D0012A54D0022A54D0032A00D1EF
:10171000164C5A6B120F120722435A634A6B8243CC
:10172000FF20000282430120C0031018032210434F
:101730004863886B154A1040032212068018800BFC
:10174000BF228003D20080188863D4E0A4F500B0E3
:101750005CF100040C5E00B0400000AACCF2000472
:10176000D0F20004FC3F000067DF00045C040000CE
:101770000780FFFFE72C010030F30004305E00B06B
:10178000441A00000A121A02131B2428FFFF00C08B
:10179000F84CF94DF94EA2E7F64CF94DF94E1B3CC9
:1017A0009DE7F44CF84DF94E2B3C98E78324E40078
:1017B000AFE7F74CADE7F64C103CAAE7002F33D06B
:1017C000012F36D0022F39D0032F03D1F14BF24D28
:1017D000F24E03934B6B8343FF20C83300028343D5
:1017E0009818032210434863886BED4A1040052285
:1017F00052058018800B8003A0308863E949039864
:1018000008624D628E62086BE74A000F000780187D
:1018100008630598002816D0012816D0022818D091
:10182000032818D0029812E0E04BE14DE14E0393FB
:10183000D0E7E14BE14DE24E0393CBE7E14BE24DC4
:10184000E24E0393C6E7E24800E0E24802904861B6
:1018500051E0E148FAE7E148F8E74B6B8343FF20AA
:10186000C833000283439818022210434008400006
:10187000486340E01F230193A7231B01A190BAA94D
:1018800001000000E00D01A0000200008CFCBD374B
:101890004B6067239B01CB600B614B6B8343FF2045
:1018A000C833000283439818032210434863886BAF
:1018B000C04A1040052252058018800B8003A030DA
:1018C0004CE7FFE7086A20221023042F01D1904340
:1018D00006E0052F01D1904307E0062F02D1104307
:1018E000984303E0072F01D1104318430862C869E9
:1018F000020F8320120740011018C861C86A020F46
:1019000021201207C0011018C862AB498031C86994
:10191000B84A1040019A12041043C86107B0F0BDE4
:10192000B54B10B501241C7058709970DA7010BD59
:10193000B14A1378002B04D10822027000200A70EB
:101940007047537803709078087001207047F3B5A2
:1019500003009948C030C16B012500222D050327E3
:1019600014006E107F0538F334EE0906150A151DB4
:10197000061506150A00019A002A0BD103E0002A79
:1019800006D0002C02D1A943314305E0002A05D13D
:10199000002C0AD02943B143B94306E0002C04D0FF
:1019A000002A02D0A943B1433943C163FCBDF7B556
:1019B00082B00026029837003400350009280196CD
:1019C00002D00398092802D10020029003900399C5
:1019D000029800F04DFC7848049B403038F3F8ED55
:1019E00009064B36CAD206CA06CA36006D4A6D4B86
:1019F00002986C49103A183B002828D001282BD0B7
:101A000002282DD0032802D17C4C7D4D1E006A484F
:101A1000C7683F0F3F073743C760674F403FFC63CE
:101A200005604468A40AA402FF343134446003987A
:101A3000002819D001281AD002281AD0032800D172
:101A40001E00786B000F0007304378639AE4554E10
:101A50004E4C4F4D1736DAE76A4C6B4D0E00D6E709
:101A60006A4C6B4D1600D2E74E4E5B3EE9E70E0026
:101A7000E7E71600E5E70023029E180019001A00A8
:101A8000002E59D0012E5BD0022E61D075FE138B33
:101A900001000000DC0F01A0000200005E302B5EA0
:101AA000032E06D10223604F604D614C18001900CF
:101AB0001A00604E3E40BF01BF0DFB181B041E43C1
:101AC000E30A6405640DDB02241A23435A4C5B4F7E
:101AD0001C401B03DB0D5B1ADB021C43230064006C
:101AE000640DA41A3B4024052343EC0A6D056D0DDB
:101AF000E40228180443504820402403E40D6118F0
:101B0000C902084304004000400D304980183C40A1
:101B1000000504430E624B628C628869FF22120446
:101B200090430B22D20480188861086B444A000F4E
:101B3000000780180863039800281BD001281BD0D9
:101B400002281DD003281DD0019817E03D4F3E4CC0
:101B50003E4D02E03E4F3F4C3F4D10231800190010
:101B60001A00A6E70423180019003C4F3C4C3D4DD9
:101B70001A009EE7204800E02048019048610BE4ED
:101B80001F48FAE71F48F8E73521C90141601521D0
:101B9000C901C160016163E766E00000771A0000D7
:101BA00066A6E60299D917D92E4E6E024F6F90881D
:101BB0001626360227374848740400000007030041
:101BC000090890000C20C000FFFF00C0800000AAA0
:101BD0008C150000003F11004F78F00459C89005A3
:101BE000001F0900273870022D68D002000F050081
:101BF00013183001173870010005085080020428BE
:101C000040010214A000010AFFFF00F0065E00B0D0
